:1000000000400020F18600003187000033870000A7
:1000100000000000000000000000000000000000E0
:100020000000000000000000000000003587000014
:100030000000000000000000378700003987000042
:100040003B870000BD5F00009D8A00003B870000E9
:100050003B870000000000003B8700003B8700005A
:10006000ED3C0000718E00003B8700003B870000E4
:100070003B8700003B8700003B8700003B87000078
:100080003B870000218B00003B8700003B8700007E
:100090003B8700003B8700003B8700003B87000058
:1000A0003B8700003B8700000000000000000000CC
:1000B0000000000000000000000000000000000040
:1000C00010B5064C2378002B07D1054B002B02D02E
:1000D000044800E000BF0123237010BD700200201F
:1000E000000000005CFD0000044B10B5002B03D0A5
:1000F0000349044800E000BF10BDC04600000000F6
:10010000740200205CFD0000164B002B00D1144B44
:100110009D46402292029A1A924600218B460F4633
:100120001348144A121A0CF0E1FC0F4B002B00D0BC
:1001300098470E4B002B00D0984700200021040068
:100140000D000D48002802D00C4800E000BF0CF064
:100150008DFC2000290008F0F3FC0CF061FCC04687
:100160000000080000400020000000000000000027
:1001700070020020D42F00200000000000000000CA
:1001800002000120104011D1042A0ED91368180969
:1001900080B2002809D001388000031D11180979A8
:1001A000002902D001309842F8D170470020FCE7C6
:1001B0000378002B03D05AB2002A01DB01307047CC
:1001C0003F229343C03B59424B41C01803789343AD
:1001D000802BF4D10130F9E710B500240378002B0F
:1001E00001D1200010BDFFF7E3FF0134F6E770B541
:1001F000002204000D00411C092004F09FF8002893
:1002000006D001236200134343600023A34200DBB6
:1002100070BD9A00A958821891600133F6E770B555
:10022000012803DC1C2001F0B7FA70BD01230D6822
:1002300011201D42F7D04868184206D1042804D97D
:100240000F2302681340042B01D00E20EBE703F0CC
:10025000D3FE6D100400002D03DDFFF7BDFFA842A3
:1002600006DA1220DFE72000FFF7A2FF0400013DBD
:10027000012DF8D120787F2809DDDF280BDCF82359
:100280003F22DB00800118406378134018430123AC
:1002900040001843C9E7EF280BDCFC226378120109
:1002A0009B0113403F220007000C0343A07810403D
:1002B000ECE7F72812DCFC22637892021B03134060
:1002C000E0228004520310403F221843E378134099
:1002D000FC220343A07812018001E8E7012040429C
:1002E000D5E7F8B54D680F00EB0706D4042D04D907
:1002F0000F232E683340092B03D00B2001F04CFA5A
:10030000F8BD6B683609B6B25C10731EA3420FD8F5
:10031000032120000AF0A6FA6421642803DC01000E
:10032000032800DA03212800891904F039F80500B0
:100330002B6800201B099BB2013B9C42E0D23A682B
:10034000A31C9B005A510123013464001C436C60C0
:10035000D6E7F0B585B0012803DC1C2001F01CFABB
:1003600012E001274B683A000093022806D08B6800
:100370003B4203D05F10002F00DC17000125009BDB
:100380002B4203D00120404205B0F0BD009B042B5E
:10039000F8D91B680C680F261900314004292DD1AB
:1003A0002C4205D1042C03D923681E40042E01D011
:1003B0000E20D3E70098FFF7E3FEB842E2DB009897
:1003C00003F01AFE0600200003F016FE0378010079
:1003D000002BD7D0781E30180CF03EFF041ED1D071
:1003E0003378002B01D0A64202D36800012521E01A
:1003F0003000FFF7DDFE01350600F1E709293ED1A7
:10040000009B5B685B1001939F42BBDC2C422ED1AA
:10041000042C2CD923683340042B28D1200003F06E
:10042000EBFD039602907E1C009AB300D0588442E4
:1004300002D178002843A7E728420ED104280CD91E
:100440000368039A1340042B07D103F0D5FD010084
:1004500002980CF0CBFE0028EBD0019B37009E42A7
:10046000E1DD8FE71F00019B9F4200DD8AE77B1CD7
:1004700000999A008A58A242F4D17800B6E703297D
:1004800000D07FE71A0992B25B0F92000B40D31A9B
:1004900001939F4200DD75E72C4229D1042C27D916
:1004A00022681640032E19D1100980B2520F800025
:1004B0003240251D801A019B2E181B1A0193009BA8
:1004C000781E0433019A904200DD5BE72A00191878
:1004D000B2420FD316D10130400087E7042E07D176
:1004E000200003F089FD05002000FFF749FEE2E748
:1004F0000F2033E70C78A4461478A44502D10131CB
:100500000132E5E70130DDE7F0B50D0085B00128E7
:1005100004DC1C2001F040F905B0F0BD012708689B
:10052000384206D1042804D90F2102680A40042A5F
:1005300001D00E20EEE76A681740FAD1042AF8D9F4
:1005400013680B40042BF4D103F056FD04006868D7
:1005500003F052FD02900CF053FE039000280FD1DF
:100560002000FFF739FE0190019B0122591C092050
:1005700003F0E4FE364E3060002815D10020CBE7B2
:10058000029920000CF068FE001B4342434120000A
:100590000193019B5E1C0028E6D0039B0299C018C2
:1005A0000CF05AFE0196F4E70122019B5B00134315
:1005B0004360039B002B18D12000FFF7F9FD019B3E
:1005C0000500BB4201DC3068A6E7291B200003F0D0
:1005D00033FF0028D2D0BB1C32689B009850280003
:1005E000FFF7E6FD01372C00E9E7019B012B02D163
:1005F0002B68836090E7029920000CF02DFE012506
:100600000700019B002F13D0AB42DCDB391B20001D
:1006100003F012FF0028B1D032680135AB009850CA
:10062000039B0299FC1820000CF016FE0700E8E777
:10063000AB42C8DB20000CF0E3FD0100200003F01A
:10064000FBFE00289AD001353368AD00E850BAE7C8
:10065000E40F002010B503F0B3FC43000120184361
:1006600010BD0000C30711D404280FD90F2302685E
:100670001340032B0AD119400133591AC0234907EB
:10068000DB051940024B1A40114301607047C04618
:10069000FFFFFF9F70B5002805DC1C2001F07CF8EF
:1006A0000500280070BD01220C68144201D10D2004
:1006B000F4E701281CD04B681342F8D05B101320DC
:1006C000FF2BEBD81A0619040A431A431B021343E3
:1006D0006410E243D2171440E11C89101A00032071
:1006E00003F02CFE051EDCD02100FFF7BBFFD8E78E
:1006F0000023EDE7F7B507000E001C20012F06DDF3
:100700004C68012322001A40009203D10D2001F011
:1007100043F853E0022F02D08A681A42F6D0012330
:1007200035681D4200D0A9E0042D00D8A6E01C4188
:10073000002C00DC1C000F2029680840092828D163
:100740006B685B100093022F05D0B368009A5B10B2
:100750009A4200DD0093009B01221D1B0135EB43F3
:10076000DB171D40691C092003F0E8FD071E09D0B6
:1007700001236D001D430300326808334560009972
:10078000A14201DA3800FEBD0134A100515802C374
:10079000F5E7042845D1280003F02EFCFFF71CFDE7
:1007A0000190022F04D0B3685B10984200DD0193E2
:1007B000019BA34204DA002003F032FE0700E1E7C8
:1007C000280003F019FC0700009BA34221DB28004E
:1007D000009703F011FC05003800FFF7E9FC019BCE
:1007E00001340700A342F7DA009BC41A200003F08B
:1007F00017FE071EC6D003F0FFFB0190306803F020
:10080000FBFB2200009B591B411801980CF052F988
:10081000B8E73800FFF7CCFC009B070001330093DA
:10082000D2E703282AD10B099BB2490F9B00014054
:10083000591A022F04D0B2685210914200DD110003
:10084000A14205DA00220320110003F077FDB5E78D
:1008500003200E1B331DD9170140C918891000222F
:1008600003F06CFD071E00D18CE701363100033424
:10087000FFF7F8FE381D29193200C7E7212046E7A7
:10088000F7B5002804DC1C2000F086FF040014E00B
:100890000D6801272E003E4011D03D41FF2D01D9AA
:1008A0001320F1E700223900032003F047FD041E66
:1008B00003D03900FFF7D6FE25712000FEBD042DC0
:1008C000EED90F232A681340042B1BD12800FFF711
:1008D00057FCC31C07000320D9170140C918891011
:1008E000320003F02BFD041EE7D03900FFF7BAFEFB
:1008F000280003F081FB231D01003A0018000CF0D2
:10090000D9F8DAE7092B1FD103206B6832005B109E
:1009100001930333D9170140C918891003F00EFD64
:10092000041ECAD00199FFF79DFE019B9E42C4DAC6
:10093000B300EB189B683B4204D05B10FF2BAFD891
:10094000A21913710136F0E7032BA9D12C00B4E7EB
:1009500010B57F2902DC0170013010BD1A4B99429D
:100960000CDC40238A115B42134303703F230B408E
:1009700080214942194341700230EEE7134B9942FE
:1009800010DC20230A135B4213433F2480220370B0
:100990008B1152422340214013430A43437082701B
:1009A0000330DAE70A4B9942D7DCF0230370603B4F
:1009B0004370113B8A11FF3B1A4382703F22114062
:1009C0001943C1700430C8E7FF070000FFFF0000B3
:1009D000FF0F010010B50124044002D04410200094
:1009E00010BD042810D90F2302681340042B07D12F
:1009F00003F002FB21000A220CF0CAFC0400EEE71F
:100A0000032B01D10430F5E70D2000F0C5FEE6E729
:100A1000F0B50E0085B0002803DC1C2000F0BCFE01
:100A200017E00F6801243D00254006D1042F1ED990
:100A30000F233A681340042B0DD13800FFF7CAFF8B
:100A400002AC01002000FFF783FF011B200003F030
:100A5000F3FC040032E0092B09D17B685B100193A1
:100A6000019B9C4205DD00F09DFE002819D02A2044
:100A7000D4E70134A300F858FFF7ACFF01237F2827
:100A80000DDD154ADB18904209DD144A013390420E
:100A900005DD0021124AC30F82424B419B00ED1835
:100AA000DEE7280003F0BCFC041E07D0376803F023
:100AB000A3FA01250600019B9D4202DD200005B03E
:100AC000F0BD0135AB00F858FFF784FF010030009E
:100AD000FFF73EFF0600EEE7FF070000FFFF000004
:100AE000FF0F0100F7B5030001900E001C20012B41
:100AF00011DD0868FFF76EFF07007068FFF76AFFF7
:100B0000019B05000124022B08D0B068FFF762FFAB
:100B1000041E03DC292000F03FFEFEBDAF421CDCBA
:100B2000E81B210009F09EFE451C691C00220920DB
:100B300003F004FC0028F0D001226B001343436053
:100B40009440002379009D42E7DD17009E000F438B
:100B50008619B76001330919F5E7781B210009F000
:100B600081FE6442451CE0E710B504000120084006
:100B700010D104290DD90F230A681340042B08D182
:100B8000080003F039FA010020000CF02FFB43426B
:100B9000584110BD0020FCE7F7B50E00012803DC2A
:100BA0001C2000F0F9FDFEBD4D68EB0706D4042DB6
:100BB00004D90F222B681A40092A01D00B20F0E734
:100BC0006A681B099BB25410A34200D85C1E01271F
:100BD00031680F404810002F35D12648FFF7C4FF79
:100BE00001230190002813D131682348FFF7BCFF8F
:100BF000002811D0002C0DD00122631C013C944030
:100C00009B005A5114436C6004E00137BA00AB50AA
:100C1000BC42FADA0020C6E701233068184223D12B
:100C2000042821D902680E331340042B1CD1FFF78E
:100C3000D1FE002807D131681048FFF795FF002842
:100C400012D01220ADE70028FBDD8442F9DB8300DF
:100C5000EB180433844209DC0123621C013C9C40F4
:100C6000920053511C43CEE711209AE75A68013095
:100C70001A60EEE797E100009BE1000049F40000F4
:100C8000002310B50C000B70C30705D50D494210A9
:100C900020000CF06FFA08E00B49002802D004286D
:100CA00004D10A4920000CF085FA10BD0428FCD9B3
:100CB0000F2302681340042BF7D103F09DF9044978
:100CC0000200E5E720EE0000A0E10000A6E1000040
:100CD000ABE10000F0B593B0060002911C20012E9C
:100CE0001DDD029B01251B681C002C4000D0ADE0DF
:100CF000042B00D8E6E01A680F231A40092A4AD1CB
:100D00000394039A029992008A5817002F4005D144
:100D1000042A03D910681840092806D0222000F0C0
:100D20003BFD0190019813B0F0BD52685210A41819
:100D3000039A013203929642E3D1611C012203F02F
:100D4000FDFA0190002802D100230193EAE7019BFC
:100D50006400190025435D600831029ABB00D05839
:100D600002684368120992B25B109A4200D8531E7F
:100D70000022934209DCDA43D21713409B00C918C2
:100D8000039B01379F42E8DBCCE794000519AD686F
:100D900001320D51EDE72700032A59D10193029A40
:100DA000BB00D3582B42B9D1042BB7D9186801998D
:100DB0000140032939D1020992B2430F92000B403E
:100DC000D31A1C190137BE42E9D10320E31CD917FD
:100DD0000140C9188910002203F0B0FA01900028E0
:100DE000B2D000252100FFF73DFC019B1E1D029A99
:100DF000AB00D45801231C421FD1042C1DD90F2154
:100E000023681940032918D1180980B25B0F8000AC
:100E10000B40C01A0023834213DBC343DB17184087
:100E200001353618BD42E2DB7CE7042900D075E7C6
:100E30001800FFF7A5F92418C4E72000FFF7A0F970
:100E4000E8E7E2181279F2540133E4E700273C00A6
:100E50000F25029ABB00D3580122134234D1042B30
:100E600032D9186801002940042935D11800FFF74C
:100E700087F924180137BE42EBD1200003F0D0FAE5
:100E80000190002800D15FE7029FB600BB19041D46
:100E9000029301233D681D4229D1042D27D90F2635
:100EA0002B681E40042E37D12800FFF769F9060091
:100EB000280003F0A1F80100200032000BF0FAFD39
:100EC000A41922E02700C3E7180005A9FFF7D8FE00
:100ED00005A80CF095F9CCE7032900D01EE702091C
:100EE00092B2430F92000B40D31A1C19C2E705A916
:100EF0002800FFF7C5FE05A80CF082F905A905003A
:100F0000020020000BF0D6FD6419029B0437BB429F
:100F1000BFD10023237005E7032EF6D11A0992B240
:100F20005B0F92001E40961B291DC5E7F0B50D0012
:100F300097B0002806DC1C2000F02EFC07003800CB
:100F400017B0F0BD0C68012123000B40009306D1BF
:100F5000042C04D922680F331A40092A01D00B202F
:100F6000EAE7626852100392002A03DC009803F05B
:100F700057FAE3E7504A019201280BD0686808420B
:100F800008D1042806D902681340042B02D103F0CB
:100F900033F8019001980CF033F906000F27039BFA
:100FA0000834013B05935E43039B02909B00E318CA
:100FB000049301232068184273D1042871D9016871
:100FC0000B003B409C46042B03D1FFF7D9F8861950
:100FD00009E0032B6CD162460B099BB2490F9B00C1
:100FE00011405A1A9619049B0434A342E1D13000EF
:100FF00003F016FA071EA2D02B680793029B002B62
:1010000003D0686802F0F8FF0190380002F0F4FFA6
:101010000400009B079A9B00D3189E68300002F0E2
:10102000EBFF0123334005000693002B01D1042E72
:1010300004D809A93000FFF723FE09AD28000CF001
:10104000DFF8069B0490002B0ED1042E0CD90F2143
:1010500033681940032907D11A0992B25B0F920035
:101060000B40D31A351D04932000049A29000BF07D
:1010700021FD049BE418029B002B0AD0059B009ADB
:10108000934206DD2000029A01990BF013FD029BAA
:10109000E418009B01330093009A039B9342B8D15C
:1010A0004DE709A9FFF7ECFD09A80CF0A9F88EE7B8
:1010B00002F0A2FFF9E7C046F3E6000010B50122F6
:1010C000002400280BDD0B681A40141E03D05C10AE
:1010D000E343DB171C400122904200D04A68611CA8
:1010E000092003F02BF9002803D0012364001C43DE
:1010F000446010BD0A6870B510000125284034D145
:10110000042A32D90F24136849681C40092C17D1CE
:1011100054681B099BB22C41A34200D85C1E844238
:1011200005DC02200133984206DB00200FE0850039
:101130005519A9600130F2E7840011510130F2E73E
:10114000032C12D1294203D1132000F025FB70BDDE
:101150004910FF29F8D81B099BB204329B00D31811
:101160009342E2D911700132FAE70B2000F014FB30
:10117000DBE700000123F7B500254E680C00334083
:101180000193AB420ED11D00042E0BD90F22336800
:101190001A40092A26D172681B099BB25510AB422E
:1011A00000D85D1E27687C10FB0746D439003D48F7
:1011B000FFF7DAFC002826D00BF078FF290009F0B1
:1011C00037FC4C1C019B002B00D069E0042E67D932
:1011D00032680F331340092B3BD10134A400A459CA
:1011E0002000FEBD042A04D13000FEF7C9FF05002F
:1011F000D8E7019D032AD5D11D09ADB25B0FAD0023
:101200001340ED1ACEE739002748FFF7ADFC002860
:101210001DD1042F16D90F233A681340042B11D186
:101220003800FFF7D7FB041E07D139001F48FFF72E
:101230009BFC002806D0122005E0002CFBDDA54217
:10124000C0DAF8E7112000F0A7FA0400C8E72C0084
:10125000B8E7042B1CD1300002F0CEFE0500012CB3
:101260000EDCFEF7A5FF461B300003F0D9F8041E84
:10127000B6D002F0C1FE320029000BF01BFCAFE734
:101280002B78013C002BD6D02800FEF791FFE5E734
:10129000032B05D13419E37801245B001C439FE73D
:1012A0000B20D0E790E100009BE1000049F4000032
:1012B000F7B54D680E002A0001210A402FD1042DF8
:1012C0002DD90F242B68B7681C40092C14D16968EC
:1012D0001B099BB24C100192A34200D85C1E3168DE
:1012E0003448FFF741FC00282DD00F232A68134013
:1012F000092B1DD1012317E0032C10D10F4203D17C
:10130000132000F049FAFEBD7A100192FF2AF7D8A7
:101310001A0992B25B0F92001C40141BDFE70B20EE
:10132000EFE701339A00AF509C42FADA0020EAE777
:10133000032BFBD12B0001335A1BA242F6DC6A4679
:101340001279DA70F7E736687010F30719D43100B4
:101350001948FFF709FC002822D1042E1ED90F23BB
:1013600032681340042B19D13000FFF733FB0028FB
:1013700007D131001148FFF7F7FB00280ED01220EB
:10138000BFE70028FBDD8442F9DB0F232A68134006
:10139000092B07D1013080004751C7E71120B0E782
:1013A0002000F2E7032BC1D16B461B792D18EB709F
:1013B000BCE7C04697E100009BE1000049F4000053
:1013C00070B501240868204207D1042805D90F25EB
:1013D00001680D40092D02D14468200070BD032D25
:1013E00008D10A0992B24B0F92002B40D31A5B002E
:1013F0001C43F2E7042DF0D102F0FEFDFEF7ECFEF7
:1014000040000443E9E7000010B5034A0E210348F9
:1014100004F0D2FE10BDC04620E1000018E100003B
:1014200000207047042070470120704710B500204D
:1014300002F0F6FF10BD002070470020704700202A
:101440007047002070470020704700207047002040
:1014500070470020704700207047000010B5034A15
:101460000D21034804F0A8FE10BDC04638E200007C
:10147000A0E2000070470378002B03D05AB2002A84
:1014800001DB013070473F229343C03B59424B413F
:10149000C01803789343802BF4D10130F9E70000A2
:1014A000F8B50127060014000800394227D10429A5
:1014B0003FD90F230A681A40042A3AD13C4213D17B
:1014C000042C11D922681340042B0DD102F094FD95
:1014D0000500200002F090FD010028000BF086FEC0
:1014E00000282EDB1FD127E0E30722D502F084FD80
:1014F0000A2200210BF04CFF0500601010E017409D
:1015000015D1042A15D90F2312681340042B10D1CA
:1015100020004D1002F070FD0A2239000BF038FF58
:1015200085420EDB08DD002E09DC00200CE04D10AA
:10153000E3E70F22054B1A700136022EF5D804207E
:1015400002E0042076173040F8BDC046B00200200B
:10155000F8B5060000242B4BE500ED182B79032B82
:1015600009D00134FF2CF6D1300004F039FE041EFE
:1015700046D1013C44E030000BF042FEE3B20200F1
:101580003100180004F0ACFE002839D12A685168F7
:101590008842E6D08300D3189B680130F02BF7D146
:1015A00001238000083012181A42DAD1042AD8D94F
:1015B0000F21136819400429D3D11B0998B20123C4
:1015C0000130800010181842CBD10428C9D90F224D
:1015D00003681340042BC4D102F00EFD032705005D
:1015E000092128000BF0F4FD0028BAD0013F451C6A
:1015F000002FF5D1310028000BF02EFE8542B0D12E
:101600002000F8BDA825002010B50124044002D018
:101610004410200010BD042810D90F230268134085
:10162000042B07D102F0E8FC21000A220BF0B0FEE7
:101630000400EEE7032B01D10430F5E70D22014B46
:101640001A70E6E7B0020020012210B5024018D15E
:10165000042802D903681A0992B201230B4012D15F
:10166000042902D90B681B099BB20024934206D1BE
:1016700004309B000431C318984206D30124200093
:1016800010BD0022E9E70023EFE704780A78002C78
:1016900001D1002AF2D0013001319442ECD0002473
:1016A000EDE70000F7B50700009101933049314B99
:1016B000002A02D002220A70013A00261A601B6832
:1016C000CE54BE4200DBF7BD009AB300D058294B80
:1016D000274D1C68C8239B0065191C1B0123184259
:1016E00006D0254A4310210028000BF011FD09E027
:1016F000224A002802D004281BD1214A21002800B8
:101700000BF006FD1A4C20000BF07AFD194A019BE4
:101710001060002B0BD07B1EB34208DD194B9842A2
:1017200005D8431C1360202222540022E2540136C3
:10173000C7E7042819D90F2301680B40042B04D1F3
:1017400002F05AFC104A0300CDE7092B03D143688D
:101750000E4A5B10C7E7032B08D10A0992B2490F62
:1017600092000B40D31A0A4ABDE70123094ABAE79F
:10177000B1020020D405002020EE0000A0E100000E
:10178000A6E100001F0300004FF4000018E5000070
:1017900027E5000032E50000014B1870002070477B
:1017A000B0020020024B1878431E98417047C04693
:1017B000B0020020002310B51A00FFF773FF034B9F
:1017C0000348196805F0F1F9002010BDD405002088
:1017D000B102002070B502F0AFF9094C0100251DDF
:1017E0001F2228000BF024FD28000BF009FD042324
:1017F00004308008000118432060200070BDC046FE
:101800008C020020C368F0B59D00836889B05D1923
:101810000300183306930369069A9F00069B029003
:10182000DF19436901939B00D3180393D04B1B78B6
:10183000002B26D17F222B68CE491C1213409B001F
:101840005B58043501929F46029B587805F08CF94D
:101850000023029A137027E0C54B1B78002B10D190
:101860002B68019A1C121340C24A9B009B580435F6
:10187000E9E7069B3A1DD11ABD4BD82928DD1A226B
:101880001A70029BBA4C9B6821780193EA1A029B5A
:1018900092109B7812021A43029B587805F06CF95B
:1018A0000023029A23701370029B069A9B6801938F
:1018B000ED1A029BAD10DD60069BFE1A029BB6106E
:1018C0001E61039B9B1A029A9B10536109B0F0BDE5
:1018D00039001B7817000C60002BD2D12B68019ABD
:1018E0001C121340A34A9B009B580435ABE7069B90
:1018F0003A1DD11A9E4BD82902DD1A221A70C0E770
:1019000038001B7817002A68291D0260002B01D0BF
:101910000D00B6E76B68019A1C121340954A9B00B4
:101920009B5808358FE7069B3A1DD11A904BD82952
:1019300002DD1A221A70A4E73900A4001B782C19C2
:1019400017000C60002B9CD12B68019A1C121340CD
:10195000884A9B009B58043575E7069B3A1DD11AAF
:10196000834BD82902DD1A221A708AE73900170042
:10197000814AA400A2581B780A60002B00D080E79F
:101980002B68019A1C1213407A4A9B009B5804351D
:1019900059E7043F784B3A68A400E250744B1B7837
:1019A000002B00D06DE72B68019A1C121340714A7E
:1019B0009B009B58043546E76F4BA400E058FFF7A7
:1019C00023FE6B4B06001B78002B09D1043F3868BF
:1019D000FFF71AFE0123861976001E43664BE65078
:1019E000634B1B78002B00D04BE72B68019A1C122D
:1019F0001340604A9B009B58043524E7069B391D21
:101A0000CA1A5B4BD82A02DD1A221A7039E70698E7
:101A1000039C0122A04202D222000C3A1268380034
:101A20001B780F000260002B00D02AE72B68019A78
:101A30001C1213404F4A9B009B58043503E7069A3B
:101A40003B1D991A4A4AD82902DD1A23137018E758
:101A500006990398814218D202000C3A126847494D
:101A600052106418A41AA40022583A601F00404B78
:101A70001B78002B00D004E72B68019A1C1213403E
:101A80003C4A9B009B580435DDE61821117000226A
:101A9000EBE7069B039A934219D213000C3B1B6899
:101AA000364A5B10A418043FE41A3A68039BA4006A
:101AB000E2502F4B1B78002B00D0E2E62B68019AF6
:101AC0001C1213402B4A9B009B580435BBE618227E
:101AD000274B1A70EDE7069B039A934228D2274BB7
:101AE000043FE61814000C3C23685B10F31A9B00BB
:101AF0009858FFF789FD04903868FFF785FD246842
:101B0000049B6410341B1E18012376001E43039BA4
:101B1000A400E650164B1B78002B00D0B1E62B68D2
:101B2000019A1C121340134A9B009B5804358AE605
:101B300018220F4B1A70EDE7069B3A1DD11A0C4B79
:101B4000D82902DD1A221A709BE639001700039A81
:101B5000A400A2581B780A60002B00D091E62B68E5
:101B6000019A1C121340034A9B009B5804356AE6F5
:101B7000B002002018E30000A02D0020FDFFFF3F71
:101B8000043F039B3A68A400E250D64B1B78002B1D
:101B900000D076E62B68019A1C121340D24A9B00B3
:101BA0009B5804354FE6039BA4001C192368043F8F
:101BB00038685E10FFF728FD0123361876001E43B3
:101BC000C84B26601B78002B00D05AE62B68019A80
:101BD0001C121340C44A9B009B58043533E6069BF5
:101BE000A4003F1BBF4CBB420CD82378002B00D075
:101BF00047E62B68019A1C121340BB4A9B009B5876
:101C0000043520E6B94802F0E7F92378002B00D02C
:101C100037E62B68019A1C121340B34A9B009B586D
:101C2000043510E6A300ED18002C00DA3CE6AD4BBD
:101C30001B78002B00D024E62B68019A1C1213405D
:101C4000A94A9B009B580435FDE5043F3B68042BE3
:101C500004D1A300ED18002C00DA25E6A14B1B7877
:101C6000002B00D00DE62B68019A1C1213409E4AEF
:101C70009B009B580435E6E5043F3B68042B04D0E9
:101C8000A300ED18002C00DA0EE6964B1B78002B13
:101C900000D0F6E52B68019A1C121340924A9B0073
:101CA0009B580435CFE501233E1F306818420AD007
:101CB00018410138002809DB01234000A400184323
:101CC0002D193060F0E5FFF79FFCF2E7854B1B789C
:101CD000002B01D03700D4E52B68019A1C12134069
:101CE000814A9B009B5837000435ACE5069E03995A
:101CF000891B3E008910049106990C36711AD82967
:101D000002DD1A231370BCE53900FF2764007F0051
:101D10003C40FE3FFF3F3C430C60029C1278A468AD
:101D200003942D1B029CAD10A4782D022543BD40C9
:101D30003D434D600125049C370064002C438C60BA
:101D4000644602998C701B588B60002A03D00833BC
:101D50001D00039695E51D00019A9B680C351C1229
:101D60001340614A9B009B5803966CE53B1F1C681F
:101D7000039A069B934232D10A20E30711D4042C24
:101D800018D90F2322681340042B16D1200002F02B
:101D900033F90BF035FAC8239B00984200D918009C
:101DA0000630643004F0E4FA00280FD1043D069BAD
:101DB000039379E50720042CF3D02000431E9841BB
:101DC000FA234042FF3318400730EAE7029B210024
:101DD000587804F0E3FE0023029A1370E7E7039BB0
:101DE000039A0C3B1B6802995B109B00D31A0C3BB7
:101DF0001C601F1D1300083B1B685A108A70D2B26A
:101E00003B49D2005B0055589B0A029A9B009560A3
:101E1000ED18039B069A043B1B685B109B00D318CC
:101E20000393304B1B78002B00D02AE52B68019AD6
:101E30001C1213402C4A9B009B58043503E53B1FA2
:101E40001868FFF7E1FBA40006003F1B1E2827DCF3
:101E500000280DDC234B1B78002B00D011E52B68EC
:101E6000019A1C121340204A9B009B580435EAE457
:101E700001F04AFE033E361801F046FE1D4B801B62
:101E80009842F9D8174B1B78002B00D0F9E42B6847
:101E9000019A1C121340144A9B009B580435D2E44B
:101EA0000123029A137001F02FFE029B0A38861953
:101EB0005E60F9E43B1F1868FFF7A6FBA40006006C
:101EC0003F1B002818DC074B1B78002B00D0D8E400
:101ED0002B68019A1C121340034A9B009B5804353F
:101EE000B1E4C046B002002018E3000044E5000061
:101EF000A82500203F420F00D64B984203DD1D224B
:101F0000D54B1A70BDE40123029A137001F0FCFD59
:101F1000FA239B005E430A3E3018029B5860C3E4DC
:101F2000A300FF1A002320001A003900FFF7BAFBB4
:101F3000CA4ECB4C3168200002F07EFAC94B3168A2
:101F40001860200004F0DAFC3168200004F02DFE57
:101F5000C14B1B78002B00D093E42B68019A1C1214
:101F60001340C14A9B009B5804356CE4BA4BA40053
:101F70001B783F1B002B00D083E42B68019A1C12B6
:101F80001340B94A9B009B5804355CE4029804F066
:101F900053FAB14B1B78002B00D072E42B68019AE6
:101FA0001C121340B04A9B009B5804354BE43B1F66
:101FB0001B68002B58D13B0001260C3B18680640DB
:101FC0002FD046103A0001217300083A0B431360EA
:101FD000002E00DC95E0012173000B433A1F1360D3
:101FE0003B00083B1B680B419B1B04933B000C3BD5
:101FF000186808423BD0049BA4005B188B400B433D
:10200000039AA350944B1B78002B00D039E42B6823
:10201000019A1C121340944A9B009B580435FFF709
:1020200012FC04281BD90F2302681340092B02D18C
:1020300043685E10C6E7042B08D101F0DDFF03788A
:10204000002BBFD0FFF717FA0136F8E7032B06D1B4
:102050001609B6B2520FB6001340F61AB2E71922AB
:102060007D4B1A70FFF70DFC5B105E1EB0E7042875
:1020700042D90F2302681340092B05D1049BA40009
:1020800002339B001B58BBE7042B2BD1039BA400FE
:102090001B19079301F0B0FF0600049C0134012CCA
:1020A00010DC3000FFF7E7F9831B1800049302F0FF
:1020B000B7F9041E0ED001F09FFF049A31000AF018
:1020C000F9FC07E03178013C002906D112220C000E
:1020D000614B1A70079B1C6094E73000FFF7CBF947
:1020E0000600DCE7032B07D10122049BA400C018E3
:1020F00003795B00134383E71922574B1A70FFF7EC
:10210000C0FB04357EE7A300069AFB189B1AD82B68
:1021100008DD1A22504B1A70FFF7B3FB01221C0096
:102120003A600437631E002CF8DC4B4B1B78002B05
:1021300001D0FFF7A6FB2B68019A1C1213404A4AF4
:102140009B009B580435FFF77EFB069A3B1D9B1AAC
:10215000414ED82B03DD1A233370FFF792FB069B09
:10216000039AA40093422AD23B1F1868FFF74CFA47
:10217000011E21DD039B0C3B1A68521082421BDBBF
:102180009007801A394B4018C018039B8000C25832
:102190003B1B1A60304B3F1B1B780437002B01D0D0
:1021A000FFF76FFB2B68019A1C1213402E4A9B000D
:1021B0009B580435FFF747FB20233370EAE71823C9
:1021C000FBE7284BA4001A683B1B1F001A60224B38
:1021D00004371B78002B01D0FFF753FB2B68019AC3
:1021E0001C121340204A9B009B580435FFF72BFB21
:1021F0003A1F1368042B02D13A00A4002D19164B84
:102200001B78002B02D01700FFF73BFB2B680199CE
:102210001C120B4014499B005B5817000435FFF754
:1022200012FB043F3B68042B04D00023A4003B6056
:102230002D190437084B1B78002B01D0FFF721FB29
:102240002B68019A1C121340074A9B009B580435C7
:10225000FFF7F9FA80EE3600B0020020D405002026
:10226000B10200200800002018E30000FCFFFF3F3F
:10227000A3009C46F81A002C17DC1C220026D34B26
:102280001A706346FF1AD14B06601B780437002B87
:1022900001D0FFF7F6FA2B68019A1C121340CC4AC2
:1022A0009B009B580435FFF7CEFA002103685B10B2
:1022B00001268A008258164003D10D22C34B1A70A2
:1022C000DFE75210934200DD130001318C42EFDC56
:1022D0005E0001231E43D4E7A3009C46F81A002C9D
:1022E00017DC1C220026B94B1A706346FF1AB74B45
:1022F00006601B780437002B01D0FFF7C2FA2B6869
:10230000019A1C121340B24A9B009B580435FFF7F8
:102310009AFA002103685B1001268A008258164051
:1023200003D10D22A94B1A70DFE75210934200DA55
:10233000130001318C42EFDC5E0001231E43D4E721
:102340003B000122083B1968A40011421DD03B1F2D
:102350001B68134219D0114113410022994200DA3F
:1023600004323B1B1A60994B3F1B1B780437002B30
:1023700001D0FFF786FA2B68019A1C121340944A89
:102380009B009B580435FFF75EFA02203B1F1A683A
:102390004042FFF785F83E1B3060E4E73B00012038
:1023A000083B1968A40001421ED03B1F1A68024274
:1023B0001AD001415010CB0FD217884253413A1B1B
:1023C0009B001360814B3F1B1B780437002B01D00F
:1023D000FFF757FA2B68019A1C1213407C4A9B00A6
:1023E0009B580435FFF72FFA01203B1F1A68404223
:1023F000FFF756F83E1B3060E4E73B00083B1868E7
:102400003B1F1968A600BE1B0423814202D004288A
:1024100002D80023336016E001231842F9D10F23BC
:1024200002681A40042AF4D1033A1142F1D1042976
:10243000EFD90A681340042BEBD1FFF705F9431ECF
:10244000984180003060614BA4001B783F1B04372B
:10245000002B01D0FFF715FA2B68019A1C121340CC
:102460005B4A9B009B580435FFF7EDF93B00083BA6
:1024700018683B1F1968A600BE1B0023814202D0CA
:10248000042802D80423336016E001231842F9D14E
:102490000F2302681A40042AF4D1033A1142F1D101
:1024A0000429EFD90A681340042BEBD1FFF7CCF8CD
:1024B0004342584180003060444BA4001B783F1BCE
:1024C0000437002B01D0FFF7DCF92B68019A1C12AE
:1024D00013403F4A9B009B580435FFF7B4F93B007B
:1024E0000122083B1968A40011421ED03B1F1B6843
:1024F00013421AD05B104A10D80FC9179A424141B3
:102500003B1B89001960314B3F1B1B780437002BA4
:1025100001D0FFF7B6F92B68019A1C1213402C4A20
:102520009B009B580435FFF78EF93B1F1A6801206A
:10253000FEF7B6FF3E1B3060E5E73B000122083B9B
:102540001968A40011421DD03B1F1B68134219D00B
:10255000114113410022994200DD04323B1B1A60F5
:102560001A4B3F1B1B780437002B01D0FFF789F96A
:102570002B68019A1C121340154A9B009B58043586
:10258000FFF761F93B1F1A680220FEF789FF3E1B27
:102590003060E5E73B1F1B68A400043B5A1E9341D3
:1025A0003A1B17009B001360084B04371B78002B65
:1025B00001D0FFF766F92B68019A1C121340044AF8
:1025C0009B009B580435FFF73EF9C046B00200203F
:1025D00018E300003B00083B1868FFF715F83B1FA5
:1025E00006001868FFF710F80121A4003B1B1F002C
:1025F000321852000A431A60EA4B04371B78002B4A
:1026000001D0FFF73EF92B68019A1C121340E64AED
:102610009B009B580435FFF716F93B00083B1868F0
:10262000FEF7F2FF3B1F06001868FEF7EDFF0121E1
:10263000A4003B1B1F00321A52000A431A60D94BF8
:1026400004371B78002B01D0FFF71BF92B68019A88
:102650001C121340D44A9B009B580435FFF7F3F833
:102660003B00083B1868FEF7CFFF3B1F06001868C9
:10267000FEF7CAFF02000121A4003B1B1F007243AA
:1026800052000A431A60C74B04371B78002B01D055
:10269000FFF7F7F82B68019A1C121340C24A9B00FF
:1026A0009B580435FFF7CFF83B1F1868FEF7ACFFC7
:1026B000061E17D11F23BB4A1370A4003B1B1F002B
:1026C0001E60B84B04371B78002B01D0FFF7D9F8F8
:1026D0002B68019A1C121340B34A9B009B58043587
:1026E000FFF7B1F83B00083B1868FEF78DFF31009B
:1026F00008F0B8F8012346001E43DEE73B1F1868C8
:10270000FEF782FF061E17D11F23A64A1370A400EE
:102710003B1B1F001E60A34B04371B78002B01D00E
:10272000FFF7AFF82B68019A1C1213409E4A9B00DA
:102730009B580435FFF787F83B00083B1868FEF705
:1027400063FF310008F074F901234E001E43DEE7F9
:102750003B1F1868FEF758FFC2178018504001222F
:10276000A4003B1B1F004000104318608D4B043732
:102770001B78002B01D0FFF784F82B68019A1C12FC
:102780001340894A9B009B580435FFF75CF8A3006F
:102790000793FB1A0493012C2CD11868FEF734FF21
:1027A00001230600C4179C43E418B44202DC330042
:1027B00026001C000134A41B0AF078FC210008F05C
:1027C00037F901238E1976001E43049B1E60079B78
:1027D000FF1A744B04371B78002B01D0FFF751F818
:1027E0002B68019A1C1213406F4A9B009B580435BA
:1027F000FFF729F8022C0AD1049B1868FEF704FFA2
:10280000049B04005868FEF7FFFE0600CDE7642431
:102810000126CFE7A300FE1A31002000049301F047
:1028200059FF049B3060FF1A5E4B04371B78002B66
:1028300001D0FFF726F82B68019A1C1213405A4A60
:102840009B009B580435FEF7FEFF3B00083B1868D1
:10285000FEF7DAFE3B1F06001868FEF7D5FE020001
:102860000121A4003B1B1F00324052000A431A60A2
:102870004C4B04371B78002B01D0FFF702F82B6874
:10288000019A1C121340484A9B009B580435FEF7DE
:10289000DAFF3B00083B1868FEF7B6FE06003B1F58
:1028A0001868FEF7B1FE32000121A4003B1B1F0097
:1028B000024352000A431A603A4B04371B78002B3C
:1028C00001D0FEF7DEFF2B68019A1C121340364A36
:1028D0009B009B580435FEF7B6FF3B00083B186889
:1028E000FEF792FE06003B1F1868FEF78DFE3200D1
:1028F0000121A4003B1B1F00424052000A431A6002
:10290000284B04371B78002B01D0FEF7BAFF2B6849
:10291000019A1C121340244A9B009B580435FEF771
:1029200092FF3B1F1868FEF76FFEC0430122A40010
:102930003B1B1F004000104318601A4B04371B78E4
:10294000002B01D0FEF79DFF2B68019A1C1213404B
:10295000154A9B009B580435FEF775FF3B00083B6A
:102960001868FEF751FE06003B1F1868FEF74CFE84
:10297000320082400121A4003B1B1F0052000A4389
:102980001A60084B04371B78002B01D0FEF779FF43
:102990002B68019A1C121340034A9B009B58043574
:1029A000FEF751FFB002002018E300003B00083B97
:1029B0001868FEF729FE06003B1F1868FEF724FE84
:1029C000320002410121A4003B1B1F0052000A43B8
:1029D0001A60EA4B04371B78002B01D0FEF751FF39
:1029E0002B68019A1C121340E54A9B009B58043542
:1029F000FEF729FF3B000C3B1868FEF705FE3B0085
:102A0000083B06001868FEF7FFFDF1170200C31728
:102A1000300008F05FF83B1F049005911868FEF73E
:102A2000F3FD02000498059908F008F80123A400BA
:102A30003E1B370040001843D04B30601B780437F2
:102A4000002B01D0FEF71DFF2B68019A1C121340CA
:102A5000CB4A9B009B580435FEF7F5FEA300FE1AF7
:102A6000310020000493FEF729FB049B3060FF1A1D
:102A7000C24B04371B78002B01D0FEF702FF2B68F6
:102A8000019A1C121340BE4A9B009B580435FEF766
:102A9000DAFEA300FF1A39002000FEF72BFBB74B2C
:102AA0001B78002B01D0FEF7ECFE2B68019A1C125C
:102AB0001340B34A9B009B580435FEF7C4FEA300A5
:102AC000FE1A310020000493FEF754FB049B306093
:102AD000FF1AAA4B04371B78002B01D0FEF7D1FE5A
:102AE0002B68019A1C121340A54A9B009B58043581
:102AF000FEF7A9FEA300FF1A39002000FEF7D8FB5D
:102B00009E4B1B78002B01D0FEF7BBFE2B68019A71
:102B10001C1213409A4A9B009B580435FEF793FE03
:102B2000A300FE1A310020000493FEF749FC049B29
:102B30003060FF1A914B04371B78002B01D0FEF751
:102B4000A0FE2B68019A1C1213408D4A9B009B58D3
:102B50000435FEF778FE3B1F186801F04DFA3A0085
:102B60000121083A12680300A4000A4229D1042A6C
:102B70000CD910680F221040013808280FD807F030
:102B8000D3FD052026220E0E0E0E24007D491800CE
:102B90000AF02CFB434258413B1B80001860774BE6
:102BA0003F1B1B780437002B01D0FEF76AFE2B6811
:102BB000019A1C121340724A9B009B580435FEF781
:102BC00042FE7149E3E77149E1E77149DFE7714985
:102BD000DDE7069B3E1DF31A684CD82B03DD1A2354
:102BE0002370FEF74EFE00F099FF01223B004000EB
:102BF0001043186023783700002B01D0FEF741FE08
:102C00002B68019A1C1213405D4A9B009B580435A7
:102C1000FEF719FE069B3E1DF31A584CD82B03DD18
:102C20001A232370FEF72DFE00F06EFF5A4A400073
:102C3000104001223B001043186023783700002B1E
:102C400001D0FEF71EFE2B68019A1C1213404C4A5D
:102C50009B009B580435FEF7F6FD069A3B1D9B1A18
:102C6000464CD82B03DD1A232370FEF70AFE00F032
:102C700055FF4A4B1A68831A904201D2484A9B1862
:102C800001213A005B000B43136023780437002BCB
:102C900001D0FEF7F6FD2B68019A1C121340384A4A
:102CA0009B009B580435FEF7CEFD00F037FF3B4BF1
:102CB000A4001860314B3F1B1B78002B01D0FEF79E
:102CC000E0FD2B68019A1C1213402D4A9B009B5873
:102CD0000435FEF7B8FD03F037FBA300002810D140
:102CE000FF1A264B1B78002B01D0FEF7CAFD2B687C
:102CF000019A1C121340224A9B009B580435FEF790
:102D0000A2FD3E00FF1A012320001A003900FEF741
:102D1000C9FC244C2068643003F02AFB002803D14E
:102D2000043D3700FEF7C0FD029B21685A781E481B
:102D300003F04DFF0123029A137000F0E5FE1B4BD8
:102D400022681B68063253431818FFF7E6F803F0B1
:102D5000FBFAA30000282BD1FF1A084B1B78002B8D
:102D600001D0FEF78EFD2B68019A1C121340044A15
:102D70009B009B580435FEF766FDC046B00200205C
:102D800018E3000054E500005CE5000063E5000086
:102D90006AE500006FE50000FEFFFF7FDC05002014
:102DA00037894100D4050020B10200200400002032
:102DB0003E00FF1A2000012300223900FEF772FCBA
:102DC000F14C2068643003F0D3FA0028A8D0EF4813
:102DD00003F07AFCAEE7A4003E1BFEF7FBFC3700D5
:102DE000EB4B30601B780437002B01D0FEF749FD18
:102DF0002B68019A1C121340E64A9B009B5804352D
:102E0000FEF721FDE24BA4001B783F1B002B01D0F5
:102E1000FEF737FD2B68019A1C121340DD4A9B0018
:102E20009B580435FEF70FFDA4003E1B300000F058
:102E3000AEFE3700D64B30601B780437002B01D034
:102E4000FEF71FFD2B68019A1C121340D14A9B000C
:102E50009B580435FEF7F7FCA4003E1B300000F041
:102E600098FE3700CA4B30601B780437002B01D026
:102E7000FEF707FD2B68019A1C121340C54A9B0000
:102E80009B580435FEF7DFFCA300FE1A310020003A
:102E9000049300F0C9FC049B3060FF1ABC4B04375C
:102EA0001B78002B01D0FEF7ECFC2B68019A1C125A
:102EB0001340B84A9B009B580435FEF7C4FCA4009D
:102EC0003F1B380000F068FEB14B1B78002B01D08F
:102ED000FEF7D7FC2B68019A1C121340AD4A9B00E9
:102EE0009B580435FEF7AFFCA300FE1A310020000A
:102EF000049300F0FDFB049B3060FF1AA44B0437E1
:102F00001B78002B01D0FEF7BCFC2B68019A1C1229
:102F10001340A04A9B009B580435FEF794FCA40084
:102F20003F1B380000F07EFE994B1B78002B01D030
:102F3000FEF7A7FC2B68019A1C121340954A9B00D0
:102F40009B580435FEF77FFC0121200000F052FE63
:102F50008F4B1B78002B01D0FEF793FC2B68019A56
:102F60001C1213408B4A9B009B580435FEF76BFCE8
:102F70000021200000F03EFE854B1B78002B01D085
:102F8000FEF77FFC2B68019A1C121340814A9B00BC
:102F90009B580435FEF757FCA4003E1B300000F0A0
:102FA0006FFE37007A4B30601B780437002B01D05E
:102FB000FEF767FC2B68019A1C121340754A9B00B0
:102FC0009B580435FEF73FFCA4003E1B300000F088
:102FD0006BFE37006E4B30601B780437002B01D03E
:102FE000FEF74FFC2B68019A1C121340694A9B00A4
:102FF0009B580435FEF727FCA4003F1B380000F067
:1030000027FE634B1B78002B01D0FEF73AFC2B68A0
:10301000019A1C1213405F4A9B009B580435FEF72F
:1030200012FCA4003F1B380004F06CFA584B1B78CC
:10303000002B01D0FEF725FC2B68019A1C121340CF
:10304000544A9B009B580435FEF7FDFBA4003E1B31
:10305000300004F031FB37004D4B30601B780437F3
:10306000002B01D0FEF70DFC2B68019A1C121340B7
:10307000484A9B009B580435FEF7E5FBA4003F1B24
:10308000380004F0BBF9424B1B78002B01D0FEF74F
:10309000F8FB2B68019A1C1213403E4A9B009B5878
:1030A0000435FEF7D0FBA4003E1B300004F0C0F94D
:1030B0003700374B30601B780437002B01D0FEF708
:1030C000E0FB2B68019A1C121340324A9B009B586C
:1030D0000435FEF7B8FBA300FF1A3900200001F009
:1030E00021FF2B4B1B78002B01D0FEF7CAFB2B686E
:1030F000019A1C121340274A9B009B580435FEF787
:10310000A2FBA300FF1A3900200001F011FD204BA3
:103110001B78002B01D0FEF7B4FB2B68019A1C1220
:1031200013401C4A9B009B580435FEF78CFBA30000
:10313000FF1A3900200001F0ADFD154B1B78002B64
:1031400001D0FEF79EFB2B68019A1C121340114A16
:103150009B009B580435FEF776FBA300FF1A39004D
:10316000200001F0BFFD0A4B1B78002B01D0FEF7B9
:1031700088FB2B68019A1C121340064A9B009B583F
:103180000435FEF760FBC046D4050020B1020020E4
:10319000B002002018E30000A300FE1A3100200056
:1031A000049304F0F9FA049B3060FF1AC64B04370D
:1031B0001B78002B01D0FEF764FB2B68019A1C12D0
:1031C0001340C24A9B009B580435FEF73CFBA3000A
:1031D000FE1A31002000049304F0E6FA049B3060EC
:1031E000FF1AB94B04371B78002B01D0FEF749FBBF
:1031F0002B68019A1C121340B44A9B009B5804355B
:10320000FEF721FBA300FE1A31002000049304F016
:10321000D3FA049B3060FF1AAB4B04371B78002BAA
:1032200001D0FEF72EFB2B68019A1C121340A74A0F
:103230009B009B580435FEF706FBA300FE1A3100E5
:103240002000049304F0C0FA049B3060FF1A9E4BE8
:1032500004371B78002B01D0FEF713FB2B68019A73
:103260001C121340994A9B009B580435FEF7EBFA59
:10327000A300FF1A3900200001F0D4FD924B1B7807
:10328000002B01D0FEF7FDFA2B68019A1C121340A7
:103290008E4A9B009B580435FEF7D5FAA300FF1A0F
:1032A0003900200001F046FD874B1B78002B01D030
:1032B000FEF7E7FA2B68019A1C121340834A9B0021
:1032C0009B580435FEF7BFFAA300FE1A3100200018
:1032D000049301F0ABFC049B3060FF1A7A4B043777
:1032E0001B78002B01D0FEF7CCFA2B68019A1C1238
:1032F0001340764A9B009B580435FEF7A4FAA300BE
:10330000FF1A3900200001F03FFC6F4B1B78002BA7
:1033100001D0FEF7B6FA2B68019A1C1213406B4AD3
:103320009B009B580435FEF78EFA002C7CDD3B1F7A
:103330001E68012C0CD1264207D1042E05D90F237B
:10334000326830001340042B11D001235B4213E09C
:10335000022CFAD13B00083B186801231842F4D133
:103360000428F2D902680E331340042BEDD100F08B
:1033700043FEFEF7EDF80300A200BF1A5A1C53D01B
:103380000020022C11D101223240824226D1042E8B
:1033900024D90F213068014009291FD171684810D4
:1033A000C0B28100914214D17F18FF2B1ED81C029D
:1033B000044323129C464648DBB2DB00C218117955
:1033C000414A032901D1FEF791FC02231370FEF755
:1033D00058FAB418A468BC500432E3E70B223A4B05
:1033E0001A7000233B600437FEF74BFA069A0299E5
:1033F000BA1A86009210BE1B0A613100984700225B
:10340000344B371D1A60304B30601B78934201D02B
:10341000FEF737FA2B68019A1C1213402B4A9B00C7
:103420009B580435FEF70FFA00233B60264B3A1DEC
:103430001B78002B02D01700FEF723FA2B680199A6
:103440001C120B4021499B005B5817000435FEF706
:10345000FAF9069B029AFB1A9B101361A300FF1A4C
:103460003900200003F072F9174B1B78002B01D0B4
:10347000FEF707FA2B68019A1C121340134A9B00AF
:103480009B580435FEF7DFF9069B029AFB1A9B1046
:103490001361A300FE1A31002000049303F056F9D3
:1034A000049B3060FF1A084B04371B78002B01D0B7
:1034B000FEF7E7F92B68019A1C121340034A9B00A0
:1034C0009B580435FEF7BFF9B002002018E3000056
:1034D000A8250020E40F00200023F7B55A1E019212
:1034E000002B07DA01F034FD03F048FA03F020FC6A
:1034F0001923019300263000194B1968B14212DDDF
:10350000184B1A6801328A420FDAF0241A601D68DB
:10351000154F6C43E35D002B1FD0E419022B06D13D
:103520002000FEF76FF9019BD8E70022EDE7012BA1
:103530000DD1002801D100F0E7FAF0226A43BB1850
:103540005B680A49C31A8B4201D80223BB54F0239B
:103550005D43054BEB5C022BE2D00136CCE7C04665
:10356000D805002000000020481C00203F420F002A
:1035700080220B4B52001A600121A822A920094B7E
:10358000D20019649A58C00005321A5006481A50E1
:10359000C122C020920000039850044B197070475C
:1035A00000E100E0008000404C0500000106002022
:1035B00004207047F8B550C9012322001A40101E9C
:1035C0002DD03340181E2AD0641000201A2C26D883
:1035D0001D4B761035009E4200DD1D001B4F3B5DEC
:1035E000012B05D00121200005F08EFC01233B5565
:1035F000174B1B78002B01D1FFF7BAFF0023154AA8
:103600009E420DDCFF2514491448D65CB44202D119
:103610005E007052D5540133042BF6D10420F8BD5E
:10362000D15C8C4203D10C4A5B009D52F6E701331A
:10363000042BF5D10023D15CFF2901D1D454F2E74A
:103640000133042BF7D1E9E788130000E4050020DB
:10365000010600201C0000200E000020DC050000F8
:1036600070B530C9012322001A40101E1BD02B4018
:10367000181E18D064101A2C00D91924154E335D69
:10368000012B05D00121200005F03EFC012333551C
:1036900069100800104A1038104B904204D90122DA
:1036A00052421A60042070BD1C600D4807F0DAF821
:1036B0000C4B040018800C4B1B78002B01D1FFF73A
:1036C00057FF0122094B9A64A922D2009958641825
:1036D0009C50E7E7E40500209086010018000020D8
:1036E00020A107000C0000200106002000800040FF
:1036F00070B501240D68254204D10D20FEF74CF869
:10370000200070BD6D101A2D17D80024012804DD8B
:103710004C68043C63425C416400094E735DA34203
:1037200004D02100280005F0EFFB7455280005F0B7
:103730001FFC03000420012BE3D00020E1E7C0467A
:10374000E4050020F8B501260D683400B04200DD24
:103750004C682B003340181E0BD023003340181E3A
:1037600007D06D10002D05DCA12300201E4ADB00D0
:10377000D650F8BD641000201A2CFAD81B4F3B5DC0
:10378000012B04D00121200005F0BEFB3E5529008D
:10379000174807F067F80A21053007F063F8154B62
:1037A000A400E258144B12021343A2221349D20080
:1037B0008B50134C0C4B9C50124C19510124124944
:1037C0005C50124B196900219950114A904200DD5A
:1037D0001000A8228021D2009850012289005A505E
:1037E00004201A60C5E7C04600F00140E40500204F
:1037F00000B4C40424F8000003000300006000408B
:1038000040A10040140500000405000000A0004095
:10381000FFFF0000030010B50120002B02DC1B306D
:10382000FDF7BAFF10BD0000F8B501240B680600D3
:103830000D00234204D10D20FDF7AEFF2000F8BD9E
:103840005B1004D103F006FE40002043F7E72000A0
:10385000072BF4D80D4A9B009C580D4F3B5D002B65
:1038600005D00021200005F04FFB00233B55012E21
:1038700006DD6B68042B03D10221200005F044FB18
:10388000200005F0EFF901244000DEE7ECE5000040
:10389000E405002010B50124044002D044102000AB
:1038A00010BD042810D90F2302681340042B07D140
:1038B00000F0A2FB21000A2209F06AFD0400EEE7F5
:1038C000032B01D10430F5E70D20FDF765FFE6E796
:1038D000F8B50C00022803DC1C20FDF75DFFF8BDE5
:1038E0000868FFF7D7FF06006068FFF7D3FF050001
:1038F000A068FFF7CFFF0100794806F0B3FF04008E
:103900001A2D01D90020EAE7764F7B5D012B05D007
:103910000121280005F0F8FA01237B550021280039
:1039200005F010FB002C0ED020000138C046C04628
:10393000C046C046C046C046C046C046C046C04657
:10394000C046C046F1D1012731002800394005F0BA
:10395000F9FA002C0ED020000138C046C046C046FF
:10396000C046C046C046C046C046C046C046C04627
:10397000C046F1D171103940280005F0E3FA002C5F
:103980000ED020000138C046C046C046C046C046E2
:10399000C046C046C046C046C046C046C046F1D13B
:1039A0000127B1103940280005F0CCFA002C0ED0C8
:1039B00020000138C046C046C046C046C046C0468A
:1039C000C046C046C046C046C046C046F1D1F11010
:1039D0003940280005F0B6FA002C0ED0200001383E
:1039E000C046C046C046C046C046C046C046C046A7
:1039F000C046C046C046C046F1D10127311139400A
:103A0000280005F09FFA002C0ED020000138C04697
:103A1000C046C046C046C046C046C046C046C04676
:103A2000C046C046C046F1D171113940280005F0AA
:103A300089FA002C0ED020000138C046C046C0468E
:103A4000C046C046C046C046C046C046C046C04646
:103A5000C046F1D10127B1113940280005F072FAB2
:103A60003900002C0ED020000138C046C046C046A8
:103A7000C046C046C046C046C046C046C046C04616
:103A8000C046F1D1F6113140280005F05BFA002C58
:103A90000ED020000138C046C046C046C046C046D1
:103AA000C046C046C046C046C046C046C046F1D12A
:103AB0000121280005F046FA002C00D122E7200061
:103AC0000138C046C046C046C046C046C046C04693
:103AD000C046C046C046C046C046F1D112E7C04607
:103AE00040420F00E40500200420704710B5002874
:103AF00003DC1C20FDF750FE10BD0B680020DB0727
:103B0000FAD40D30F6E700000122034B1A64A82214
:103B1000D20098587047C046008000400122054BF3
:103B200010B51A64A822FA21D2009858890006F02C
:103B30000FFE10BD00800040004870470CE60000FA
:103B40001B20704770B5054E0400335C0D008B429E
:103B500002D005F0D9F9355570BDC046E405002006
:103B600070B50024084D635D012B09D100212000B0
:103B700005F0E8F90021200005F0C6F9002363559F
:103B800001341B2CEED170BDE405002070471120DC
:103B90007047372070470000F8B5012605683542A8
:103BA00002D04468344203D10D20FDF7F5FDF8BD85
:103BB0006D101A2DFBD80A4F7B5D012B04D031000C
:103BC000280005F0A1F97E55064964108C4202DCFC
:103BD000E143C9172140280005F0CAF8E7E7C046CD
:103BE000E4050020FF03000010B50800FFF7D4FF34
:103BF000002010BD70B504000D001A280ED8084E24
:103C0000335C012B04D0012105F07EF901233355EB
:103C1000290020004D1EA94105F094F970BDC04651
:103C2000E4050020036810B5DA0703D40D20FDF782
:103C3000B3FD10BD4168581004394A425141FFF7A5
:103C4000D9FFF6E710B50800FFF7ECFF002010BD24
:103C500037B569460A00064B30CB30C203680220F4
:103C6000042B02D101F016F837BD01F03BF8FBE759
:103C70007CE5000010B50800FFF7EAFF002010BD4A
:103C800010B5084C237D002B05D00021142005F031
:103C90003BF900232375142005F06AF9434258418B
:103CA000800010BDE405002010B5084CA37D002B5A
:103CB00005D00021162005F027F90023A375162052
:103CC00005F056F943425841800010BDE40500203C
:103CD000A02200230349D2008B50034910328B509D
:103CE0007047C04600F0014000600040F7B52F4D1E
:103CF0002F4EEB6C002B14D0A9240023E40037597D
:103D0000EB642C4B186800280BDB2B4B19784A42CC
:103D10005141C9B2197005F015F9284B1B88DF19FC
:103D200037512B6D002B38D00021254B254FF458EF
:103D300029653A780193244D8A4206D02B68032BDB
:103D400003D8224AD05C05F0FDF82B68204A0133E5
:103D5000134004D50422013B5242134301331B4953
:103D600000228C462B60042B18D06046C05C591C86
:103D7000FF2802D10B000122F5E7002A00D02B60BA
:103D8000012105F0DFF801233B702B68114A5B002D
:103D90009B5A0C34E418019BF450F7BD01235B429D
:103DA0002B6000233B700C4BF4E7C046FC800040C6
:103DB0000080004018000020000600200C000020B9
:103DC0004C050000FF050020E00500201C0000203D
:103DD000030000800E0000205C460000084B094AEA
:103DE000FF201A805A809A80DA800023064A074909
:103DF0001370074A087048708870C8701360704765
:103E00000E000020DC050000FF0500201C00002043
:103E1000E00500200122024B52421A607047C04662
:103E20001800002010B5034A0D21034802F0C4F920
:103E300010BDC04684E5000057EF0000E12170B5D9
:103E40004902194804F084FC002401220320174B86
:103E500017491A615C500431585080180831585085
:103E60001A60063004F0F8FEFF21124AA154013412
:103E70001B2CFBD1012200200F4B01001A600423F0
:103E80000E4A0F4D1468002CFCD02C680002013B38
:103E900020431160002BF5D101220A4B1A6004F077
:103EA00013FE01F09BF970BDD01B00200080004084
:103EB00004050000E405002000D0004000D10040CF
:103EC00008D5004004D00040F8B50B4E0700300084
:103ED0000D0004F085FC0400A84200DD2C003D002C
:103EE000EB1B9C4205DD300004F084FC287001359A
:103EF000F6E72000F8BDC046D01B002010B5010039
:103F0000014804F02DFC10BDD01B002010B5054C5D
:103F1000200004F033FCE1212000490204F018FCE9
:103F200010BDC046D01B0020C3070CD4064B1B6835
:103F3000834208D8054B1B68984204D8031F1B68AE
:103F4000002B00D0180070470C0600200806002047
:103F50000023012210B50A48990001334250642B16
:103F6000FAD1084C084B00211A602000074A08F0DB
:103F7000BDFD074B074A6360074B1A6010BDC04682
:103F8000A02D00201006002008000020D409000009
:103F900030270000140600200406002010B5044B52
:103FA000044A1A60044B054A1A60FFF7D1FF10BD9E
:103FB0000C0600201006002008060020E40F002058
:103FC000044B1B681868000980B20238C343DB1732
:103FD000184070470406002000B59BB00200054958
:103FE00001A809F0C7F801A802F08AFB02F0A0FEC0
:103FF000FCE7C046E3E600000B4BC20704D40428EC
:1040000004D80A4B00D00A4B180070470F220368EF
:104010001A40031D042AF7D0064B092AF4D0064B98
:10402000032AF1D0054BEFE7BDE60000A6E1000052
:10403000A0E10000C7E60000D7E60000CEE60000E1
:104040000020064A0649131F186013681B099BB21B
:1040500002339B00D2188A42F5D370471406002021
:10406000E40F0020F7B50F240126314B314A1968BF
:10407000314B324D186813681F002740072F26D890
:1040800013681B099BB202339B00D218AA42F2D3D9
:1040900000242B4EA500AD192868FFF745FF013419
:1040A0002860642CF6D1274C2068FFF73DFF206084
:1040B000254C2068002802D0FFF736FF206000253D
:1040C000224B1B680093009B9D4214DBF7BD1B092C
:1040D0009BB29B00D3189A42D2D01F68374208D1B6
:1040E000B94206D2B84204D3043F3F68002F00D043
:1040F0001F60043BEFE7F0236B43154A9B181A78C7
:10410000002A01D10135DEE71F693C2300266B43FD
:10411000DB199B0001930136BB1BF3D4019BB40058
:104120001C1B0B4B1C19A069FFF7FEFEA061F2E7F8
:104130000C0600201406002008060020E40F0020D2
:10414000A02D002008000020E40F0020D80500204A
:10415000481C0020F7B50124204246D1234B1B68A0
:104160009C46984241D3224B1B68019398423CD80D
:10417000031F1B68002B38D10200036800941B0941
:104180009BB2002B0FD10099131F196090422CD0C5
:1041900015682B1F1B68990069180C68013B146097
:1041A0000A602A00EDE79D0055192968009C21420C
:1041B00019D18C4517D8019C8C4214D30E1F34683A
:1041C000002C10D10F680F343C40072C08D92F6009
:1041D000151F2B600B680A601B099BB20A00D0E711
:1041E00000993160CDE7013BCBE7F7BD0C0600201D
:1041F000080600200D4970B50A000D4D1368141F04
:104200001B0926689BB2981C002E0BD000238A4203
:1042100000D00B0023608300C91880001218AA4246
:10422000ECD370BD1B011360F7E7C04614060020F5
:10423000E40F0020F8B5124C27000F223B681D093F
:10424000ADB213420DD06E1CB600A74204D03200AE
:104250003900200008F037FC0022A3190436A41905
:104260001A600235AD00074B7F199F42E5D31B1B37
:104270009B10013B1B012360034B1C60F8BDC04633
:1042800014060020E40F002004060020F0B59BB0C7
:10429000FFF73AFC00240700214AA300D05801345C
:1042A000FFF758FF642CF7D11E4B1868FFF752FF39
:1042B0001D4B1868002801D0FFF74CFF00261B4B50
:1042C0001B689E4217DBFFF795FFFFF7CBFEFFF75A
:1042D000B1FFFFF719FC164BC21B1B6815491B6881
:1042E00001A81B099BB2023B08F044FF01A802F0A1
:1042F00007FA1BB0F0BDF02575430F4BED182B7876
:10430000002B01D10136DAE72B695C1E002CF9DBAA
:10431000A300EB189869FFF71DFF013CF6E7C046C4
:10432000A02D002008000020E40F0020D805002068
:10433000040600209DE60000481C0020F7B5174D3C
:104340004F1C2B6806001B680C001B099BB20192D6
:104350009F420BDBFFF79AFF2B681B681B099BB280
:104360009F4203DB0A20FDF717FAFEBD2868A71C51
:10437000BA00DB1B81181B010B6029600021031FA1
:1043800019600F231E4003002401264340C3083A4E
:104390009A189A42E9D9019902C3FAE70406002063
:1043A000F7B503000122134004000D000193002B18
:1043B0002BD1174B1B68834227D8164B1B688342AF
:1043C00023D90F23144F386000681840FFF7B6FF59
:1043D000019B3C68061E3B6017D0236804301B0914
:1043E0009BB29D4200DD1D00AA00211D251F08F083
:1043F00061FBFFF725FE2E60FFF734FE00232B60E4
:104400002268064B1340236034002000FEBDC046E6
:104410000C06002008060020E40F0020F0FF0F002B
:104420000323043010B5C117194009188910002260
:104430000420FFF783FF10BD70B5050008000C00D5
:10444000FFF7EEFF0023002804D170BDE95CC2181D
:1044500011710133A342F9DBE343DB171C40002356
:1044600004192371F1E7F0B50C009BB0022804DCBD
:104470001C20FDF791F91BB0F0BD0123086818421C
:1044800006D1042804D90F2601683140042901D03F
:104490000E20EEE761680D001D40F9D10429F7D91F
:1044A0000A683240042AF3D1A2681A4201D10D20D1
:1044B000DFE7FFF7A1FD06006068FFF79DFDA76835
:1044C000010001AC7F103000257003F06BFD390056
:1044D0006423220003F0CBFD200008F091FE0100D0
:1044E0002000FFF7A9FFC6E710B51C4CA544041E29
:1044F00002D1FFF795FF0BE003F06CFC01380628B2
:1045000028D806F011F909091118290424000020FF
:104510008023DB009D4410BD200003F0D7FC011B6D
:104520002000FFF789FFF3E7200003F07DFC430044
:1045300001201843ECE780226946D200200003F0F6
:104540008AFC684608F05CFE01006846E9E7042141
:104550000348E6E70020CCE70420D9E700FCFFFF92
:104560003CE7000070B50C00022803DC1C20FDF7BE
:1045700013F970BD01230868184206D1042804D934
:104580000F2501682940042901D00E20EFE761685A
:104590001942FAD10429F8D90A682A40042AF4D128
:1045A000A2681A4201D10D20E1E7FFF725FD0500C1
:1045B0006068FFF721FDA46801006410280003F083
:1045C000F1FC210003F02EFDFFF78EFFD1E770B55F
:1045D0000D00012803DC1C20FDF7DEF870BD01246E
:1045E0000868204206D1042804D90F2102680A4035
:1045F000042A01D00E20EFE76A682242FAD1042A89
:10460000F8D913680B40042BF4D1FFF7F5FC060032
:104610006868FFF7F1FC0100300003F0C3FC03F011
:1046200045FD40002043D9E7F8B507000C001C20E9
:10463000012F0BDD01250868284206D1042804D982
:104640000F2102680A40042A03D00E20FDF7A4F8C7
:10465000F8BD62682A42F8D1042AF6D913680B40E3
:10466000042BF2D1FFF7C8FC06006068FFF7C4FC1A
:104670000100022F14D0A4682C4211D06410300025
:1046800003F090FC050003F0A5FB012811D1002CDC
:1046900002DD0135012C06D12800FFF725FFD7E701
:1046A00001246442EBE7280003F01DFC013C0500F7
:1046B000F0E70228F0D1002CEEDD0135012CEBD023
:1046C00000222800110003F040FC03F00CFC013C28
:1046D0000500F3E7086870B501240500254006D100
:1046E000042804D90F2302681340042B03D00E20A2
:1046F000FDF752F870BDFFF77FFC03782900233BDC
:104700005A4253411022C01808F042FE80239B05F4
:10471000C218044B9A4201D91420E9E74000204313
:10472000E8E7C046FFFFFF3F10B50124044002D078
:104730004410200010BD042810D90F230268134034
:10474000042B07D1FFF758FC21000A2208F020FEB5
:104750000400EEE7032B01D10430F5E70D20FDF74F
:104760001BF8E6E710B50868FFF7DEFF06F00EFB62
:10477000094906F0D9F908F0BFF804F007FD074B26
:10478000002207F073FA04F0A9FC08F045F8430092
:104790000120184310BDC046D30237390000D04075
:1047A000F7B50C00042803DC1C20FCF7F5FFFEBD68
:1047B0000868FFF7B9FF01906068FFF7B5FF0600D2
:1047C000A068FFF7B1FF0500E068FFF7ADFF070045
:1047D0002069FFF7A9FFAE4201D11F20E5E7019B49
:1047E000C01B9B1B5843A91B06F03CF8C7190120AE
:1047F0007F003843DBE7000010B5034A0821034877
:1048000001F0DAFC10BDC046FCE60000F4E6000052
:104810000020704710B51E20FCF7BEFF10BD10B57C
:104820001E20FCF7B9FF10BD10B51E20FCF7B4FF29
:1048300010BD10B51E20FCF7AFFF10BD10B51E2037
:10484000FCF7AAFF10BD10B51E20FCF7A5FF10BD98
:1048500010B51E20FCF7A0FF10BD10B51E20FCF700
:104860009BFF10BD10B51E20FCF796FF10BD10B5C4
:104870001E20FCF791FF10BD10B51E20FCF78CFF29
:1048800010BD10B51E20FCF787FF10BD10B51E200F
:10489000FCF782FF10BD10B51E20FCF77DFF10BD98
:1048A00010B51E20FCF778FF10BD10B51E20FCF7D8
:1048B00073FF10BD10B51E20FCF76EFF10BD10B5C4
:1048C0001E20FCF769FF10BD10B51E20FCF764FF29
:1048D00010BD10B51E20FCF75FFF10BD10B51E20E7
:1048E000FCF75AFF10BD10B51E20FCF755FF10BD98
:1048F00010B51E20FCF750FF10BD10B51E20FCF7B0
:104900004BFF10BD10B51E20FCF746FF10BD10B5C3
:104910001E20FCF741FF10BD10B51E20FCF73CFF28
:1049200010BD10B51E20FCF737FF10BD10B51E20BE
:10493000FCF732FF10BD000010B5034A1E210348EA
:1049400001F03AFC10BDC04690E7000080E800008E
:104950000120034B1860034B1B68834018437047CA
:1049600004100020E80F0020F0B5EFF310810123C0
:10497000194083F31088134AA1261268124D013A98
:104980009340A022114FD205F600002B17D02C68BF
:10499000945103420BD0C046C046C046C046C046F4
:1049A000C046C046C0462C68D4515B08EDE7D451E0
:1049B000C046C046C046C046C046C046F5E781F383
:1049C0001088F0BD20000020F40F00200C0500002E
:1049D00030B585B001AD0C220649280008F06AF810
:1049E0000024285D01210134FFF7ACF80C2CF8D12C
:1049F00005B030BD0DEA000030B585B001AD0C2228
:104A00000649280008F056F80024285D00210134EA
:104A1000FFF798F80C2CF8D105B030BD0DEA000076
:104A2000F7B56A463B4B01AE1380062393703A4BB1
:104A300033800F23B370FFF767F8384B384DC01839
:104A40002B68984201D200232B602C68002C41D1A6
:104A5000375D01213800FFF775F801340021380077
:104A600004F070FA032CF3D1002401276B461E5D7D
:104A700039003000FFF766F801343900300004F0E7
:104A800061FA032CF2D1C8200138C046C046C046A6
:104A9000C046C046C046C046C046C046C046C046E6
:104AA000C046F1D16B4600211878FFF74BF86B46F2
:104AB00000215878FFF746F86B4600219878FFF7F9
:104AC00041F8FFF721F8FA2300241B01C0182860E1
:104AD0002000FEBDFFF718F82B6800249842F7D39A
:104AE000042004F0BFF80600052004F0BBF83618D7
:104AF000062004F0B7F80B4B9B1B181A0A4BA04278
:104B000006DB18600023094A2B6013600124DFE7ED
:104B10001C60F7E7040500000D0E000010270000E0
:104B2000FC0F002043030000E80F002004100020C9
:104B30000022054B10B51A60044B1B68934201D04C
:104B400003F0E8F8002010BD00100020F41A002047
:104B500010B5041E0CDA1A24084BA400E2581F23D7
:104B60001A401E3B9340064A1360064A136010BD6C
:104B7000FEF7E6FFA042EEDDEEE7C04624F80000B7
:104B8000F40F0020180500500200086810B5C30794
:104B90000FD540101823012A03DD4A68042A00D1EA
:104BA0000833054A1360FEF7F1FFFFF7D1FF00203D
:104BB00010BD01204042EDE72000002010B5002884
:104BC0000CDD0A68131F591E8B4107490B60042A2C
:104BD00006D0FFF711FF0022044B1A60002010BD21
:104BE000FFF7F6FEFAE7C046F80F0020E80F0020B6
:104BF00010B50124044002D04410200010BD042848
:104C000010D90F2302681340042B07D1FFF7F4F9E2
:104C100021000A2208F0BCFB0400EEE7032B01D1BF
:104C20000430F5E70D20FCF7B7FDE6E70868F8B5B6
:104C3000C3071AD5FFF7DCFF0300203B5E2B25D806
:104C40000520434301221D180020114E9D4219D01A
:104C500005211024F75C3C4200D080180139520035
:104C600064100029F7D10133F0E704280ED90F2290
:104C700003681A40042A09D11B099BB2002B05D0F6
:104C80000379DAE7012340001843F8BD0120FCE76F
:104C900019EA000070B508680D00FFF7A9FF0400CD
:104CA0006868FFF7A5FF621E0100042A14D8451E9C
:104CB000042D11D805236B439B18012215009D403C
:104CC0002B00064805682B430360054B1B68002B2F
:104CD00002D0200003F01FF8002070BD001000205B
:104CE000F41A002070B508680D00FFF781FF04007A
:104CF0006868FFF77DFF621E0100042A13D8451E75
:104D0000042D10D805236B439B1801229A400748B5
:104D1000036893430360064B1B68002B03D00022FB
:104D2000200002F0F8FF002070BDC04600100020F7
:104D3000F41A0020F0B5050089B008680C00FFF7F0
:104D400057FF0690022D36DD6068FFF751FF019096
:104D5000A068FFF74DFF04000127231D661E07937F
:104D6000731C0293079B9E4235D005237343059322
:104D7000019B019D05330493049BAB421ED0042E7E
:104D800016D86B1E042B13D80122059B2349013B27
:104D90005B199A409446224A0B681068069A3A407A
:104DA00003920DD062461A430A60012200280DD1F9
:104DB0007F000135E0E701240194CDE7029ECFE7B3
:104DC000624693430B600028F2D0039A02992800B0
:104DD00002F0A1FFECE7019B1E1D042E1AD8012C46
:104DE00018D1002505273B0021006B439B199940F2
:104DF0000B000A4A013511689943094B11601B6881
:104E0000002B05D0019B0022581D290002F083FFD2
:104E1000052DE8D1002009B0F0BDC04600100020EB
:104E2000F41A0020F0B53B4B85B01B680C00002B3A
:104E300003D101204042FFF78BFE012627683E4048
:104E40003CD1042F3AD90F233A681340092B35D1AE
:104E50007B685B100293029B9E4258DAB300FB18FA
:104E60009868FFF7C5FEFF230500041400121840E0
:104E70001C4029492B404043019305F0F3FC0304F7
:104E8000200025496043039305F0ECFC039C0002DD
:104E9000044301982049404305F0E4FC1F4B2043A4
:104EA0001B68202B06D1AD00AD0E1D4BAD00EC589C
:104EB00000022043FFF758FD0136CCE73800FFF72A
:104EC00097FEFF26050007140012304012494043A8
:104ED00005F0C8FC3740040438000F49784305F05A
:104EE000C1FC2E400002044330000B49704305F022
:104EF000B9FC0A4B20431B68202B06D1AB009B0E4C
:104F0000074A9B009B5800021843FFF72DFD002025
:104F100005B0F0BDF40F002059060000200000206D
:104F2000F4EB0000086810B5C30703D5FFF760FE77
:104F3000054B1860054B1B68002B03D0024B18680B
:104F400002F0EAFE002010BD00100020F41A00203C
:104F50009D4B70B51B68002B0DD19C4C2368002B1A
:104F60000AD19B4A1268002A06D19A4B1B68002B73
:104F700001D0FFF755FD70BD974D2A68002A1BD15F
:104F8000944A1268002A10D0FFF74AFD0028F2D098
:104F9000FFF71EFD8E4B226819681A6000290BD09E
:104FA000002A09D1FFF728FDE5E7894A1268002A9F
:104FB000F0D1002BEED0EBE700210D2003F0C2FF73
:104FC00000210E2003F0BEFF00210F2003F0BAFFE6
:104FD0002E68012E5DD0022E00D1A2E0002E51D10C
:104FE000013631007A4C04202368994303F0AAFF6C
:104FF00004212368052019404B42594103F0A2FFC8
:1050000010212368062019404B42594103F09AFFB2
:1050100080212368090119404B4259410C2003F0BB
:1050200091FF80212368090219404B4259410B200E
:1050300003F088FF80212368490219404B425941FF
:105040000A2003F07FFF80212368890219404B4228
:105050005941092003F076FF80212368C9021940D5
:105060004B425941082003F06DFF802321681B0348
:1050700019404B425941072003F064FF31000D20D5
:1050800003F060FF2B680321581C05F0D1FC296058
:1050900071E702214E4C0720236819404B425941C9
:1050A00003F050FF0820216801404B42594103F0B2
:1050B00049FF80212368C90019404B42594105200E
:1050C00003F040FF80212368490119404B425941B8
:1050D000062003F037FF80212368C90119404B42A5
:1050E0005941042003F02EFF8021236889031940D1
:1050F0004B4259410A2003F025FF802321681B04FD
:1051000019404B425941092003F01CFF31000C208B
:1051100003F018FF31000B2003F014FF31000E20C4
:10512000AEE720212A4C0720236819404B42594101
:1051300003F008FF40212368082019404B425941E1
:1051400003F000FF80212368092019404B42594198
:1051500003F0F8FE80212368490019404B42594171
:105160000A2003F0EFFE80212368890019404B429A
:1051700059410B2003F0E6FE802123688901194084
:105180004B4259410C2003F0DDFE80212368490386
:1051900019404B425941062003F0D4FE8021236878
:1051A000C90319404B425941042003F0CBFE802330
:1051B00021685B0419404B425941052003F0C2FEAF
:1051C00001210F205CE7C046F80F002000100020EE
:1051D000F00F002004100020EC0F0020012010B57B
:1051E0004042FFF7B5FC0020FFF7BEFB10BD0000FA
:1051F00010B5034A0A21034800F0DEFF10BDC04687
:10520000F4EC000044ED00008023F0B502255B05BE
:105210001A690A4C0A4BA1261D5103278025F60066
:10522000ED00BA43884202D300221A51F0BD5F5903
:10523000002FFCD098518018F4E7C0460405000008
:1052400000E0014010B5002806D1C020B021400286
:105250008902FFF7D9FF10BDB02080218002C9026A
:10526000F7E7000043425841064B40421840B02344
:105270009B02C018036800201A0E532A01D11B029A
:10528000180A704700C0FEFF30B501248025054B89
:10529000054AED009C505C59002CFCD001600021B7
:1052A000995030BD00E001400405000043425841E0
:1052B000074B40421840B0239B02C018A62310B5EC
:1052C0000902DB05090A1943FFF7DEFF10BDC046DE
:1052D00000C0FEFFF0B5012480260D4B0D4DF600F9
:1052E0005C51002902DC00225A51F0BD5778147835
:1052F0003F022743947824042743D47804322406B9
:105300003C439F59002FFCD010C00139E9E7C0464B
:1053100000E001400405000070B505004B680A007C
:105320009C1C2100A400FFF7D5FF281970BD0000C8
:10533000134B1B68002B0CD08022B023D2029B029F
:1053400000280BD11A1D5B681B0E522B00D11000D8
:105350007047B022C02392025B02F1E782420DD96E
:1053600003681B0E522B09D1436802339B00C018FF
:10537000824203D903681B0E522BE9D00020E7E7D5
:1053800008110020F0B50020B7B00024FFF7D0FFCF
:10539000270005002600002D2ED1284D2868FFF794
:1053A00061FF32003B0001900094254904A807F0FA
:1053B000E1FE04A801F0A4F9224B64201C682B68CC
:1053C000A0215A425341204A5B421340B02292022C
:1053D0009B18E41A6043490205F044FAA0225202E5
:1053E000030000921949220004A807F0C3FE04A894
:1053F00001F086F937B0F0BDFF226B6829689C4642
:105400000233FF180B12013613409C4200DA1C00D5
:10541000FF200A140240039262460140019200916B
:10542000039A0B4904A807F0A5FE04A801F068F947
:105430002800FFF77DFF0500ADE7C04608110020FA
:105440005EEE00000C11002000C0FEFF08EE000020
:105450004AEE000070B50020FFF704FF04000120B1
:10546000FFF700FF844200DA04000A4B1D686A421D
:10547000554128001D60FFF7E5FEA0226B42520255
:105480001340054A28009B18044A611C1360FFF76B
:105490000DFF70BD08110020048001000C110020D8
:1054A000F8B50020FFF7DEFE07000120FFF7DAFE67
:1054B0003E00204D0643204C0DD18021C020C90262
:1054C0004002FFF7A1FE01213000FFF7EFFE1B4B6A
:1054D0002E6023601DE0874209DD0023B0212B6090
:1054E000164B8902236023680020012517E0012361
:1054F00080212B60124BC9022360F4E7120E522A5E
:1055000008D0002800D023600E4801F0F9F8FFF71A
:10551000A1FFF8BD28005A68023292009B188B4206
:1055200005D21A68561CE9D10028F2D0D1E72160D3
:10553000EFE7C046081100200C1100200480010094
:1055400004C0020023EE000070B50020FFF7F0FE5B
:10555000FF260500002801D1280070BD03681C1437
:105560003440FFF7E5FEDA2CF4D10500F2E7000045
:10557000FF2270B51F4CD2000021200007F0B6FAC0
:10558000FF25FFF7E1FF0026002818D1F0210A22AD
:10559000194849420B00962553432D011B185D19EC
:1055A0002D78002D07D0154D154E5D199B191B78D0
:1055B000DB00E3582B60013A002AEBD170BD036891
:1055C0001A142A400A2A0AD11A122A40FF2A03D0A2
:1055D000D200A1180B71A050FFF7AAFED4E7132A3E
:1055E000FAD11B122B40FF2BF6D0DB00E21816710C
:1055F000E650F1E7A8250020481C002068090000BB
:105600006109000010B59AB0FFF74AFFFFF7B0FF3D
:1056100000231A000A48D900415801334C1EA14109
:105620005218FF2BF7D1074901A807F0A3FD01A8E5
:1056300001F066F8044801F063F81AB010BDC046E6
:10564000A825002093EE0000A7EE00008022F0B510
:105650005200A1B00021684807F048FA80220021DA
:105660005200664807F042FA654BFF271B681A0094
:10567000049353425A4110000592FFF7E3FD049C46
:105680000020631E9C415F4B64421C405E4BE4184B
:10569000FFF75AFF0600002E2FD10498FFF7E2FD16
:1056A000411C0598FFF702FE059A554B574D1A60AD
:1056B0002C60FFF75DFFFEF729FC514B64201B684F
:1056C000A0215A4253414F4A5B421340B0222C68FA
:1056D00092029B18E41A6043490205F0C3F8A02225
:1056E0005202030000924A49220007A807F042FD37
:1056F00007A801F005F821B0F0BD326813141212AA
:105700003A403B4003921A000A3A092A49D83A4BD8
:10571000039A995C002931D110223E4807F0E6F93E
:1057200035002B6803991A123A40914209D11A1494
:105730003A400B2A27D0132A2DD00A2A01D1354B03
:105740001D602800FFF7F4FD051EEAD1314B1968F2
:1057500000290FD02000FFF7DFFD04002D4B5B195F
:105760005968002903D02000FFF7D6FD0400043556
:105770000C2DF3D1204B0121039A99543000FFF7EF
:10578000D7FD060087E73B40022BDADC214A9B006D
:10579000D3185D60D5E7102200211E4807F0A6F956
:1057A000CFE71A00153A082AE8D8144A0399525C40
:1057B000002AE3D13500152B00D015003000036816
:1057C0001A143A40152A0FD01D2A00D10025FFF7E0
:1057D000AFFD0028F3D1002D04D020002900FFF7F1
:1057E0009BFD0400054BC6E7039A1B123B409A42FF
:1057F000EDD10500EBE7C046081000201011002095
:105800000811002000C0FEFF04C002000C1100209F
:10581000EDED0000302F002010B5FFF717FF10BD91
:10582000F0B585B0039203220333DC17294D1440F1
:10583000E4182B68284F5A42534180225B42D2021F
:10584000A4103B409B18A21C0291244E9100009191
:105850000190316800980A18934215D2FFF7F6FEBE
:105860002B685A42534180225B421F40D202BF182C
:105870003368009A9B189F4206D2194800F040FFF7
:105880000025280005B0F0BD029B356819066B465F
:105890001A7BA423DB051343FF222F00090C1943B5
:1058A000019B12041B04134019432800FFF7ECFC72
:1058B0000837281D21003760FFF7E6FC002C04D0D4
:1058C0000A9A21003800FFF705FD009B083BFF18EE
:1058D0003760D6E70811002000C0FEFF0C11002041
:1058E000C7ED0000704770470021094B094A596015
:1058F0000131516059680029FCD000211961012350
:1059000093600222044B8131FF315A501A60704774
:10591000FC1000400010004000E100E00222064BB5
:105920000121DA670022054B5A61054A11615A6963
:10593000002AFCD07047C04604E100E0FC100040A3
:105940000010004010B5044C2378002B01D0FFF765
:10595000E5FF0020207010BD111200200120024B35
:105960001B685B0018437047941200200120024B13
:105970001B685B0018437047240000201FB5064BCE
:1059800006491A6801A807F0F5FB082101A8FEF7EF
:1059900053FD05B000BDC0469812002038EF00004E
:1059A0001FB580235B051A6E044901A807F0E2FBCE
:1059B000082101A8FEF740FD05B000BD38EF00004A
:1059C00010B5044C200007F01BFC01002000FEF77E
:1059D00033FD10BD9D1200200E4B10B51B680E4C00
:1059E0005A1C0FD00D4C002B0CD00D4C012B09D0A4
:1059F0000C4C022B06D0094C042B03D00A4C052B6F
:105A000000D1074C200007F0FBFB01002000FEF74F
:105A100013FD10BD280000203DEF00005CE50000F4
:105A200048EF000063E5000042EF000070B504009D
:105A30000D001600FEF772F88023012200215B059D
:105A40001B6E6270E270020AA271020CE2711A0A05
:105A500060716372000EA2721A0C1B0E2670257103
:105A6000A1702072E272237370BD000070B5214CEA
:105A70002278002A3DD1204B01215A608022D20594
:105A800011605A68002AFCD0002207201B4B1C49D9
:105A900001255A500439585008315A5019481A49AA
:105AA00058501A491A485A501A495A50A622D20038
:105AB0009D50082218495A50043158500220174965
:105AC000585017491748585017480439585018204B
:105AD00016495850C12189005A500539FF39585884
:105AE000921802435A501249124A9950FFF7FCFE8D
:105AF000257070BD11120020FC0000400010004015
:105B00000C050000746962751C0500002405000086
:105B1000200004022C0500001405000034050000DC
:105B20003C050000FFFF00002110010054050000AB
:105B3000121200200405000013B5094B0400009365
:105B4000084B019307280AD8074B1B78002B01D17B
:105B5000FFF78CFF6B46054A1957054BD15013BD13
:105B6000E2ECF0F4F8FC00041112002000100040F8
:105B70000C05000070B50E4B06001B78002B01D100
:105B8000FFF774FF00200B4D2C7884420ED00A4B97
:105B9000202219780323091B1940084B4901C91811
:105BA000300006F087FF0120013C2C7070BDC0461C
:105BB000111200209C12002010120020121200204E
:105BC000002370B588B0984235DD0D6801262C00A1
:105BD00034409C422FD12300042D2CD90F222B6856
:105BE0001A402300092A26D16A683F2A23DD684625
:105BF000FFF7C0FF230000281DD06B461978330043
:105C0000A14203DB6B461B5D5B003343A200AA1875
:105C100001349360202CF2D1092169444A780B7831
:105C200012021A438B781B041A43CB781B061343CA
:105C3000024A13600423180008B070BD98120020B7
:105C400070B5454B8AB01B78002B01D1FFF70EFFD2
:105C500002AC2000FFF78EFF002802D100200AB01E
:105C600070BD23780B2BF9D96378012BF6D1E3783B
:105C7000012BF3D100231120384E394D33602B70A6
:105C800068442379374A4178136002780902114346
:105C9000827812041143C27812060A4332490A601C
:105CA000002B0ED1152169444A780B7812021A4351
:105CB0008B781B041A43CB781B06134333600023F5
:105CC00018E0012B1AD1152169444A780B78120289
:105CD0001A438B781B041A43CB781A211B061343F3
:105CE00033600E23627C6944934200DD130000227E
:105CF0009A422CD100220420EA54B0E7022B03D1AF
:105D0000627B10331621EEE7042B0DD115210822FA
:105D10006944684606F0CEFE0098019903F04EF9FA
:105D200006F07AFD3060CAE7052BC8D1152108229C
:105D30006944684606F0BEFE0098019903F03EF9FA
:105D400006F06AFD3060627D0A231E21CBE7885C85
:105D5000A8540132CCE7C046111200209412002052
:105D60009D120020280000209812002010B5134B2F
:105D700004001B78002B01D1FFF778FEFFF7CEFD62
:105D800000200F4A0F49104B5450586001301060EA
:105D900058680028FCD00020186101309060186914
:105DA0000028FCD0094B0A481B785B011B18535094
:105DB000FFF7B4FDFFF798FD10BDC046111200209B
:105DC0000010004004050000FC10004010120020EC
:105DD0001212002010B588B000281DDD0A680121CC
:105DE00013000B4018D1042A16D90F201468204044
:105DF000092811D150683F280EDD980010188068DE
:105E00000024084201D04010C4B26846C454013393
:105E1000202BF2D1FFF7AAFF002008B010BD000030
:105E200010B5002813DD0C68E30710D56410532C5F
:105E30000DD8084B1B78002B01D1FFF717FEFFF799
:105E40006DFDA123044ADB00D450FFF74DFD002077
:105E500010BDC046111200200010004010B50028EF
:105E60000EDD0C68E3070BD56410FF2C08D8054B3A
:105E70001B78002B01D1FFF7F9FD034A034BD450E7
:105E8000002010BD11120020001000402405000069
:105E900010B5002805DD0868C30702D54010FFF7DC
:105EA0004BFE002010BD70B588B0002820DD012415
:105EB000086804401CD104281AD90F230268134033
:105EC000042B15D1FEF798F8060007F099F90500A4
:105ED000122800D912252A0002210D326846FFF748
:105EE000A5FD6B465D73A54205DC6846FFF73EFFE6
:105EF000002008B070BD2300325D6B449A730134FA
:105F0000F1E7F0B50D008BB0012832DD0868012201
:105F1000040014402DD104282BD90F2301680B4015
:105F2000042B26D16B68134223D0FEF765F86E6808
:105F300007007310019307F063F905000E2800D9DC
:105F40000E252A000121113202A8FFF76FFD6A46D3
:105F5000127902AB5A7302AA73129373019B7614DF
:105F60001B0ED67313745574A54205DC02A8FFF707
:105F7000FDFE00200BB0F0BD3A5D02A963189A74D3
:105F80000134F1E730B589B0002814DD0C68E3076F
:105F900011D5102268460021FFF748FD6B466A467E
:105FA00065105D73684663122D0E64149373D47389
:105FB0001574FFF7DBFE002009B030BD174B184AFF
:105FC0005968002903D00021596001319160196995
:105FD00000291FD0002018618023DB00D35811490D
:105FE000012B18D1A923DB00D3585B420B600E496B
:105FF0000B78032B01D801330B7003200B490B786E
:10600000013303400B700A495B015B180949535087
:106010000123936070470860FAE7C046FC10004017
:1060200000100040240000209C12002010120020CC
:10603000121200200405000010B50A4B1B78002B3B
:106040000ED0FFF76BFCA1230722074CDB00E250C8
:10605000FFF74AFC0022054B0620E250FFF76CFDDB
:1060600010BDC046111200200010004024050000A1
:1060700010B5034A1021034800F09EF810BDC04639
:10608000B8EE0000AFEE0000044A05491368C8549A
:1060900001339B059B0D13607047C046D01600204E
:1060A000D012002070B5124C124A2368834202DCE1
:1060B0000023236018E0115C451C0E00FA3E012EFF
:1060C00007D8AB4211DD515D002902D028399F2944
:1060D00001D82800EAE70100151A565C6E54013118
:1060E0008B42FADC181A206070BD1170FAE7C046C6
:1060F000DC1A0020DC16002010B5FDF705FD064B6C
:106100001A68824201D900221A601B68C31A034828
:1061100098428041404210BDC8120020204E00002D
:1061200070B5FFF711FAFF250400002801D1200007
:1061300070BD03681B142B401D2B00D10400FFF71A
:10614000F7F8F2E770B5002601250D4C0D4A2368DB
:106150001268934205D00C4AD05CFDF7CFFE0028B0
:1061600006D1002E03D0FDF7D9FC084B186070BD96
:1061700023682E0001339B059B0D2360E5E7C04695
:10618000D4160020D0160020D0120020CC120020FF
:1061900010B50400064B074A1B6812689B1ADB43C4
:1061A0009B059B0DA34200DB10BDFFF7CBFFF1E782
:1061B000D0160020D416002070B5074E33680B2B84
:1061C00008DC0C255D43054C0133285164196160DE
:1061D000A260336070BDC046D8160020402F00205A
:1061E000F0B5B7B0040007F00BF8012802D8002082
:1061F00037B0F0BD23785B2BF9D1013825182B7807
:106200005D2BF4D101343A21200006F0E1FF061E97
:10621000EDD0071B002FEADD210000243A0004A87E
:1062200007F006F804AB711CDC556F1AA742DEDDDF
:106230001DAD3A00280006F0FBFF134BEC551B6820
:1062400003950193019BA342D1DD0C2666430F4BBE
:1062500004A9F618306806F0C9FF051E05D1736859
:10626000B6680293029B9D4201DB0134EAE7306885
:10627000039906F0BBFF37000836002801D1786883
:10628000B6E70135EEE7C046D8160020402F0020C3
:1062900010B5FBF7B9F8FEF7ABFFFBF7DFF8FDF73A
:1062A000C1FDFEF7A9FAFEF747FBFFF7E1FE01F09B
:1062B000FDF801F005FD01F031FD01F07BFF10BD9F
:1062C000962210B512010021034806F00FFC0022AF
:1062D000024B1A6010BDC046481C0020D8050020A3
:1062E00070B514007F22174BC000C0580D008368A2
:1062F00013401C2B01D0002070BDC3681900114051
:106300000429F8D101690A40192AF4D11B0A013382
:106310009B000C30C018FDF76FFE037806000120CB
:10632000002BE9D0300006F06BFF0023A042E2D141
:10633000A34201DB0120DFE7F15CEA5C9142DAD1A4
:106340000133F5E7A825002010B5FDF7E7FB064B64
:106350001A68824201D900221A601B68034AC31AD4
:1063600000209A42404110BDCC120020CF0700000F
:10637000064B074A1B6812689B1ADB439B059B0D63
:106380000122834200DC002210007047D01600205A
:10639000D4160020F8B505000C0016001F1E0ED103
:1063A0000320FFF7E5FF002808D0FA20FFF76CFE76
:1063B000E8B2FFF769FEE0B2FFF766FEF8BD501DD8
:1063C000FFF7D6FF0028F9D0FB20FFF75DFEE8B20B
:1063D000FFF75AFEE0B2FFF757FEF0B2FFF754FEA8
:1063E0003012C0B2FFF750FE3C00E31B9E42E5DDD9
:1063F0002078FFF749FE0134F7E7000070B500246C
:10640000F0250B4B1B68A34202DCFFF759FF70BD60
:106410002B006343074A9B181A78002A05D0597845
:10642000002311201A00FFF7B5FF0134E9E7C04649
:10643000D8050020481C0020F8B507000024F025EE
:106440002B0063430C4A01349E18B74211D03178B7
:1064500000290BD00133D15C002311201A00FFF773
:1064600099FF2A000021300006F040FB0A2CE7D1FA
:10647000F8BD024B1C60F9E7481C0020D80500203D
:10648000F0B5150001222F007A4C1740A544019069
:106490000291002F11D005AB1A706A105A70120EBB
:1064A0001A710522691299706D140299DD70FFF757
:1064B00071FFCF239B009D44F0BD042D2AD90F24EA
:1064C00028680440042C32D1022304AA2800137146
:1064D000FDF792FD050006F093FEC82302009B0025
:1064E000984200DD1A007C1C97420DD1984206D9D3
:1064F000614804AB03226149C01806F0DBFA2200B0
:1065000005AB02990198D2E72700611E695C05ACD2
:10651000E155E8E7042D00D0A7E0032304AA043DD9
:1065200013716B425D4105AB55710222E9E7092CFD
:106530007ED1042205AB1A706A6851100091694639
:10654000521209789A70009A59701F2A01DD202290
:1065500000926A46127806ACDA70009BBB4202DCFD
:1065600005ABE21ACDE70126BB00EB1898680640A0
:1065700006D1042837D90F210368194002290CD10C
:10658000012323704310637042121B0E4014A2704B
:10659000E070237105340137DFE7042921D102239C
:1065A0002370FDF729FD039006F02AFEA31C0C289A
:1065B00009D86070864201D19C19ECE7039A925D7C
:1065C0009A550136F6E70C226270039A925D9A554D
:1065D0000136092EF9D12E23E372237363730E342F
:1065E000D9E7012907D103230438237043425841D6
:1065F00060700234CFE7092909D10423237043686E
:106600005A1062705B12A370E6700434C3E703296A
:106610000BD1052323700068020992B2430F920048
:106620000B40D31A63701B12EDE726700134B2E7FA
:10663000032C00D03DE7052205AB01091A7089B291
:10664000420F890022408A1A11125A709970642AE6
:1066500000DD64220421DA70081F824201DC04326A
:106660004FE7685C58540131F6E7002D00D020E771
:1066700053E7C046C4FCFFFF22030000B0E1000066
:1066800070B502000024F0210D4E0800604380190F
:106690004578954203D001340A2CF6D170BDF02222
:1066A000002106F023FA074A1368013BA34200D1F8
:1066B0001460002329001A001120FFF76BFEEDE79C
:1066C000481C0020D805002010B5B2B002236A464D
:1066D0000400137006F094FDC72800D9C7200023DA
:1066E000984207DC421C6B46FE211420FFF752FE45
:1066F00032B010BD694601335A1EA25CCA54EFE79E
:1067000030B5B3B00500FFF71FFE002816D00223F6
:106710006A462800137006F073FD0400C72800D9EC
:10672000C7240023A3420BDB20003230FFF730FDEB
:10673000621C6B46FF211420FFF72CFE33B030BDE6
:10674000694601335A1EAA5CCA54EBE7F0B5BDB0E6
:1067500005900C00012803DC1B20FBF71DF855E019
:106760002C4B08680393C30709D4042807D90F23C7
:1067700002681340042B02D1FDF73EFC0390254B29
:1067800060680493C30709D4042807D90F2302685B
:106790001340042B02D1FDF72FFC049000261E4B62
:1067A0001B680893089BB3420BDC049B1B4A0093B5
:1067B000C821039B0AA806F0ABFC0AA8FFF7A0FFBC
:1067C000CAE70C257543164B0399ED18286806F0A7
:1067D0000DFD071E05D16B68AD680993099B9F42AB
:1067E00001DB0136DEE728680499079506F0FEFC18
:1067F0000835069000280BD121000598079B083129
:106800005B6802389847074B069A1A603DB0F0BDA6
:106810000137E3E7F3E60000D816002019F0000086
:10682000402F0020E40F0020F7B5234B06001B6823
:10683000F02100930023009A9A4211DC0024F023F7
:106840001A006243019201991C4A55182F78002FB3
:1068500012D001340A2CF3D11948FFF751FF29E077
:106860000A005A43154882185078B04202D1127873
:10687000002A1FD10133DEE7F0223900280006F09C
:1068800035F902230D4A0199EB6053540D4AF1008A
:106890008A58009B6E70AE70AA602F616F61A34230
:1068A00002DC054B01341C60002331001A0010206B
:1068B000FFF770FDF7BDC046D8050020481C00203A
:1068C00061F40000A825002010B5FFF797FDFF2414
:1068D000084AE3005B429B18074AD35C043B012B48
:1068E00003D8E043C0B2FFF79FFF013C002CEFD17B
:1068F00010BDC046FC070000A8250020F8B5050023
:106900000E00FDF799FDFF240D4B18600D4AE300C2
:106910005B429B180C4AD35C062B01D0032B0BD196
:10692000E743FFB2320029003800FFF7D9FC002806
:1069300002D03800FFF778FF013C002CE6D1F8BD0B
:1069400008000020FC070000A825002070B5050005
:10695000FF24084AE3005B429B18074AD35CAB4222
:1069600003D1E043C0B2FFF75FFF013C002CF0D140
:1069700070BDC046FC070000A8250020F7B5FDF754
:10698000C3F8574B1A68824201D900221A601A686C
:106990005449821A8A420DD9FF2253491860D30004
:1069A0005248CB1A1B181B78073B022B0CD9013A13
:1069B000002AF4D1F7BD0720FFF7C8FF4C4B27E0B2
:1069C0000820FFF7C3FF38E0FDF7A8F8071E00D145
:1069D00001270020FDF754F901900020FDF764F92C
:1069E000019B0090434C444D002B12D02368002B98
:1069F0006ED12B682760002B6ED0404B01261B7890
:106A0000002BD8D10920FFF7A1FF394B1E703B4B5B
:106A10001E70009B002B12D02B68002B0FD1236817
:106A20002F60002B1ED0324B01261B78002BC7D1C4
:106A30000920FFF78BFF2E4B1E70304B1E70236812
:106A4000002B0FD02A4E3278002A0BD19F4200D261
:106A500027602368FB1A312B04D90720FFF776FF44
:106A6000012333702B68002B0FD0244E3278002A7C
:106A70000BD1BB4200D92F602B68FF1A312F04D9EC
:106A80000820FFF763FF012333702368002B0CD02D
:106A9000019B002B09D1164E3378002B02D1072021
:106AA000FFF754FF0023236033702B68002B00D1C5
:106AB00080E7009B002B00D07CE7104C2378002B54
:106AC00002D10820FFF742FF00232B60237071E7FB
:106AD000009A002AA0D1B5E7009B002B9FD1AEE71A
:106AE000C41200200F270000A8250020FC0700008A
:106AF000B8120020B4120020BC120020C0120020E6
:106B000013B50400FFF77AFCFEF7EDFE00230093B7
:106B1000134B1B68002B02D16846FDF799F804233C
:106B200001A901200193FEF749F800210800FDF7B3
:106B3000FFFFFEF70DFAFFF77FFAFDF7C9F8FDF743
:106B40004DF9FDF767F9FEF749FBFDF709F8002C51
:106B500004D0FDF7FDF90348FFF7D2FD13BDC04691
:106B6000F41A002052F40000002310B501001A00AE
:106B70001120FFF70FFC10BD07B56B461970694671
:106B80005A7013128B701314120ECB700A716B466D
:106B9000010005221320FFF7FDFB07BD10B50A0019
:106BA00001001220FFF76CFC10BD70B505000C0051
:106BB000FFF7CAFB002809D020003230FFF7E8FABF
:106BC0002B00220000211B20FFF7E4FB70BD10B555
:106BD0000C000300110014202200FFF7DBFB10BDA6
:106BE000012370B5FF24084A41185B42884201D353
:106BF000D84370BD06781D0A234073409B009B5804
:106C000001306B40F2E7C04634F0000013B50400D9
:106C1000FE2813D80A4BC200D05800280ED0436873
:106C200008309900FFF7DCFF01900920FFF7B0FA68
:106C300001AB042221001720FFF7ACFB13BDC046B7
:106C4000A8250020F8B500231800254DDA00AA5821
:106C50000133511E8A418018FF2BF7D1052444438C
:106C60000A20FFF795FAFB20FFF70EFA2720FFF71F
:106C70000BFA0020FFF708FAE0B22412FFF704FA3B
:106C8000E0B2FFF701FA174BFA21186803F0EAFDAA
:106C900000260700F300E85800281CD0436808309D
:106CA0009900FFF79DFF04000520FFF771FAF0B28D
:106CB000FFF7EAF9E0B2FFF7E7F92004000EFFF76B
:106CC000E3F92002000EFFF7DFF9200EFFF7DCF9F1
:106CD000380001F017FF0136FF2EDBD1F8BDC046AA
:106CE000A825002004000020F7B50190FFF718FA4E
:106CF00001250400FF276D42002C01D12800FEBDB4
:106D0000266833143B40152B0DD121000198083122
:106D100006F06CFA002801D135123D402000FEF744
:106D200007FB0400E8E71D2BF8D101256D42F5E7CC
:106D3000F0B5A1B0FFF706FA8021A64CA64F206857
:106D4000C900091AC019FDF7BFF82368C0182060F0
:106D5000002811D0FCF7D8FEA04B18603B78FA2B26
:106D600000D049E12368022B08DCFFF7C5F90028B1
:106D700002D00120FFF796F921B0F0BD7B78BC78F6
:106D8000981E242800D919E103F0D8FC250038000A
:106D90003C00400043004C0018015600880092005F
:106DA0009900AF00EE000501180118011801180143
:106DB0001801180118011801180118011301180110
:106DC00018011801180118011801180118011801FB
:106DD000180118019600FF2C0ED02000FFF750FC80
:106DE00000227F4BE100CA505B181A71210000920B
:106DF00013001320FEF714FD0320BBE72000FFF76C
:106E000013FDF9E72000FFF73BFCF5E7FFF75CFD1A
:106E1000F2E7FFF7F3FA0020FFF772FE7148FFF781
:106E20006FFCE9E7632CE7D86F4BA200D258210032
:106E30001520FFF725FBDFE7FFF772F9FF270400B6
:106E4000002CD9D025682B143B40152B04D02000F2
:106E5000FEF76EFA0400F3E72000083006F0D0F9E0
:106E600006000530FFF794F9FB20FFF70DF92D120E
:106E70001D20FFF709F9E8B2FFF706F9F0B2FFF7B6
:106E800003F93012C0B2FFF7FFF825002B1B9E421A
:106E9000DDDD287AFFF7F8F80135F7E700211D203E
:106EA00000910B000A00FEF7BBFCFDF751F8A3E7C9
:106EB0002000FFF7ABFE9FE7FFF7C4FE9CE7FCF75F
:106EC0003BFE07AC494A64210090494B200006F084
:106ED0001FF902232000237006F092F9230002001C
:106EE00000211620FFF756FA86E7424BFA21186870
:106EF00003F0B8FC00260490394AF3009B181C6884
:106F0000002C28D01B790593636808349F00B81DB6
:106F10000393FFF73DF9FB20FFF7B6F801207D1C36
:106F2000FFF7B2F8F0B2FFF7AFF8E8B22D12FFF7B3
:106F3000ABF8E8B2FFF7A8F80598FFF7A5F8E7194E
:106F4000A7420CD8FFF7FEF8049B0398584301F0C2
:106F5000D9FDFFF7F7F80136FF2ECDD14CE72078A9
:106F6000FFF792F80134EBE70024FFF747FA23001C
:106F7000220021000094DA20FEF752FCFF222100BB
:106F8000D200174805F0B2FDFCF7E2FF2100200017
:106F9000FDF7CEFD30E7012C02D1FEF7F3F92BE728
:106FA000022C02D1FEF738FC26E70120FFF7A8FDEE
:106FB00022E7002321001A001A2093E71A00C83A9A
:106FC000052A00D918E7002218001100FAF752FA32
:106FD00012E7C046DC1A0020DC160020C812002090
:106FE000A825002034F40000A02D00204BF4000060
:106FF00046F4000004000020FB2B00D0B9E6226814
:10700000042A00DCB1E63E79F878614B360206438B
:107010009E4200DDADE6331D9A4200DCA5E6FB5C36
:10702000FE2B00D0A5E67878BC78751E1B2869D0A9
:107030001AD807284FD0082824D0012819D1FF2CAE
:1070400010D02000FFF71CFB7D79524AB31E00923E
:1070500021002A000A20FEF7E3FB4F4BE400E0503A
:107060001B191D71701D85E61D285DD04FD31E288C
:1070700071D00300C83B052BF4D8484A2900FAF721
:10708000F9F9EFE7632CEDD87A79022A13D0032AB5
:107090001BD0012AE6D1F979BB79090219433B7A61
:1070A000A4001B0419437B7A1B060B435B001343AC
:1070B0003B4AA350D6E7002DD4DDB11E3548FDF77D
:1070C000BBF9374BA400E050CCE7BB79A4005A1EB3
:1070D00093419B00ECE7632DC4DC07AF2A002F49E6
:1070E000380005F0E7FC002338007B55FFF7FCFD76
:1070F0000028B7DB2A4B8000C25821001520FFF77B
:10710000BFF9AFE729002548FFF7F8FBAAE7FF2CF6
:10711000A8D07A79022AA5D81E490B200091210017
:10712000B31EFEF77DFB9DE7632D00DD6325002385
:1071300007A99D420ADCEB430022DB172B40CB184A
:107140001A70152000916B1C2100EAE7FA18527999
:10715000CA540133EDE7022C13D0032C14D0012CB8
:1071600000D07FE7002D00DC7CE77B79002B03D08B
:107170001C00322B00DD322464235C43094B1C606D
:1071800070E7FEF7AFFB6DE7FEF7ADFB6AE7C046C1
:10719000F6030000E2160020A8250020E1160020DA
:1071A000A02D0020040000200120704710B5064CDF
:1071B000200001F013F90549200001F043F90122F4
:1071C000034B1A6010BDC046181B0020801A060031
:1071D000E01A00201FB500211020FCF7B3FC0121AC
:1071E0001120FCF7AFFC01211620FCF7ABFC1C4C76
:1071F000200001F051F81B4B1B4A1B6812681B4909
:10720000D2B28B420BD880239B04019301AB1A713D
:107210000199029A0023200001F05AF81FBD144979
:107220008B4202D88023DB04EFE712498B4202D85D
:1072300080231B05E9E710498B4202D880235B05B8
:10724000E3E70E498B4202D880239B05DDE70C491A
:107250008B4202D88023DB05D7E780231B06D4E7C7
:10726000F81A0020300000202C00002048E801001F
:1072700090D0030020A1070040420F0080841E0030
:1072800000093D0010B5002815DD01240B682342DC
:1072900011D023410C4A13600C4AA04209D04B681C
:1072A000234206D02341022B09D0032B09D0A3424D
:1072B00003D002231360002010BD0023FAE703234C
:1072C000F8E71460F7E7C046300000202C000020EB
:1072D00010B500280FDD0C68E3070CD56410012CF5
:1072E00009DD064B1B68002B01D1FFF75FFF210072
:1072F000034801F0A7F8002010BDC046E01A0020A6
:10730000181B0020F8B501250868284203D10D207C
:10731000FAF742FAF8BD4010FCF738FC041E14DB03
:10732000FCF70EFCA04210DB02212000FCF70AFC57
:10733000FA222900D200200001F016FC0025A84204
:1073400005D101002000FCF7FDFB0020E2E700274B
:107350000726FA2201219200200001F005FC0028F6
:10736000F3D0282802DD0123B3401F43013EF0D2B1
:107370000E4EAF550135052DE9D100212000FCF757
:10738000E1FB012206210920FCF7D8FF0028DCD010
:107390000B23012443600023F25C99005200411842
:1073A000224301338A60052BF6D1B3E7E41A0020AB
:1073B00070B500281EDD0D68EB071BD4042D19D90C
:1073C0000F242B681C40032C14D11A0992B25B0FB6
:1073D00092001C40141B2E00FFF7FCFE731B064896
:1073E0009C4205DD317900F079FF0136F070F5E758
:1073F00000F073FF002070BDF81A002010B504687B
:107400000D20E30703D56410FF2C03D91720FAF7EA
:10741000C3F910BDFFF7DEFEE1B2044C200000F01E
:107420005DFF200000F059FF0020F2E7F81A00206D
:1074300070B5FFF7CFFE064D0021280000F04EFF8B
:107440000400280000F049FF01206400204370BDC3
:10745000F81A0020A02101220B4BC9005A500B48FA
:107460000B4958500B491A604A68002AFCD0002288
:107470004A60A121C900585801215960A021C900C2
:107480005A50054BC0187047007000406A10000049
:1074900004050000FC700040FBFDFFFF10B5FFF786
:1074A000D9FF43000120184310BD000010B5034A66
:1074B0000F210348FEF780FE10BDC04678F400009F
:1074C000F0F400000D4B70B51B6804000E001500B1
:1074D000002B01D1FFF76AFEE1B2094C200001F058
:1074E00048F8F1B2200000F045FFE9B2200000F0BA
:1074F00041FF200001F0A8F870BDC046E01A00204E
:10750000181B002010B501240368234205D04168F0
:10751000214202D08268224203D10D20FAF73CF9C1
:1075200010BD5810802801D91520F7E74910FF2910
:1075300001D91620F2E75210FF2A01D91720EDE7F2
:10754000FFF7C0FF0020EBE710B5002803DC1C208C
:10755000FAF722F910BD0B68DA0701D40D20F7E71E
:107560005B100322012B06DD0522022B03D00C2227
:10757000042B00DC08220F211820FFF7A3FF0220B4
:1075800001F0C0FA0020E5E7F7B5012214009042AF
:1075900026DD0D682A4223D02D4B15411B684C680F
:1075A000002B01D1FFF702FE2A4EE9B2300000F0B5
:1075B000E0FF27000122174014D01441FF2C02D90C
:1075C0001720FAF7E9F8E1B2300000F0D3FE3000FE
:1075D00001F03AF80024A04202D02320FAF7DCF8A8
:1075E0002000FEBD042CF2D90F2523681D40092D73
:1075F0001CD1636801925B100093009BBB42E6DDE7
:10760000BB00E3189D68019B1D420BD06D10FF2D40
:1076100002D91720FAF7C0F8E9B2300000F0AAFE4C
:107620000137EAE71720FAF7B7F8F9E7032DCED1CB
:1076300027001A0992B25B0F92001D40551B3B1B9D
:107640009D42C4DD3979300000F094FE0137F6E741
:10765000E01A0020181B0020154B70B51B680500B0
:107660000E00002B01D1FFF7A1FD124CEDB2290055
:10767000200000F07EFFF1B2200000F07BFE002130
:10768000200000F081FF002801D0404270BD72B69A
:1076900001222900200000F067FF62B6200000F000
:1076A0005AFE0028F2D0200000F05AFEEEE7C04655
:1076B000E01A0020181B002010B5012403682342A3
:1076C00002D04168214203D10D20FAF765F810BDC0
:1076D0005810802801D91520F7E74910FF2901D952
:1076E0001620F2E7FFF7B8FF40002043EFE7000065
:1076F00070B5284D04002B68002B08D105211820F7
:10770000FFF7AAFF022001F0FDF901232B60012CF5
:1077100014D105211820FFF79FFF7F282BDC0300E1
:107720007F3301DA7F204042C8235B4258437F21E8
:1077300003F098F8052C00D1404270BD032C11D104
:1077400021001820FFF788FF7F2814DC03007F3317
:1077500001DA7F204042C8235B4258437F2103F077
:1077600081F8EAE70020052CF5D107211830FFF752
:1077700073FF7F2802DD0138FF38D0E703007F3335
:1077800001DA7F204042C8235B4258437F2103F047
:1077900069F8D1E7EC1A002010B50120FFF7A8FF27
:1077A00043000120184310BD10B50320FFF7A0FFD0
:1077B00043000120184310BD10B50520FFF798FFC6
:1077C00043000120184310BD10B508211820FFF711
:1077D00043FF0300C00FC0180123401015304000C4
:1077E000184310BDF8B5514B05001B68002B01D1A3
:1077F000FFF7DCFC4E4C23787F2B00D892E007216A
:107800000E20FFF729FFC42833D101220E26494B51
:1078100010211A70484B30001A702670FFF752FE84
:10782000802211213000FFF74DFE00216156002912
:107830001EDB424EC9B2300000F09BFE3D4B3000D3
:10784000197800F097FD300000F0FEFE2178062246
:10785000300000F089FEAC1D300000F07CFD0028F7
:1078600006D0300000F07CFD28700135A542F3D130
:10787000F8BD0F211920FFF7EFFE33280FD1682242
:107880002C4B1E261A7000222B4B60211A703000E0
:107890000C322670FFF716FE02226121C2E700219A
:1078A0001820FFF7D9FEFA281CD14222214B1026BE
:1078B0001A700022204B4B211A70300001322670C2
:1078C000FFF700FE042001F01DF938224C213000A2
:1078D000FFF7F8FD0F2251213000FFF7F3FD1B22C7
:1078E00052219FE70F211C20FFF7B6FE3D289CD1B7
:1078F00028221C2600270F4B20211A700E4B263AF7
:1079000030001F702670FFF7DDFD3A0022213000A5
:10791000FFF7D8FD3A0023213000FFF7D3FD4022C6
:1079200024217FE70021615683E7C046E01A00204A
:10793000340000203600002035000020181B0020F5
:1079400073B5002606220021684605F0CFF8684688
:10795000FFF748FFFFF7ECF91A4B6A469E576C4653
:107960006B4691781878D5785B7812796479002E17
:107970001FD000020902034329431BB209B21202BD
:1079800011482243007812B240B2102802D152109E
:10799000DB10C910D8171B184340C81709184140FD
:1079A00001205918D317D2185A408A185200104390
:1079B00076BD1B022D02034329431BB209B22402E8
:1079C000DEE7C0463500002034000020F8B5012372
:1079D0001C0098422BDD0F683B4228D04E683500D2
:1079E0001D4024D1042E22D90F2231680A40092AD1
:1079F0001DD173685C10202C00DD2024144B1B6803
:107A0000002B01D1FFF7D2FB72B67F10F9B2114FF4
:107A10002200380000F0A8FD62B6A54214DA380052
:107A200000F099FC002804D101246D002C432000B3
:107A3000F8BD380000F094FC0122AB004000F318C0
:107A400010439860AD18E8E764000125EEE7C046F2
:107A5000E01A0020181B002070B52B4B86B01B6865
:107A6000002B02D10120FFF743FE01AD14220021BB
:107A7000280005F03BF8254E1821300000F079FD74
:107A80000321300000F076FC0021300000F07CFD86
:107A9000041E13D172B605221821300000F064FDD7
:107AA00062B6300000F057FC002802D0300000F031
:107AB00057FCA3000134E850052CF2D1019B7F2B29
:107AC00001DD013BFF3BAA687F2A01DD013AFF3A55
:107AD00029697F2901DD0139FF39C8204343424329
:107AE0004843DB11D2115243C0115B4340439B1802
:107AF000181804F0C7FE01F091FB04F08DFE43005E
:107B00000120184306B070BDEC1A0020181B00209D
:107B100010B5054C2368002B02D01B20F9F73CFE62
:107B20000020206010BDC046F01A002010B50028CB
:107B300003DC1C20F9F730FE10BD0B68DA0706D411
:107B4000042B04D90F221B681340032B01D02420DF
:107B5000F0E7034B25201B68002BEBD01B20E9E747
:107B6000F01A002010B5002803DC1C20F9F714FEE1
:107B700010BD0B68DB0701D40D20F7E71B20F9F7D8
:107B80000BFE0020F4E700001D4B70B51B680C00D5
:107B9000002B03D12520F9F7FFFD70BD012801DC82
:107BA0001C20F8E708680121084207D1042805D9FC
:107BB0000F2302681340DD1E8D4201D92420EAE71D
:107BC00065680D4201D11120E5E7042B0BD1FCF7CC
:107BD00013FA05F015FB63685B10013B01D4834287
:107BE00008DB1220D7E7100980B252008000920F04
:107BF000801AF0E71B20F9F7CFFD0120CDE7C04642
:107C0000F01A002010B50400802803DD2620F9F7C3
:107C1000C3FD10BD002CFCDD1B20F9F7BDFDFEF7F8
:107C2000ADFEFFF785F8012000F06CFFF2E70000E1
:107C300010B5002805DC1C20F9F7AEFD040020007B
:107C400010BD184B1B68002B01D12520F4E701243F
:107C5000086804400FD04010FF2801D92820EBE726
:107C60001B20F9F799FDFEF789FEFFF761F8012067
:107C700000F048FFF4E70428E1D90F210268114021
:107C8000042906D1FCF7B8F905F0BAFAFFF7BAFFF4
:107C9000D5E70329D3D1100980B2520F80000A40E2
:107CA000801AF3E7F01A0020044B10B51B6825205A
:107CB000002B00D01B20F9F76FFD10BDF01A00203B
:107CC00010B5034A06210348FEF776FA10BDC046F8
:107CD0009CF50000CCF500000020704701207047A3
:107CE0000020704700207047002070470120704737
:107CF0000020704700207047002070470020704728
:107D00000020704700207047002070470020704717
:107D100000207047704770477047000010B5034A55
:107D20000F210348FEF748FA10BDC046ECF50000ED
:107D300064F600000378013B1F2B00D97047013027
:107D4000F8E710B5FFF7F6FF0378002B0BD00130F2
:107D5000222B11D10378002B03D0421C222B03D1FC
:107D60001000FFF7E7FF10BD5C2B03D14378002B19
:107D700000D0821C1000EDE73A2BF2D02C2BF0D073
:107D80007B2B0BD1FFF7D6FF0378002BE9D07D2B9F
:107D900001D10130E5E7FFF7D4FFF5E720225B2BA7
:107DA00014D1FFF7C7FF0378002BDAD05D2BF0D09A
:107DB000FFF7C7FFF7E7202BD3DD2C2BD3D019001B
:107DC00091435D29CFD0222BCDD001300378002BF9
:107DD000F1D1C6E7002210B5904216D0FFF7AAFFF6
:107DE00003780422222B10D0023A7B2B0DD0013ACB
:107DF0005B2B0AD0190030390232092905D92D2B05
:107E000005D14178303909290AD8100010BD052262
:107E1000742BFAD00132662BF7D001326E2BF4D0DE
:107E2000581E83415A42F0E770B5FFF783FF03788D
:107E300001222D2B01D18018023A00230A2502E0ED
:107E40006B430130CB1801783039CCB2092CF7D90B
:107E50005A43100070BDF8B50C001500FFF76AFF1B
:107E60000378222B02D000232370F8BD0D236A1E55
:107E7000210008250C260A279C4601300378222B76
:107E800002D100230B70F0E7002BFAD0441C5C2BCE
:107E90000BD14378841C622B0ED0662B0ED06E2B38
:107EA0000ED0722B0ED0742B0ED0002AE9DD0B7091
:107EB000013A01312000E1E72B00F6E73300F4E757
:107EC0003B00F2E76346F0E70923EEE710B5040054
:107ED000FFF737FFA04203D90378013B1F2B00D9DE
:107EE00010BD0138F6E710B5002815D00378002B37
:107EF00013D0FFF71FFF2021037802008B430020DF
:107F00005D2B09D01000FFF71CFF03782C3B5A4271
:107F10005341C018FFF70EFF10BD1800FCE7030027
:107F2000002070B50C0081420EDD1A785B2A0BD15F
:107F3000581CFFF7FFFE0125AC4205D0FFF7D3FF29
:107F4000002801D00135F7E770BD70B50C001500B1
:107F5000002901D000230B70002820D00378002BCB
:107F60001ED0FFF7E7FE037806002C2B03D101306B
:107F7000FFF7E0FE0600337800207D2B0FD084420F
:107F800004D02A0021003000FFF765FF3000FFF722
:107F9000D8FE03783A2B02D10130FFF7CBFE70BD3B
:107FA0001800FCE7F0B50D0004009DB02E78002EFF
:107FB00035D02E21280005F00BF9071E14D0431BE5
:107FC0000193303E092E14D82800FFF72DFF010041
:107FD0002000FFF7A4FF0400002C20D0002F1ED0AB
:107FE000019B0133ED18E1E7280005F009F9019044
:107FF000E7E723787B2B11D1601C642203A9FFF7EC
:10800000A4FF041E0BD0019A290003A805F0FFF875
:108010000028E1D02000FFF794FEEEE700242000C6
:108020001DB0F0BD70B5050000200C0081421DDDC3
:108030002800FFF7CFFE0300681C012B14D000209E
:10804000022B13D10022681C1100FFF77EFF012CC8
:108050000CD0FFF748FF00221100FFF776FF013C2C
:10806000F5E7FFF740FF013C012CFAD170BDF8B5F0
:10807000050000200C0016001F0081420DDD2800C5
:10808000FFF7A8FE03000020022B06D1681C3A006F
:108090003100FFF75AFF012C00D1F8BDFFF723FF95
:1080A0003A003100FFF751FF013CF4E710B500241E
:1080B000A04218D0FFF73EFE03787B2B0AD1013097
:1080C00000221100FFF741FF00280CD0FFF739FE16
:1080D0000134F5E75B2B06D10130FFF704FF0028E0
:1080E00001D00134F9E7200010BDF8B5002816DDF5
:1080F0000D68EB0713D56D10013D0124FDF724FA3F
:108100000026FF27644200280CD1002E21D0300029
:1081100005F076F801003000FCF78EF9F8BD012576
:108120006D42EAE703681A143A40152A0BD11B1274
:108130003B409C4200DA1C009D4201D106000836FB
:10814000FDF7F6F8DFE71D2AFAD101240026644284
:10815000F6E70120013464002043DFE710B508682A
:108160000C00FBF749FFFEF7BFFD002803DB626848
:10817000024B8000C250002010BDC046A02D002040
:1081800010B50868FBF738FFFEF7AEFD01230028A5
:1081900002DB024B8000C358180010BDA02D002048
:1081A00010B50868FBF728FFFEF79EFDC043C00F1F
:1081B000800010BD10B5034A04210348FDF7FCFF01
:1081C00010BDC04600F70000FAF6000010B5FBF73E
:1081D00035FEFBF7E3FEFEF75BF80448FEF790FA86
:1081E000FDF710FAFEF770FB10BDC0464FF7000018
:1081F00010B5FBF771F910BD70B5002504AC2478FB
:108200000573A94205D10A4B0A4A25210A4804F000
:10821000E3FB01600949920052589B0002715B58D0
:10822000A40083716358856043710223C37170BDDC
:1082300067F70000C6F7000075F7000024F800009B
:10824000037B002B04D143738373036101330373F6
:10825000704700001FB50191A02100240068C900EB
:10826000D2B24450012A10D0A24209D0032A0AD027
:10827000074A8350074B019AC250012343501FBD48
:1082800002221343F4E70422FBE70622F9E7C04683
:10829000540500002405000010B50400FFF7D0FFCE
:1082A000A1222368A179D20099506179064A200061
:1082B0009950217904329950044B19685A689B6887
:1082C000FFF7C8FF10BDC0460C0500000C1B0020C6
:1082D0001FB5FFF7BFFF05B000BD70470368074A31
:1082E00099501A00FC32D1680029FCD0A321C900A2
:1082F00058580023C0B2D3607047C0461C05000028
:1083000007B58022074BD2051A6000229A6002321C
:108310001A7111230E320093034905330348FFF706
:108320006BFF07BD0C1B002000300040F81A002036
:10833000F8B505000E0017000024BC4208D02B68D9
:10834000315D1B6828009847002801D00134F4E70C
:108350002000F8BD704710B51C3000F0AFF910BD1B
:1083600010B51C3000F09CF910BD10B51C3000F0A9
:10837000ABF910BD70B5437E0D00002B01D100207C
:1083800070BD6430040000F0A8F90028F7D1200087
:10839000290000F076F90120F2E70000F7B501931B
:1083A000FA23002504009B0083600B4B45600833D3
:1083B00003601C300F00160000F058F920006430F4
:1083C00000F054F96B461B79276166756576A576D2
:1083D0002000A375FEBDC04604F80000012330B59F
:1083E000A024C375837D13499B005A58437DC13235
:1083F000114DFF32E40592009B005B581551CC22D1
:10840000C133FF339B001D5104690C4B5204E250F1
:1084100005220469243BE250837D04699B005A587D
:10842000A123DB00E250437D02699B005958044BB5
:10843000D15030BD24F800000C06000024050000D7
:108440000C050000A022002310B50469D200A3503F
:108450000A4CA1420FD90A4C8C425B4109495B424C
:108460000B40CD21C9045B180469074963500521FD
:108470000369995010BDCC235B04F5E7A086010089
:1084800090D00300000098FD24050000F7B504001B
:1084900000200D000193824265D01600402A00D9C9
:1084A000402627001C37380000F0F6F8B123226977
:1084B000DB00D55080220123216992008B50A27EDF
:1084C000002A03D122691362226913600025731EFA
:1084D000AB4207D1019B002B04D0802202212369EB
:1084E00092009950012223691A622369FC33DA68E9
:1084F000002A02D19A6A002AF9D09A6A002A0BD17E
:10850000DA60A3232269DB00D1583800C9B20135F3
:1085100000F0B7F8B542DAD3019B2269002B0FD1E6
:108520001300FC339B6A002B0AD10133A376D3617D
:108530002369FC33DA6C002AFCD00022DA640AE0FA
:1085400000230121A37651611A002369FC33996845
:108550000029FCD09A602369FC339A6A002A01D072
:1085600000229A62E8B2FEBD10B50123FFF78EFF2C
:1085700010BD0300AC3310B504001970643000F076
:108580008BF80123637610BD0023020070B5AC3276
:1085900043760D001178B12204000069D2008150A9
:1085A0008022216992008B50226901331362226973
:1085B000936026006436300000F080F8002812D066
:1085C000300000F06DF81E4B2269D0502369FC3357
:1085D0001A6A002A02D19A6A002AF9D09A6A002AF5
:1085E00001D11A62E5E723690122002D0DD119009E
:1085F000FC31896A002908D1DA612369FC33DA6C1D
:10860000002AFCD00022DA6407E05A612369FC33B7
:108610009A68002AFCD000229A6000202369FC336B
:108620009A6A82420BD098622169064A8B588B5015
:108630001800022B03D0181F431E9841033070BD51
:108640001C050000C404000010B50121FFF79CFFC9
:1086500010BD000010B51323122202490248FFF793
:108660009DFE10BD00400040181B002010B54022A8
:108670000021040004F03AFA00232000236463641C
:1086800010BD10B53F24026C531C2340446C9C4227
:1086900001D08154036410BD002303644364704718
:1086A000436C026C934206D03F21C25C01330B4005
:1086B00043641000704701204042FBE7036C406CAC
:1086C000181A00D540307047436C026C934201D0B9
:1086D000C05C704701204042FBE73F22036C406CC6
:1086E00001331340181A43425841C0B2704700008A
:1086F00003210A4802680A430260094802680A43E3
:1087000002600849084A094B9B1A03DD043BC8581C
:10871000D050FBDC00F012F8F7F7F6FC240500401F
:108720005405004068FD0000000000207002002099
:10873000FEE7FEE7FEE7FEE7FEE7FEE7014B024A43
:108740001A607047380000200024F40001207047B0
:1087500010B503681322DB69984710BD704700000D
:10876000054B0269D1500369FC331A6A002AFCD018
:10877000002201201A6270471C050000030010B59A
:108780005C331A781F231A401E3B19009140114A8E
:10879000D167C222042104699200A150026953608A
:1087A0000269D360A02300220169DB00CA500123C3
:1087B0000169094A5B428B500169084A8B50016983
:1087C0000C3A8B50016908328B501430FFF764FF6C
:1087D00010BDC04604E100E00C05000014050000D7
:1087E00010B51430FFF76AFF10BD10B51430FFF755
:1087F0006BFF10BD10B51430FFF752FF10BD000025
:10880000030070B55E331A780469724BE2500300BE
:108810005D331A780469704BE250030061331C78B1
:1088200002696E4B012C00D09EE005005F352E786A
:10883000A225ED005651020060321578A12206698A
:10884000D200B5500269D4509623DB00994200D87B
:108850008CE096231B01994200D88AE096235B01A5
:10886000994200D888E096239B01994200D885E080
:10887000E1239B01994200D882E09623DB019942D3
:1088800000D880E0E123DB01994200D87DE0962307
:108890001B02994200D87AE0E1231B02994200D8DA
:1088A00077E096235B02994200D874E0E1235B02F3
:1088B000994200D871E0E1239B02994200D86EE012
:1088C000474B994200D86CE0E123DB02994200D883
:1088D0006AE0E122002312038A425B41414A5B4283
:1088E0001340802252059B1801693F4A8B50A023F8
:1088F00004220169DB00CA5000210369FC33D960FE
:108900000369FC331962012301690B6001698B6003
:10891000C1210469890062501F215C3002780A403D
:1089200093406231314AFF315350002141560029B2
:108930003CDA0F230B40083B2D4C9B089B001B1976
:1089400003242140A140FC348C40DD69A5432C0068
:10895000C0258D4029002143D9611F23017819408A
:108960001E3B8B40136070BD00246CE79E23DB022E
:10897000BAE79D231B03B7E71E4BB5E71E4BB3E7D2
:10898000EC239B03B0E71D4BAEE71D4BACE71D4B43
:10899000AAE71D4BA8E71D4BA6E71D4BA4E71D4BFF
:1089A000A2E78023DB049FE71B4B9DE78C080F4B5E
:1089B000A400E41803230B40FF21C025DB009940ED
:1089C000AD0066598E433100C0269E4033000B43F4
:1089D0006351C2E70C050000140500006C0500009F
:1089E00090D0030000D0BEFE2405000000E100E0AE
:1089F00000ED00E000B013000050270000A04E0082
:108A000000F0750000509D0000F0EB0000903A016E
:108A100000E0D70100B0AF0300705F07F7B5009327
:108A200008AB1B7800250193FA2304009B008360A8
:108A30000E4B45600833036014300F001600FFF73B
:108A400015FE23005C3327611E70009B084A9B00C3
:108A5000995823005D331970019B20009B009A58A0
:108A600023005E33DD701A70FEBDC046A0F8000022
:108A700024F80000036910B51A00FC32D268040023
:108A8000002A0AD0A322D20099581430C9B2FFF7A5
:108A9000F8FD00222369FC33DA6010BD10B50248EE
:108AA000FFF7E8FF10BDC046D01B00201D2307B50F
:108AB00002220093024901330248FFF7AFFF07BDCE
:108AC00000200040D01B002010B5002801D004F089
:108AD000C9FA10BD0849094A094B10B51B688858E6
:108AE000FA22190A1B0618439200002301F0F2FF34
:108AF0004904C00B084310BD0010014004050000EC
:108B0000341C002070B5041E09D0FFF7E3FF0500F8
:108B100000F014F8FFF7DEFF401BA042F8D370BD51
:108B20000022044B9A60044A13680133DBB21360DD
:108B30007047C046FC100140341C0020704770474D
:108B400010B500F05FF8FFF7FAFF0120FFF7DAFF3A
:108B5000FFF73CFBFFF74CFB024B002BFAD000E089
:108B600000BFF7E700000000F8B54C1EA141012549
:108B7000104B114F8000C3584C4238680F499D403C
:108B8000160001F0E5FD0A21704301F0E1FD2C40E3
:108B90000300220029000A4800F016F8FA21094CC7
:108BA00089004443386801F0D3FD0100200001F042
:108BB000CFFDF8BD24F800003800002040420F002F
:108BC000100500501027000030B504680C40944296
:108BD00006D1013B002BF8D112E0013B002B0FD056
:108BE00004680C409442F8D1002405680D40954279
:108BF00004D101349C42F8D1002002E0201C00E0A6
:108C0000181C30BDC420114B80001A581049114067
:108C1000C02212020A431A50C02180224900920247
:108C20005A501A608023A3220021DB05D2009950FC
:108C30000122F9309A60074BFF301950C1200231F0
:108C400080001950403019501A60704700E100E070
:108C5000FF00FFFF00100140014B18607047C04645
:108C600084000020F7B500231E285AD8384B800016
:108C7000C258042A5BD007D8022A54D055D80423FE
:108C8000012A09D000234CE0062A54D051D31A2AD5
:108C900053D002231B2AF5D12E4A116808294ED938
:108CA00009294FD00A240226A02001252A4AC00003
:108CB00015502A482A4D07681C20BF000740294844
:108CC000019700685759009027481B0207401F432F
:108CD000C02300989B020340FF20575157590002C0
:108CE00007401F43019B1F43009B5801602318400E
:108CF00007433E43565101251C4B15605868002818
:108D0000FCD000205860A1230125DB00D35855601A
:108D1000A025ED0050511BB2A14202D015D2611A1C
:108D2000CB401800FEBD0823B6E71023B4E720238C
:108D3000B2E74023B0E78023AEE70123ACE7082485
:108D40000026B1E70C000126AEE7091B8B40E8E7DF
:108D500024F8000080000020007000403C0000204B
:108D60000405000040000020FF00FFFFFC700040F1
:108D7000F0B51E285BD8364B8000C258354B1E68B4
:108D8000002E30D1C227344BBF00D859334C0325B5
:108D90000440C02000022043D851C0248020640039
:108DA000800018512E4F18602E4B803CD859FF3C44
:108DB000A043D8510437D859A8432043D851083785
:108DC000D8590C35A8438446072065462843D85116
:108DD000A820C0001E50C1208026800076021E50B0
:108DE0001C601C4B1C60142500202B001E4C2E0008
:108DF00046433659771C1BD14343E250A023032539
:108E0000C132FF329200DB05D550184B1A68082A90
:108E100014D114234343E3189A6812485132FF32A5
:108E2000920059601150DA68C1239B00C250F0BD16
:108E30009642E1D001300328D9D1F8E7082A02D9B7
:108E4000083AD140E5E708239A1A9140E1E7C04685
:108E500024F80000381C002000E100E0FF00FFFFC4
:108E60000405000000900040440000208400002021
:108E70002149F0B54A6C2148002A14D0A025A1262A
:108E800000230124ED05F600C258571C06D0C71870
:108E90007F68002F02D027009740AF5114333C2B3E
:108EA000F2D100234B64A0230121DB0500260F0033
:108EB0009C4614234B43C3181A1F1268104C0E4DC6
:108EC000920014195219526C002A10D01A00143A48
:108ED0001268551C09D0103B1B68FF2B05D03B00C6
:108EE000934065461A00074BEA50FC346664013132
:108EF0000429DED1F0BDC046FC90004044000020B3
:108F0000009000400C05000000B51E2810D80C4A47
:108F10008000835803290BD8A0220800C133FF33F7
:108F2000D2059B0001F000FC020905070021D15089
:108F300000BD0C21FBE70421F9E70321F7E7C04658
:108F400024F800001E280AD8074B8000C2580123CD
:108F50009340A022D205002902D104495350704702
:108F6000A121C900FAE7C04624F800000C05000062
:108F7000030000201E2B0AD8A021A222C905D2007E
:108F80008858034A9B009B58D840012318407047DB
:108F900024F80000F7B506000D000C008B180193B3
:108FA000019B671B9C4207D0336821781B68300007
:108FB000984701340028F3D13800FEBDF0B5C6460D
:108FC00000B5CB0F9846404A4B005B0D9A1882B013
:108FD0000D000400132A2FDC002A49DB3B4F174108
:108FE0003E000E40064323D07F08390029400C4341
:108FF0000AD03749BD438C4663445C425C418023C0
:10900000DB021341E4071D434146CE0031492B00EA
:109010008E192200346875682000290001F000FFD5
:10902000009001910098019922002B0003F090F824
:1090300002B004BC9046F0BD332A08DD8023DB007B
:109040009A42F5D102000B0001F0EAFEF0E7224A55
:109050009446012263445242DA400242E8D0520868
:109060000242D1D094438022D2051A411443CBE767
:109070004B005B080343DBD00B031B0B1C43634219
:10908000234380244D0C24031B0B23406D042B43EE
:1090900019004346DA000F4B9B181C685D680200FC
:1090A0000B002000290001F0BBFE00900191009808
:1090B000019922002B0003F04BF842464B005B085D
:1090C000D60733431900B3E701FCFFFFFFFF0F0092
:1090D000EEFBFFFFD0F80000EDFBFFFFF8B5274ADD
:1090E0004B005B0D9A180C000700132A10DC002AB5
:1090F00036DB234B13410B423AD080242403144126
:10910000002064189C430600250030002900F8BDAB
:10911000332A0EDD80230600DB000D009A42F4D1D5
:1091200002000B003800210001F07AFE06000D005D
:10913000EBE7144D0600AC46012563446D42DD406B
:10914000AC4663460D000342DFD033239A1A323B0C
:1091500093401818874200D94C1C63469843D2E7C5
:10916000C90FCC070020531CCDD1074B1C43CAE7C5
:1091700006000D000028C0D1C7E7C04601FCFFFF74
:10918000FFFF0F00EDFBFFFF0000F03F30B5214A6D
:109190004B0087B05B0893421EDD1F4A934205DDFA
:1091A00002000B0002F0D4FF07B030BD02AA00F0AD
:1091B00095F803231840049A059B012813D0022830
:1091C0001DD0002814D00298039900F06FFB802373
:1091D0001B069C466144E7E700230022009300231E
:1091E00001F0DEF8E0E70298039900F05FFBDBE7AF
:1091F000012402980399009401F0D2F8D4E70124E5
:1092000002980399009401F0CBF880231B069C463A
:109210006144C9E7FB21E93FFFFFEF7FF0B5474617
:10922000CE4680B58DB004000D0000F067FA294BE2
:1092300006001B780F005BB29846013310D0220065
:109240002B002000290003F0CBFA8146002807D12B
:10925000002200232000290001F014FC002806D180
:10926000300039000DB00CBC90469946F0BD01238A
:109270000293194B0694079503934B460A93434672
:1092800004940595002B15D000230022190010002E
:1092900002F0E2F8434608900991022B0ED103F048
:1092A000B9FB212303600A9B0193002B0CD1089E7C
:1092B000099FD5E7002300240893099402A801F030
:1092C000C1F90028EFD1EAE703F0A4FB0A9B019360
:1092D0000360ECE788000020E0F80000F0B54E469F
:1092E0004546DE465746E0B5E14B4C008FB0904610
:1092F000894664089C4200DC87E0DE4B9C4222DC0D
:10930000DD4A002900DC92E0DC4B02F021FFDB4B60
:1093100006000F009C4200D17EE1D94AD94B02F0F1
:1093200017FF02000B00414630000A604B60390015
:1093300002F00EFFD34BD24A02F00AFF434601254A
:109340009860D9606BE0D04B9C4200DC8FE0CF4B43
:109350009C4200DD55E1CE4A231592469A4451467F
:109360000905631A19001D00040003F055FA03F003
:1093700089FA02000B00200029000892099302F0EC
:10938000E7FE0022C34B02F071FC0F00060003F061
:1093900043FA03F077FA04000D0002000B003000DE
:1093A00039000A940B9502F0D3FE0022B94B02F06B
:1093B0005DFC002200230C900D9101F05DFB002864
:1093C00000D192E1002300222000290001F054FB8B
:1093D000434243410133B04A41460192022208A868
:1093E0000092524600F07CFB4B460500002B16DA3B
:1093F000802243461206944642465B6845426344D7
:109400005360D3686344D36009E00B000200414617
:109410000A604B600022002300258A60CB60280090
:109420000FB03CBC90469946A246AB46F0BD934B6C
:1094300001F0F6FC914B06000F009C4200D13DE18B
:109440008F4A904B01F0ECFC02000B0041463000CB
:109450000A604B60390002F07BFE894A894B01F0BB
:10946000DFFC012543466D429860D960D7E701F0E3
:1094700049F88A4A8A4B06000F0002F0F7FB0022E7
:10948000884B01F0CDFC03F0C7F9050003F0FAF9B1
:10949000794A7A4B0490059102F0E8FB02000B0038
:1094A0003000390002F054FE754A06000F0004989F
:1094B0000599744B02F0DAFB029003911F2D00DC3A
:1094C000C7E0029A039B3000390002F041FE834658
:1094D0008A4653465B0024155B0DE31A102B6CDDA6
:1094E00004980599D322674B520502F0BFFB020096
:1094F0000B00300039000292039302F029FE0A00AB
:10950000010013000691079202003900300002F0BA
:109510001FFE029A039B02F01BFE06000F00049838
:109520000599614A614B02F0A1FB32003B0002F059
:109530000FFE069E079F0B000200390030000292CA
:10954000039302F005FE4B005B0D83468A46E41A46
:10955000312C32DD04980599B822544B920502F063
:1095600085FB03000C000200029303940B00069895
:10957000079902F0EDFD02000B0006000F000698AF
:10958000079902F0E5FD029A039B02F0E1FD484ACB
:109590000290039104980599464B02F067FB029AEA
:1095A000039B02F0D5FD02000B003000390002924F
:1095B000039302F0CDFD83468A465A465346414600
:1095C00030000A604B60390002F0C2FD029A039B32
:1095D00002F0BEFD44460B000200A260E3604B4671
:1095E000002B00DB1BE75B46236080231B065344F4
:1095F000636080231B069C466144A060E1606D426D
:109600000DE70B00020002F0A3FD43460025986021
:10961000D9601860596002E7D3221A4B520502F054
:1096200097FD214A214B0D00040002F091FD02003C
:109630000B00414620000A604B60290002F088FDC3
:109640001A4B194A02F084FD434601259860D960FF
:10965000E5E602000B003000390002F079FD6B1ED8
:10966000154A9B009B5883468A46A342A5D130E702
:10967000FB21E93F7BD9024000004054FB21F93F28
:109680003163621A61B4D03DFB213941FFFFEF7FA6
:10969000EAFBFFFF0000704168F9000083C8C96D54
:1096A000305FE43F0000E03F7370032E8A19A33B54
:1096B000C14920259A837B39E8F80000D3220C4B5E
:1096C000520501F0ADFB0B4A0B4B04000D0001F0FD
:1096D000A7FB02000B00414620000A604B602900F6
:1096E00002F036FD034A044BB9E6032373E6C04695
:1096F00061B4D03D7370032E8A19A33BF8B5474679
:10970000CE46674B80B50A000F00190005003940AE
:10971000994200D19BE004000100002F69DD3F1554
:1097200000D1B4E05F4B12039C468023120B5B0315
:1097300013435B00CA0F67449B184A00F80703D520
:10974000D20F5B009B188A0079108C460021802084
:109750001624894680030D189D4202DC29185B1BE4
:109760008144D50F5B00013C5B1952004008002C7E
:10977000F1D100208046802020250027000609E046
:109780008B425CD0D40F5B00013DE31852004008CF
:10979000002D16D0C4198B42F2DD27180E00002CC4
:1097A00049DB5B1AA242894149425B1A121BD40F62
:1097B0005B00013D80443100E31852004008002D59
:1097C000E8D113434ED143465B0837494A468846A1
:1097D000494652104244C90702D5802109060B436D
:1097E00061460F05BD18180029000CBC904699462B
:1097F000F8BD7B005B0803433900002BF5D0002F38
:109800003CD1E30A153A6405002BFAD080204003CE
:1098100003423FD1002700E00F005B00791C0342A8
:10982000FAD0250020208D40401A2900D71B2200A5
:10983000C2401A4376E7FE43F60F8E19B1E7944211
:10984000A0D82718002CF6DB1E000023AEE702008C
:109850003B002800390002F009FA2A003B0001F021
:10986000DFFAC2E74346013303D0434601335B08C6
:10987000ABE7012398460023C144A6E73B00020062
:1098800002F066FC02000B0001F0E6FDADE71300FC
:109890000022BBE70127210020207F42C6E7C04607
:1098A0000000F07F01FCFFFF0000E03FF0B54746FD
:1098B000CE4680B587B000920193754B4F0081462C
:1098C00088467F089F4263DC02F0A6FF002800D193
:1098D000D4E04A4643464846414602F0C7F90400F0
:1098E0000D006C4A6C4B02F0C1F96C4A6C4B01F0F4
:1098F00097FA22002B0002F0B9F96A4A6A4B02F08B
:1099000027FC22002B0002F0B1F9684A684B01F0F5
:1099100087FA22002B0002F0A9F9664A664B02F092
:1099200017FC22002B0002F0A1F9644A644B01F0FD
:1099300077FA22002B0002F099F90290039100229D
:10994000604B2000290002F091F9029A039B060067
:109950000F002000290002F089F9009A019B040001
:109960000D004846414602F081F902000B0020003C
:10997000290002F0EDFB02000B003000390002F07C
:10998000E7FB02000B0000204F4902F0E1FB70E012
:1099900002000B0002F06AF904000D003D4A3E4B44
:1099A00002F064F93D4A3E4B01F03AFA22002B00E6
:1099B00002F05CF93B4A3C4B02F0CAFB22002B0050
:1099C00002F054F9394A3A4B01F02AFA22002B00EE
:1099D00002F04CF9374A384B02F0BAFB22002B0058
:1099E00002F044F9354A364B01F01AFA2B002200F6
:1099F00002F03CF9354B029003919F429FDD344BBE
:109A000000229F423DDC334900207B182E4916007E
:109A10001F0002F09DFB049005910022294B2000BD
:109A2000290002F023F932003B0002F091FB029A78
:109A3000039B06000F002000290002F017F9009A8E
:109A4000019B04000D004846414602F00FF9020058
:109A50000B002000290002F07BFB02000B0030000D
:109A6000390002F075FB02000B000498059902F022
:109A70006FFB07B00CBC90469946F0BD0020124920
:109A8000F7E7154B002604920593144FC5E7C0462F
:109A9000FFFF3F3ED43888BEE9FAA8BDC4B1B4BDCB
:109AA0009EEE213EAD529C804F7E923E9015CB198A
:109AB000A001FA3E7751C1166CC1563F4C55555521
:109AC0005555A53F0000E03F0000F03F3233D33F43
:109AD0000000E93F0000E0FF0000E73F0000D23F48
:109AE000F0B5DE464E4645465746E0B5DC4CA5444B
:109AF0000D9114001900A49A0993DA4B9200D658DC
:109B00004D1E03901821E01E0696029500F0AAFE55
:109B1000C3430100DB1719404B1C9A009B1ADB0062
:109B20001B190B9105934C1B771918D4A59BA50005
:109B30009C463F1922AE6544013707E0286802F0D1
:109B4000A1FE013403C60435BC4208D0002CF5DA6E
:109B500000200021013403C60435BC42F6D1069B27
:109B6000002B01DA00F0FDFB069B03990133DB00BB
:109B70009A46099BDA00944600920022914672AA06
:109B80000492B94A6144934688469AAB63449B4425
:109B9000029B002B00DABCE15D4600260027039CF7
:109BA0004D442A686B6803CC02F060F802000B0099
:109BB0003000390001F034F9083D06000F0044453B
:109BC000EFD1049B4B441E605F6008239C46E14438
:109BD000D145DDD10EA804218446494261448C461A
:109BE000069A93009C44614684460A910399083B77
:109BF00063448C460C93009B009263449B46009AFE
:109C00000498D10003008C46634408911E685F6885
:109C1000002A33DD954980468C466244D30098443F
:109C200070AB9A460EAB99460022914B300039003A
:109C300002F01CF802F0F0FD02F024FE00228D4B31
:109C400004000D0002F012F802000B003000390091
:109C500002F07EFA02F0E0FD4B4601C3994643460E
:109C600020001A685B68290001F0DAF808235B42DB
:109C70009C46E04406000F00D045D5D1059B30003E
:109C80001A003900984600F0DFFCFF2300229B05F4
:109C900004000D0001F0EAFF00F038FC0022764BD2
:109CA00001F0E4FF02000B002000290002F050FA4E
:109CB0000D00040002F0B0FD814602F0E3FD020059
:109CC0000B002000290002F043FA060040460F0076
:109CD000002800DCEEE0009B18215A1E92000EAB1B
:109CE0009B58091A1D000D41A9448D405D1B0EAB08
:109CF0009D5017231B1A1D41002D2DDD01239C466D
:109D0000009BE144002B00DC1CE20E9C0123002C94
:109D100000D0B5E0009A012A09D099000EAA545843
:109D20000133002C00D0ACE0009A9A42F5D1059B9B
:109D3000002B0EDD012B00D1A8E1022B09D1009BE5
:109D40000EA95A1E92000EAB9B5807939B029B0ACA
:109D50008B50022D00D1C1E00023002230003900D9
:109D600000F08AFE009B002800D194E2069A591E5A
:109D70008A4210DC414A0A9894460EAA63449446EB
:109D800000229B0063441C68043B22438342FAD1B7
:109D9000002A00D0C0E0069B0EAA013B9B00D358CE
:109DA000002B00D0B3E001220C9B043B5968013228
:109DB0000029FAD0009B9C466244110007921A00C9
:109DC00001338B4246DC0B9863468046A59C434496
:109DD000A046099C9B00A1464A449844D30022AA6D
:109DE0009146049A99449446089BA59A63448446F4
:109DF000614494469A468B006344009343465868F6
:109E000002F040FD4B4618605960029B002B24DB9A
:109E10004D46039C0026002701E0286869680CCCA9
:109E200001F024FF02000B003000390000F0F8FFC1
:109E3000083D06000F005C45EFD153469E60DF6091
:109E400004239C460433E0449C46009BE144E244E6
:109E50009845D3D1079B0093D1E600260027ECE775
:109E600094FDFFFFB0FA000018FEFFFFFFFFFF1F89
:109E70000000703E0000704100002040FFFFFF3FE7
:109E8000002180225204141B0EAA545000999942BA
:109E90000EDD0EA884469B000EAA8900D2586144AC
:109EA0006344CF4800E01A68821A04C38B42FAD197
:109EB00001243CE7059B002B06D1009B0EAA013B29
:109EC0009B00D558ED1517E70022C64B300000F077
:109ED000F7FD002800D024E100253DE732003B00DB
:109EE0000020C14902F034F906000F00002C00D117
:109EF00032E7059A0020BC4900F0A6FB02000B00E7
:109F00003000390002F024F906000F0024E7012296
:109F100050E70026002754E64B46059A07938846EB
:109F20008B000EA9CB58183A08950592002B0DD13D
:109F30008C464146AD4B43449B006344043B586808
:109F40000139183A0028F9D088460592059A002070
:109F5000A54900F079FB434604000D00002B00DA10
:109F600005E29E000EAB9C464346DB0066449C46E1
:109F7000059370AB9946049F67440097306802F0E0
:109F800081FC22002B0001F071FE00223860796014
:109F9000974B2000290001F069FE083F04000D00E6
:109FA000043EB945EAD14AAB03939B4600239A4647
:109FB000069B4246994643460132029204934B4621
:109FC000002B00DAAAE080208A4B009D9846C0054D
:109FD000894900260027002408E008239C4608350C
:109FE000E044544511DC4346186859682A686B6898
:109FF00001F03CFE02000B003000390000F010FFC1
:10A00000013406000F00A145E7DA5B46C0C39B465A
:10A0100001239C46009BE244083B0093029B9A4527
:10A02000CDD1049B9846A49B022B00DD8EE0002B33
:10A0300037DC1FD1059B00271D00039B00249C4695
:10A040001E006544083E2A686B683800210000F055
:10A05000E7FE083D07000C00AE42F4D1089B002B40
:10A0600003D080231B069C4664443A0023000D99CC
:10A070000A604B600720079B18409B239B009D4470
:10A080003CBC90469946A246AB46F0BD009B0EA94B
:10A090005A1E92000EAB9B5807935B025B0A8B50D3
:10A0A00057E64346002B00DA70E100200021DB0078
:10A0B0004AAAD61848AF32687368083E00F0B0FE6E
:10A0C000B742F8D1089B002B00D025E10B0002001D
:10A0D0004A984B990D9C2260636002F039F8434620
:10A0E00007000C00002B13DD01254CAEB1463800F3
:10A0F0002E0021004C4601360CCC00F091FEA1460A
:10A10000B045F7DA089B07000C00002B00D015E1E2
:10A110003A0023000D998A60CB60ABE70026002748
:10A1200073E701239C46009BE1440225002B00DDE0
:10A13000EBE532003B0000202B4902F009F8060055
:10A140000F0009E60024F2E54AAB0393A49B032B1E
:10A1500000D08FE74346002B00DC14E1039ADB00BC
:10A160009B46130091465B441E685F68234B434443
:10A170000293DB00994448AB9A464B465C681B68E7
:10A180001800210032003B000090019100F048FED1
:10A1900004000D0002000B000098019901F0D8FFA7
:10A1A0003B00320000F03CFE4B469860D9601C60DA
:10A1B0005D6008235B429C46E14426002F00CA45AF
:10A1C000DBD14346012B00DCE3E0039A13005B4440
:10A1D0001E685F68029BDB0099464A44904610E087
:10A1E000FFFFFF000000E03F0000F03FFFFFFF3FE8
:10A1F0000000703E70FA0000FB21F93FFFFFFF1FD7
:10A20000984643465C681B681800210032003B00FA
:10A210000090019100F004FE04000D0002000B000C
:10A220000098019901F094FF32003B0000F0F8FD26
:10A230004346039A9860D9601C605D60083B260025
:10A240002F009A42DCD14D46944600260024474612
:10A25000083565442A686B683000210000F0E0FD95
:10A26000083D06000C00AF42F4D1039B4A9F5D6895
:10A270009968D868089B002B65D080221206944606
:10A280000D9B6544604464441F605D609960D860C4
:10A290001E615C61EEE69A464B460793059B3000D3
:10A2A0005A423900089500F0CFF900223A4B0600D7
:10A2B0000F0000F005FC002824D0384B00223000AD
:10A2C000390001F0D3FC02F0A7FA524604009500D1
:10A2D00002F0D8FA0022304B01F0C8FC02000B005B
:10A2E0003000390001F034FF02F096FA0EAA505106
:10A2F0000122059B524418339046059393000EAA01
:10A30000D45023E65346300039009C0002F084FA12
:10A310000EAB1851D04619E680230D9A1B06CB18B8
:10A32000106053600B0002004A984B9901F010FF37
:10A33000434607000C00002B00DDD5E680231B06FA
:10A340009C466444E4E62B003A000D9D2A606B6055
:10A350000A000300AA60EB60320023002A616B61EF
:10A3600088E6099BDB00009372AB049332E4A49B64
:10A37000022B00DDE8E6002B00DD92E600D079E656
:10A38000002700246AE6002600246EE70020002152
:10A3900098E60026340068E7000070410000703E37
:10A3A000F0B5CE46474680B587B000920193474A44
:10A3B0004B00814688465B08934207DC414648468D
:10A3C00002F02AFA4146031E484666D04A464346F2
:10A3D0004846414601F04AFC04000D0002000B0013
:10A3E0004846414601F042FC394A3A4B06000F000C
:10A3F0002000290001F03AFC374A384B01F0A8FE52
:10A4000022002B0001F032FC354A364B00F008FDEB
:10A4100022002B0001F02AFC334A344B01F098FE55
:10A4200022002B0001F022FC314B324A00F0F8FCF4
:10A430000E9B02900391002B34D0009801990022CA
:10A440002D4B01F013FC029A039B04900591300000
:10A45000390001F00BFC02000B000498059901F093
:10A4600077FE22002B0001F001FC009A019B01F015
:10A470006FFE224A04000D00214B3000390001F02C
:10A48000F5FB02000B002000290000F0C9FC0200CF
:10A490000B004846414601F05BFE07B00CBC9046FD
:10A4A0009946F0BD02000B002000290001F0DEFB00
:10A4B000124A134B01F04CFE32003B0001F0D6FB78
:10A4C0004A46434600F0ACFCE7E7C046FFFF3F3E8C
:10A4D0007CD5CF5A3AD9E53DEB9C2B8AE6E55A3E2E
:10A4E0007DFEB157E31DC73ED561C119A0012A3FCA
:10A4F0001111813FA6F810110000E03F4955555554
:10A500005555C53F49004B0819007047474AF0B5FB
:10A510004F4691464B005B0D99444646D6464A4607
:10A52000C0B505000C000E0088460700132A27DC82
:10A53000002A4BDB3E4B13419A460B005246134018
:10A54000034318D03B4A3C4B2800210000F068FC34
:10A550000022002300F0AAFA002847D0002C04DAD9
:10A5600080234A465B0313419844464653460027DE
:10A570009E43380031001CBC90469946A246F0BD6F
:10A58000332A08DD8023DB009945F4D102000B005B
:10A5900000F046FCEFE7294A944601226344524208
:10A5A000DA4092460242E6D0224A234B280021009C
:10A5B00000F036FC0022002300F078FA002815D0C5
:10A5C000002C1EDB534646469F430FE0194A1A4BA8
:10A5D0002800210000F024FC0022002300F066FA8D
:10A5E000002803D0002C04DB0027002638003100AF
:10A5F000C1E76400640825430027002DF6D0104E03
:10A60000F4E74B46142B0BD03422D21A012393408B
:10A610005D19BD4208D201239C462F00E044D1E7DA
:10A62000133B9C46E044CDE72F00CBE701FCFFFF46
:10A63000FFFF0F009C7500883CE4377EEDFBFFFFB9
:10A640000000F0BF002070474B0070B55B0D140098
:10A650000A00002B1AD14B005B08034315D0234B93
:10A66000002201F003FB224B9C422DDB0A004B0031
:10A670005B0D363B1F4DE318AB422ADC002B0DDD92
:10A680001D4C1B0522401A43110070BD1B4DAB42EF
:10A69000F0D102000B0000F0C3FBF6E71D003535DA
:10A6A00019DA174B02009C4209DD0B0015481649C8
:10A6B00000F032F8134A144B01F0D8FAE5E70B002A
:10A6C0001248134900F028F8104A114B01F0CEFA55
:10A6D000DBE70200E9E7084C363322401B05134351
:10A6E000190000220B4B01F0C1FACEE700005043E5
:10A6F000B03CFFFFFE070000FFFF0F80FF070000D8
:10A7000050C300009C7500883CE4377E59F3F8C2C2
:10A710001F6EA5010000903C30B54A00DB0FDB073F
:10A7200052081A43110030BD02B47146490849006D
:10A73000095C49008E4402BC7047C04603B47146B0
:10A74000490840004900095A49008E4403BC70473B
:10A75000002243088B4274D303098B425FD3030A60
:10A760008B4244D3030B8B4228D3030C8B420DD373
:10A77000FF22090212BA030C8B4202D31212090201
:10A7800065D0030B8B4219D300E0090AC30B8B423F
:10A7900001D3CB03C01A5241830B8B4201D38B03ED
:10A7A000C01A5241430B8B4201D34B03C01A524192
:10A7B000030B8B4201D30B03C01A5241C30A8B42D5
:10A7C00001D3CB02C01A5241830A8B4201D38B02C0
:10A7D000C01A5241430A8B4201D34B02C01A524164
:10A7E000030A8B4201D30B02C01A5241CDD2C309D6
:10A7F0008B4201D3CB01C01A524183098B4201D352
:10A800008B01C01A524143098B4201D34B01C01A3C
:10A81000524103098B4201D30B01C01A5241C308B4
:10A820008B4201D3CB00C01A524183088B4201D323
:10A830008B00C01A524143088B4201D34B00C01A0F
:10A840005241411A00D20146524110467047FFE77B
:10A8500001B5002000F0F0F802BDC0460029F7D095
:10A8600076E7704703460B437FD4002243088B42B0
:10A8700074D303098B425FD3030A8B4244D3030B87
:10A880008B4228D3030C8B420DD3FF22090212BA4C
:10A89000030C8B4202D31212090265D0030B8B42C8
:10A8A00019D300E0090AC30B8B4201D3CB03C01AB2
:10A8B0005241830B8B4201D38B03C01A5241430B8D
:10A8C0008B4201D34B03C01A5241030B8B4201D37D
:10A8D0000B03C01A5241C30A8B4201D3CB02C01AE8
:10A8E0005241830A8B4201D38B02C01A5241430A60
:10A8F0008B4201D34B02C01A5241030A8B4201D34F
:10A900000B02C01A5241CDD2C3098B4201D3CB01F5
:10A91000C01A524183098B4201D38B01C01A5241A4
:10A9200043098B4201D34B01C01A524103098B42A8
:10A9300001D30B01C01A5241C3088B4201D3CB0093
:10A94000C01A524183088B4201D38B00C01A524176
:10A9500043088B4201D34B00C01A5241411A00D226
:10A9600001465241104670475DE0CA0F00D049428F
:10A97000031000D34042534000229C4603098B42FF
:10A980002DD3030A8B4212D3FC22890112BA030A87
:10A990008B420CD3890192118B4208D38901921109
:10A9A0008B4204D389013AD0921100E08909C3098E
:10A9B0008B4201D3CB01C01A524183098B4201D390
:10A9C0008B01C01A524143098B4201D34B01C01A7B
:10A9D000524103098B4201D30B01C01A5241C308F3
:10A9E0008B4201D3CB00C01A524183088B4201D362
:10A9F0008B00C01A5241D9D243088B4201D34B007D
:10AA0000C01A5241411A00D20146634652415B10BE
:10AA1000104601D34042002B00D54942704763469F
:10AA20005B1000D3404201B5002000F005F802BDE4
:10AA30000029F8D016E770477047C046D0400B1C7D
:10AA40001141203A03D49C461341184363465242B5
:10AA5000934018437047C0468446101C62468C469B
:10AA6000191C634600E0C0461FB501F097F80028A6
:10AA700001D40021C8421FBD10B500F0EFFF4042D5
:10AA8000013010BD10B501F089F8002801DB00206D
:10AA900010BD012010BDC04610B501F07FF80028A0
:10AAA00001DD002010BD012010BDC04610B501F031
:10AAB00011F8002801DC002010BD012010BDC046A7
:10AAC00010B501F007F8002801DA002010BD0120C0
:10AAD00010BDC046F0B5CE46474615042D0C2E00DD
:10AAE00080B50704140C3F0C9946030C7E435D436C
:10AAF000674363437F19340CE4199C46A54203D98C
:10AB000080235B029846C4444B4643435143250C83
:10AB100036046544360C2404A4195B195918200026
:10AB20000CBC90469946F0BDF0B54E46574645469A
:10AB3000DE46E0B543025B0A450083B00F1C994630
:10AB40002D0EC60F002D57D0FF2D24D08020DB0006
:10AB5000C0041843002381469A469B467F3D7C02F1
:10AB60007A00FB0F640A120E984623D0FF2A4BD0BE
:10AB7000E30080240020E4047F3A1C43AD186B1CE2
:10AB800047460193534677403A000F2B48D87D49FA
:10AB90009B00CB589F46002B00D085E008339A4697
:10ABA000063B9B467C027A00FB0FFF25640A120ECF
:10ABB0009846DBD1002C00D090E0524601231A4386
:10ABC00092460120DBE74C4658461700022824D065
:10ABD000032800D1CFE00022002301284DD15802E4
:10ABE000D205400AFF071043384303B03CBC9046EF
:10ABF0009946A246AB46F0BD002B5BD104239A4692
:10AC0000033B00259B46AAE7FF35002C60D1524646
:10AC100002231A4392460220B1E7FF220023DEE717
:10AC20004B461B0C9C464B462604360C18046146CA
:10AC30003300220C6446000C43434E4350435443BC
:10AC400080191A0C1218964203D9802149028C46A9
:10AC500064441B041B0C1004C01883015E1EB34126
:10AC6000800E1843130C1B199B0103431C00230186
:10AC700079D5012362081C401443019A7F32002ACF
:10AC80004DDD630704D00F232340042B00D0043490
:10AC9000230103D53C4B019A1C408032FE2ABCDCC8
:10ACA000A3015B0AD2B29AE70C239A46093BFF251F
:10ACB0009B4654E7180001F071FE4A46431F762573
:10ACC0009A4000236D4291462D1A9A469B4646E7CC
:10ACD000524603231A439246032050E7200001F016
:10ACE0005DFE431F2D1A9C40763D002047E78023E0
:10ACF0000027DB03FF2272E7424666E74C4632003C
:10AD0000584662E780234A46DB031A4222D01C429F
:10AD100020D123435B025B0A4746FF225FE7012302
:10AD20009A1A1B2A21DC23000199D3409E318C40C2
:10AD30001A0023005C1EA34113435A0704D00F22BC
:10AD40001A40042A00D004335A0111D49B015B0A33
:10AD5000002244E780234A46DB0313435B025B0A7D
:10AD60003700FF223BE7019587E70022002336E703
:10AD70000122002333E78023DB0323435B025B0ACA
:10AD8000FF222CE7C0FA0000FFFFFFF770B5002894
:10AD90003DD0C317C5185D40C40F280001F0FEFD6B
:10ADA0009E22121A962A07DCD2B2082833DD083810
:10ADB00085406802400A23E0992A0BDD052329001B
:10ADC0001B1AD94003001B339D402B005D1EAB4175
:10ADD00019430D00052801DD431F9D402B000F493D
:10ADE0000B406E0709D00F263540042D05D00433E3
:10ADF0005D0102D59F220B40121A9B01580AD2B264
:10AE00004002D205400AE4071043204370BD0024ED
:10AE100000220020F4E76802400AF1E7FFFFFFFB91
:10AE2000F0B54F464646D6460C000903C0B5490A60
:10AE3000470F5E0039431F03DB0F9C4665007B0A0A
:10AE4000570F1F436D0DE40F760DA146C000B846A5
:10AE5000D200AB1B64457BD0002B5FDD002E00D001
:10AE6000A4E03E00164300D112E15E1E002E00D089
:10AE70009EE1871A4346B84280410125C91A4042E3
:10AE8000091A0B0200D431E149024E0A002E00D10A
:10AE90006EE1300001F082FD0300083B1F2B00DD56
:10AEA00061E120223900D21A9E40D1409F400E43DA
:10AEB0009D4200DD51E15D1B6B1C1F2B00DD7CE121
:10AEC0002021C91A3D0030008F408840DD40791EA6
:10AED0008F41310007222843D940002507433A40DB
:10AEE000002A09D00F233B40042B05D03B1DBB4259
:10AEF000BF417F42C9191F000B0200D426E26A1C21
:10AF0000C64B55056D0D9A4200D106E1C44AFF08B3
:10AF10000A40530752023B43120B8EE0002B00D035
:10AF2000B8E06B1C5B055B0D012B00DC30E1871A80
:10AF30004346B842B641CB1A76429E1B330200D537
:10AF40004CE13B003343A1D100220024002570E0F6
:10AF5000002B00DCE5E0002E00D183E0AF4EB542CF
:10AF600060D0802636043743B846382B00DC3EE1FB
:10AF7000434613431F007A1E97413F188742804182
:10AF8000404209180B0200D4B0E0A44B01359D42A9
:10AF900000D1C3E0A24A7B080A4001210F401F43B1
:10AFA0005108D30707221F433A4099E79B4EB54209
:10AFB00038D0802636043743B846382B00DDDCE035
:10AFC0001F2B00DC30E11E004746203EF740BC4608
:10AFD000202B04D04026F31A46469E4032431700E9
:10AFE00063467A1E97411F43CCE0002B00D104E258
:10AFF0004346134300D159E14B07C008184380234F
:10B00000C9081B03194208D04546ED081D4204D16A
:10B010004346D008590708432900420FC9007F4D15
:10B020001143C0004B07CA087C49C00803438D4246
:10B0300068D012036D05120B6D0D0021120318006C
:10B04000130B0A0D12051A43764B2D0513402B43A3
:10B050005B00E4075B08234319001CBC904699463B
:10B06000A246F0BD3E00164312D05E1E002E00D058
:10B0700000E1871887428041414440420918012578
:10B080000B0233D5022585E76446330041461000A4
:10B090001D00C7E7002D00D0DAE00C000443F3D018
:10B0A0005C1C00D19FE15D4CA64200D12FE1DB4347
:10B0B000382B00DD66E11F2B00DD83E12024050035
:10B0C000E41A0F00DD40D940A0404346A7405B1A78
:10B0D000441EA04198462F433843171ABA42924162
:10B0E00043465242991A64463500CAE607223A405E
:10B0F000002A00D0F6E64B07CA084849FF083B4340
:10B100008D4296D11900114300D19EE1802109039F
:10B110000A431203120B414D8FE715000022002352
:10B120008BE7002B00D0C7E06B1C5F057F0D012F64
:10B1300000DCF1E0394DAB4200D1B9E085180A00DE
:10B14000854289414244494251180722CF076D0880
:10B150002F4349083A401D00C2E607223049ED1A44
:10B1600031403A40BCE63E002838864000279FE642
:10B17000380001F013FC20308EE6434613431F00D5
:10B180007A1E9741C71BB84280414042091A78E6AF
:10B190000E003B0006431343002D61D1002E00D06A
:10B1A000F4E0002B00D11BE164463900100039E7C0
:10B1B0001A4FBB427AD03300FFE630001F3DE84013
:10B1C000202B03D04021CB1A9E4037437B1E9F414A
:10B1D000072207433A400021002589E7171A434612
:10B1E000BA42B641591A76428E1B64464EE61F2B70
:10B1F00000DDADE020264746F61AB740B9461700F5
:10B20000B246DF404E463E4337005646B240561ED9
:10B21000B24117434246DA408918AEE6FF07000004
:10B22000FFFF7FFFFFFF0F8020264746F61AB7403B
:10B23000B9461700B246DF404E463E4337005646F9
:10B24000B240561EB24117434246DA40891A99E786
:10B250007F4CA6425BD0802424045B42214327E735
:10B26000002E0CD1002B00D1CBE064463900100039
:10B27000774DD7E6764FBB4218D0330075E6002BEA
:10B2800014D04B07C00818438023C9081B03194278
:10B2900007D0FC081C4204D17907D0080843E146D6
:10B2A00021004C46420FC9001143C000684DB9E669
:10B2B0001D0000220023C0E6002D5BD10D000543D8
:10B2C00000D1E2E65D1C00D1B0E0614DAE421FD07E
:10B2D000DB43382B71DC1F2B00DD96E020250F00AF
:10B2E000ED1AAF40B9460700AA46DF404D463D4340
:10B2F0002F005546A840D940451EA8418844074321
:10B30000BF18974292415142414435003AE66446A3
:10B3100035004146100085E60B000343002D00D0A8
:10B3200063E6002BF5D04346134300D17AE6871835
:10B330008742804107224144404209183A400B02AB
:10B3400000D4D5E6434B01351940C9E5380069E61C
:10B350001E004746203EF740BC46202B04D0402626
:10B36000F31A46469E403243170063467A1E9741C1
:10B370001F4302E6364DAE42CAD080252D045B4203
:10B380002943A6E70843411E8841A6E6002B00D1C9
:10B3900048E6871A4346B842B641CB1A76429E1B0E
:10B3A00033024BD5171A4346BA429241591A5242B8
:10B3B000891A072264463A4092E501430F00791E3C
:10B3C0008F419DE71C000F00203CE740202B03D05D
:10B3D0004024E31A99400843411E884138437CE6E3
:10B3E0000022002425E6171A4346BA429241591A10
:10B3F0005242891A6446350043E541461000144D17
:10B4000010E680220024120380E61D000F00203D7C
:10B41000EF40BC46202B03D04025EB1A994008434F
:10B4200007006346781E87411F4369E787189742E4
:10B430009B4141445B42C9183500A3E53B003343BF
:10B44000CED0072231003A4052E600231A00F4E53C
:10B45000FF070000FFFF7FFFF0B55746DE464E4670
:10B460004546E0B5834607000E03480085B0924686
:10B470001C00360B400DCD0F002800D19DE0954BF0
:10B48000984239D08023F6001B041E43924A7B0F5A
:10B4900033439946944603006344009300230026F7
:10B4A000FF00029323031B0B98466300E40F5246F0
:10B4B0005B0D019400D1B3E086498B4200D19EE040
:10B4C0004246D100802212040A435146490F1143DB
:10B4D0008B46814952468C4600996344CB1A002121
:10B4E000D20000932B0063409A460F2E00D905E14D
:10B4F0007A4BB6009B599F465B463343994600D032
:10B50000B8E002230826002700900293CAE7CB4642
:10B510003A0002990195019B9A46022927D00329F6
:10B5200000D180E2012944D06D49009B8C466344E0
:10B530001C00002C38DD530700D013E2D2085B4614
:10B54000DB0109D55946674B19408B468021C9005C
:10B550008C46009B63441C00634B9C4207DC5B46AB
:10B5600064055F075B0217431B0B620D02E00023BB
:10B570000027584A00211B031C0B0B0D1B052343FE
:10B5800014055A4A380013401C4353466400DB0735
:10B5900064081C43210005B03CBC90469946A24675
:10B5A000AB46F0BD0122524201231B1B382B00DCAD
:10B5B000ADE1002200230027DCE75B4633439946D8
:10B5C0005ED0002E00D18AE1300001F0E7F90300DF
:10B5D0000B3B1C2B00DD7BE11D22D31A5A460100D8
:10B5E000DA4008398E4013005F46334399468F4056
:10B5F0003F4B00261B1A00930023029352E741465B
:10B6000053460B433B499B468C46009B6344009347
:10B610005B46002B3BD1022300221E43022161E73F
:10B62000434613439B4637D04346002B00D162E18B
:10B63000404601F0B3F903000B3B1C2B00DD53E146
:10B6400002004146083A914088461D21CB1A5146D6
:10B65000D9400B0041460B439B46534693401A008A
:10B66000009B25499C46604403008C46634400933C
:10B67000002137E70323B14600900C26029311E71F
:10B680000023009301330426002702930AE70323D3
:10B69000C3461E43032125E701331E430022012137
:10B6A00020E700239A46802300271B03094A61E70D
:10B6B000802349461B03194200D1E2E05946194252
:10B6C00000D0DEE00B431B0317001B0BA246014A10
:10B6D00050E7C046FF07000001FCFFFF00FB000031
:10B6E000FF030000FFFFFFFEFE070000FFFF0F80CB
:10B6F0000DFCFFFF01F8FFFFF3030000D94500D95F
:10B70000CBE000D1C6E03C0048460027009B013B4F
:10B7100000935B46160E1B021E4313029846330429
:10B720001B0C9946310C0191FFF798F84A464243A9
:10B730000B04210C050019438A4207D98919013DE0
:10B740008E4203D88A4201D9851E8919881A019927
:10B75000FFF784F809048C464A46210464464243B4
:10B76000090C030021438A4204D98919013B8E4206
:10B7700000D8F1E02D041D43AB464346891A4246EA
:10B78000280C12041D0C5B46140C22001B041B0C1D
:10B790005A4303946B434443029568431B19150CA9
:10B7A000EB189C4203D980246402A44660441C0C1C
:10B7B00015041B042D0C20185D19814277D373D01A
:10B7C0000C1AA24A7D1BAF42BF419446009B7F42A8
:10B7D0006344E01B1C00864200D1DBE00199FFF7C7
:10B7E0003DF84A4642430B04290C070019438A429C
:10B7F00007D98919013F8E4203D88A4201D9871E91
:10B800008919881A0199FFF729F809044A468946D7
:10B8100029044D464243090C030029438A4207D9B3
:10B820008919013B8E4203D88A4201D9831E8919A6
:10B830003F04891A3A00039F1A43380013041B0C73
:10B84000584381460298150C6F434343454348468D
:10B85000000C8446DB1963449F4203D980204002D8
:10B860008446654448461F0C00041B04000C7D19E7
:10B870001818A94200D284E000D17FE001231A43C6
:10B8800057E680234A461B0313431B031B0BAA46A0
:10B890006F4A6FE6BA4200D935E74B46DC075808D5
:10B8A0007B081C43FF0734E70024AF4289D247449A
:10B8B0004745A4415B466442A4196418013BA64273
:10B8C0001ED2A0426DD800D1B6E0241A9B4678E77C
:10B8D00003005A46283B9A400027914688E658467E
:10B8E00001F05CF8203072E603005246283B9A4093
:10B8F00093460022B4E6504601F050F820309AE614
:10B90000A642E2D1B845DCD9341A9B4659E71F2B31
:10B9100065DC504C0099A4465C46614408008C40AC
:10B9200011008240D940501E82410C4314435A46B4
:10B93000DA401300620709D00F222240042A05D002
:10B940002200141D9442894149425B181A0262D5B3
:10B950000122002300270DE68A4200D80AE7831E51
:10B96000891907E70F231340042B00D1E6E5171DC3
:10B970009742924153429B44FA08E0E5002800D1E7
:10B98000D7E57118531EB14227D3A94215D358D019
:10B990001A0073E7002B00DC04E6012300229B441D
:10B9A000CDE502234744474589415B429C464942D5
:10B9B00089190C19E344241A03E743465F004745FD
:10B9C0009B41B8465B429E19023A8919A94200D0B0
:10B9D00054E7404500D051E7ABE51A00F6E71F21D8
:10B9E0005F4649420C1BE740202B07D01A49009BB9
:10B9F0008C46634418005B4683401A43501E8241C4
:10BA00003A4307270023174009D00F210023114094
:10BA10001400042995D122005F075B021B0BD2089A
:10BA200017430022A6E5802359461B030B431B0343
:10BA300017001B0B064A9DE5BD42B2D89B46002469
:10BA4000BFE68045B9D31A00C3E7C046FF03000034
:10BA5000FF0700001E0400003E040000F0B54F4642
:10BA60004646D6468446C0B58046194E18030F0395
:10BA70004D00000B5C0082463F0B6D0DC90F9146D7
:10BA8000640DDB0F0120B5420AD0B44203D0A542B9
:10BA900001D157450CD01CBC90469946A246F0BD3A
:10BAA00066463E43F7D1AC42F5D154461443F2D139
:10BAB0000120C845EFD1994207D0002DEBD1634654
:10BAC0001F433800471EB841E5E70020E3E7C046C2
:10BAD000FF070000F0B54F464646D6464D00C0B5BC
:10BAE0000E03C90F8A462C491F035C008046360BA3
:10BAF0006D0D91463F0B640DDB0F8D421ED08C42C5
:10BB000016D0002D1ED130438446002C01D13A437B
:10BB100023D06246002A1AD09A4529D051460220E5
:10BB20000139084001381CBC90469946A246F0BD38
:10BB300039001143E5D002204042F4E73043FAD106
:10BB4000AC420FD0002C0FD13A43E7D00CE00122D9
:10BB5000013B934318000130E5E763460020002BCA
:10BB6000E1D0DBE73A43E6D19A45D7D1A542D5DC0F
:10BB7000A54205DBBE42D1D808D00020BE42D2D2B9
:10BB800050460123013898430130CCE7C845C5D859
:10BB90000020C845F4D3C6E7FF070000F0B54F46C4
:10BBA0004646D6464D00C0B50E03C90F8A462E49FB
:10BBB0001F035C008046360B6D0D91463F0B640DF4
:10BBC000DB0F8D4218D08C4211D0002D18D130439C
:10BBD0008446002C1ED13A431CD163460020002B22
:10BBE00030D0514602200139084001382AE039009E
:10BBF0001143EAD0022025E03043FBD1AC4226D0ED
:10BC0000002C26D13A4324D1514602200139084064
:10BC1000013817E06246002A0FD09A45E1D1A542CB
:10BC200005DBBE42DDD819D00020BE420AD2504604
:10BC3000012301389843013004E00122013B934382
:10BC4000180001301CBC90469946A246F0BD3A430C
:10BC5000D0D19A45C5D1A542C3DCE0E7C845C0D8DC
:10BC60000020C845E3D3EDE7FF070000F0B55746D5
:10BC7000DE464E464546E0B5834606000F034800C3
:10BC800087B092461D003F0B400DCC0F002800D11D
:10BC90006FE0DE4B984238D08023FF001B041F4327
:10BCA000730F3B430193DA4B0027994600239B46D1
:10BCB000F60081442B0369001B0B52469846490D40
:10BCC000ED0F002900D185E0D04B994200D173E0FF
:10BCD0004346DA0080231B0413435246CC48520FDC
:10BCE00084461343524600206144D2008944210017
:10BCF000694000918C46012149448A460F2F00D9A2
:10BD000090E0C449BF00CF59BF465B463B43019317
:10BD100000D06AE102230827002681469B46C9E736
:10BD200032005846019B61460091022800D175E01F
:10BD3000032800D1FEE1012800D02CE100230027D8
:10BD4000002600253F032A0D3F0BB34812053A4356
:10BD500002401B051343009A5B00D1075B080B43AD
:10BD60003000190007B03CBC90469946A246AB464D
:10BD7000F0BD5B463B43019300D12FE1002F00D182
:10BD8000A5E1380000F00AFE03000B3B1C2B00DD90
:10BD900096E11D22D31A5A460100DA405E46083960
:10BDA0008F4013008E403B4301939C4B00271B1A8E
:10BDB000994600239B467DE7414653460B439349F2
:10BDC0008C46E144002B00D01AE1022202201743E6
:10BDD00000228CE7134300D10DE14346002B00D134
:10BDE00081E1404600F0DAFD02000B3A1C2A00DD3A
:10BDF00072E10100434608398B4098461D239A1A88
:10BE00005346D3401A004346134352468A4049469C
:10BE1000081A824989468144002068E77B4B002745
:10BE200000268EE7140C1204120C1100370C360495
:10BE3000350C794328008C462E00604360448346CD
:10BE400056432100300C80465846794340440291C5
:10BE5000844506D98846802149028C46E044414603
:10BE600002913604010C360C00048B4681191E0C1D
:10BE70001B041B0C0391190079438C462800754361
:10BE80006544A8465843050C45447743A94203D965
:10BE9000802149028C466744290C8C4639000004F5
:10BEA000000C2D042D186144AB44059159460491B2
:10BEB00001990F043F0C080C39005143424390464E
:10BEC00002008C46090C8B4662437C4344445C442C
:10BED000A04503D98021490288464244210C884666
:10BEE00061460904090C8C463900594343437043A9
:10BEF0007E430F0CF6182404BE19644442448C4659
:10BF0000B34203D980235B0298464044029B6146BA
:10BF10009846049B370443449B46AB45AD416B4276
:10BF20000D0405992D0C8C467F196744FD18A84611
:10BF30005D462D19A542A44193466442A446C344DC
:10BF4000DC448F42BF4198459B4193459241A445B3
:10BF5000A4415B427F421F43360C52426442BF19E8
:10BF60002243BF18624638184302D20D0399134387
:10BF70006A020A43501E82416146ED0D2A434E0279
:10BF80003243D90100D4B3E00126500832400243C5
:10BF9000DE0732435B08224C5444002C62DD51071B
:10BFA00009D00F201040042805D0101D9042924166
:10BFB00052429B180200D90104D580241948E4009C
:10BFC000034054441848844200DD27E75E075B02C3
:10BFD000D2081F0B630516435B0DB2E6002399469A
:10BFE0000133042700269B4664E60323019781461C
:10BFF0000C279B465EE6012201201743002276E6CD
:10C00000032303201F43434671E6C046FF07000099
:10C0100001FCFFFF40FB0000FFFF0F800DFCFFFF56
:10C02000FF030000FFFFFFFEFE0700000023802744
:10C0300000933F030026434B83E6019B3200A44656
:10C04000584670E6AC466EE6802701993F033942B8
:10C050002DD03B422BD11F433F033F0B00951600D1
:10C06000384B6EE601252D1B382D00DD66E61F2DB1
:10C0700040DC35481C005044160082408440EE40AD
:10C08000501E824134431443EB40620709D00F2213
:10C090002240042A05D02200141D944280414042CF
:10C0A0001B181A023ED501230027002649E68027E7
:10C0B000019B3F031F433F033F0B0094214B40E68E
:10C0C00003005A46283B9A40002601926DE65846E6
:10C0D00000F064FC203057E603005246283B9A40AB
:10C0E0001300002293E6504600F058FC20307BE617
:10C0F000CA4650E71F201E004042041BE640202D88
:10C1000003D0124C5444A3401A43501E8241324380
:10C1100007260027164009D00F20002310401400E6
:10C120000428B9D122005E075B021F0BD208164318
:10C13000002306E680273F031F433F033F0B160003
:10C14000004BFEE5FF0700001E0400003E04000057
:10C15000F8B557464E464546DE460C000903E0B5A5
:10C16000490A460F5F0031431E03DB0F760A9B46E8
:10C17000530F3343C84E6500C000E40FD2006D0D6D
:10C18000A24681467F0D9C469046B74200D1B9E059
:10C190005B46012673409B46EE1BA34500D183E01E
:10C1A000002E63DD002F00D0B1E06346134300D1C1
:10C1B00023E1731E002B00D0BAE1861A6346B04219
:10C1C00080410125C91A4042091A0B0200D447E1F7
:10C1D00049024B0A98464346002B00D189E140466C
:10C1E00000F0DCFB0300083B1F2B00DD7CE120227C
:10C1F0003000D21A4146D040994002009E400A4386
:10C200009D4200DD6AE15D1B6B1C1F2B00DD94E18C
:10C21000202110003500C91A8E40DA408840DD40E8
:10C22000711E8E411100072228430025064332402B
:10C23000002A09D00F233340042B05D0331DB3420D
:10C24000B641764289191E000B0200D43DE26A1CF9
:10C25000914B55056D0D9A4200D119E18F4AF608B0
:10C260000A40570752023743120B9BE0002E00D0C2
:10C27000C5E06E1C7605760D012E00DC48E16746B0
:10C28000861ACB1BB042BF417F42B8461F004346CF
:10C29000FF1A3B00B8461B0200D55FE137439AD135
:10C2A00000220024002579E0002E00DCFAE0002FB7
:10C2B00000D18DE0784B9D4267D0802367461B04F8
:10C2C0001F43BC46382E00DC52E1634613435A1E1E
:10C2D00093411E1886428041404209180B0200D447
:10C2E000BEE06D4B01359D4200D1D2E06B4A730830
:10C2F0000A4001210E401E435108D30707221E4366
:10C30000324095E71E00164300D045E740E7624BF8
:10C310009D423AD0802367461B041F43BC46382EFB
:10C3200000DDEBE01F2E00DC3AE133006746203BE6
:10C33000DF403B00202E05D04027BF1B6646BE4095
:10C34000324390464646721E96413343DAE0002B54
:10C3500000D114E26346134300D168E180234E0705
:10C36000C008C9081B030643194208D06046C0082C
:10C37000184204D163460100D2085E071643F30059
:10C380009946C900720F444D11434B46DE08424B9B
:10C390004F073743CA089D4200D16EE012036D0576
:10C3A000120B6D0D00211203130B0A0D12051A4317
:10C3B0003B4B2D0513402B435B00E4075B082343F5
:10C3C000380019003CBC90469946A246AB46F8BDE1
:10C3D0006346134311D0731E002B00D007E186186B
:10C3E0008642804161444042091801250B0237D53D
:10C3F00002257BE73E00614691463500C5E75C4675
:10C40000002D00D0E1E00B000343F3D0731C00D1FA
:10C41000ACE1214B9F4200D13AE1F343382B00DDE0
:10C420006FE11F2B00DD8CE120250E00ED1AAE40E0
:10C43000B0460600AA46DE40454635432E00554626
:10C44000D940A8406346451EA8415B1A9C4630432C
:10C45000161AB242924163465242991A3D00B4E61E
:10C4600007223240002A00D0E4E60B4BF6084F07C3
:10C470003743CA089D4200D090E73B00134300D1E8
:10C48000A6E180231B031A431203120B024D89E716
:10C4900015000022002785E7FF070000FFFF7FFF50
:10C4A000FFFF0F80002E00D0C7E06B1C5E05760DED
:10C4B000012E00DCF0E0C84DAB4200D1B9E0851898
:10C4C0000A00854289416244494251180722CE0739
:10C4D0006D082E43490832401D00A9E6BF49ED1AF8
:10C4E000114007223240A3E632002838824000265D
:10C4F00086E6300000F052FA203073E663461343BC
:10C500005A1E9341C61AB04280414042091A5CE665
:10C510000E00674606431743002D5ED1002E00D063
:10C52000F3E0002F00D11EE15C46614691462CE706
:10C53000A94FBE427BD01E00F1E610001F3DE8402F
:10C54000202B03D04021CB1A9A401643731E9E41E4
:10C550000722064332400021002583E7161A63466E
:10C56000B2428041591A40420B1A98465C4632E664
:10C570001F2E00DDABE02027BB1B9A4663465746C3
:10C58000BB40994613004F46F3401F433B005746BC
:10C59000BA40571EBA4113436246F240891898E6E2
:10C5A0002027BB1B9A4663465746BB40994613005B
:10C5B0004F46F3401F433B005746BA40571EBA410F
:10C5C00013436246F240891A9CE7834B9F425FD037
:10C5D00080252D047342294320E7002E0CD1002F23
:10C5E00000D1D0E05C46614691467B4DCDE67A4F66
:10C5F000BE421CD01E0065E6002F18D0C0084E07B2
:10C6000006438020C9080003014208D06346DC08C5
:10C61000044204D12100DA46D2085E071643F30033
:10C62000994601245346C900720F11431C406A4DBC
:10C63000ABE61D0000220027B4E6002D59D10B0007
:10C64000034300D1D6E6731C00D1B2E0624B9F4297
:10C650001ED0F343382B6FDC1F2B00DD97E0202525
:10C660000E00ED1AAE40B0460600AA46DE40454632
:10C6700035432E005546A840D940451EA8418C445C
:10C680000643B61896429241514261443D0025E668
:10C690003D006146914678E60B000343002D00D033
:10C6A00055E6002BF5D06346134300D16DE686189E
:10C6B0008642804161444042091800220B0200D4A6
:10C6C000D0E6464B01351940B2E5B1465DE6330090
:10C6D0006746203BDF403B00202E05D04027BF1B94
:10C6E0006646BE40324390464646721E96413343EC
:10C6F000EFE5394B9F42CBD080252D04734229436F
:10C70000A8E70843411E8841A2E6002F00D13CE67D
:10C710006346861ACF1AB0429B415B42FB1A984689
:10C720001B024ED5161A6346B2429241591A524222
:10C73000891A5C4600227BE501430E00711E8E4182
:10C740009FE71D000E00203DEE40B046202B04D098
:10C750004025EB1A99400843814648464346411E0E
:10C760008841184374E60022002417E6161A63462F
:10C77000B2429241591A5242891A3D0025E561465A
:10C780009146154D01E680220024120379E61D0032
:10C790000E00203DEE40B046202B04D04025EB1A81
:10C7A0009940084381464E464346711E8E411E43C2
:10C7B00067E7861896429B4161445B42C9183D0079
:10C7C0008CE547463743CED007224146324049E602
:10C7D00000273A00E6E5C046FF070000FFFF7FFFA5
:10C7E00070B50C4E0D031C0349005B002D0B490D69
:10C7F000240B5B0DB14208D0064900208B4203D1C7
:10C8000014432000441EA04170BD05430120002DAB
:10C81000FAD1F1E7FF07000030B5144D0A034B00D1
:10C82000120B5B0DC90F0024AB4211DD104CA3426B
:10C8300010DC8024640322430E4CE41A1F2C0CDD10
:10C840000D48C31ADA4013005C42002900D11C00D5
:10C85000200030BD094BCC18FAE7094DE040AC464A
:10C8600063449A4013000343EEE7C046FE03000012
:10C870001D0400003304000013040000FFFFFF7FCD
:10C88000EDFBFFFF70B500282DD0C317C5185D4024
:10C89000C40F280000F082F8154B1B1A5B055B0DD6
:10C8A0000A2815DD0B38854000222D032D0B0021B1
:10C8B00010002D030A0D2D0B12052A430D4D1B05EB
:10C8C0002A4013435B00E4075B082343190070BD53
:10C8D00002002900153291400A000B21081AC540B8
:10C8E0002D032D0BE3E70024002300250022DEE7C3
:10C8F0001E040000FFFF0F804100090E4B1C70B5A5
:10C90000DBB24602750AC40F012B14DDE0239B0045
:10C910006D07360BCB1800210A0D280012051C4D9F
:10C9200032435B052A405B0813435B00E4075B0866
:10C930002343190070BD002914D1002D1ED02800FA
:10C9400000F02CF80A281CDC0B232A001B1ADA4002
:10C95000030015339D400F4B12031B1A5B05160B8A
:10C960005B0DD8E7002D06D0320B802636036D070D
:10C970001643094BCFE7084B0026CCE700230026DF
:10C98000C9E703002A000B3B9A400025E3E7C046B5
:10C99000FFFF0F8089030000FF0700001C21012317
:10C9A0001B04984201D3000C10391B0A984201D392
:10C9B000000A08391B09984201D30009043902A270
:10C9C000105C40187047C0460403020201010101D7
:10C9D000000000000000000030B51C00094B0500FD
:10C9E0001B6885B0D868084B002A01D1074B1A0094
:10C9F0000292019300912B002200054900F026F8D5
:10CA000000F0A6FD8C00002080FB0000F3E6000093
:10CA10008DFB0000014B18687047C0468C00002059
:10CA2000084B10B50400002B02D0002100E000BF2D
:10CA3000054B1868836A002B00D09847200001F04E
:10CA40005DFBC04600000000BCFB00000EB403B557
:10CA5000010003AB044804CB0068019300F076F8B2
:10CA600002B008BC03B018478C00002070B5002647
:10CA70000C4D0D4C641BA410A64209D1002601F0F8
:10CA80003FFB0A4D0A4C641BA410A64205D170BDA1
:10CA9000B300EB5898470136EEE7B300EB589847E0
:10CAA0000136F2E75C0200205C0200205C020020FC
:10CAB0006C020020002310B59A4200D110BDCC5C5E
:10CAC000C4540133F8E710B5884202D98B18984254
:10CAD00003D3002307E08B5C8354013AFBD210BDE3
:10CAE000CC5CC45401339A42FAD1F8E7030012181F
:10CAF000934200D1704719700133F9E7936810B57C
:10CB0000013B9360002B04DA9469A34207DB0A29F6
:10CB100005D01368581C10601970080010BD00F093
:10CB20004BFC0100F9E7F8B506000F001400D5181A
:10CB3000AC4201D1002007E021783A003000FFF735
:10CB4000DDFF0134431CF3D1F8BD0000F0B59FB008
:10CB500002900F0016000593002805D08369049306
:10CB6000002B01D100F0F4FD7B4B9F425BD1029B77
:10CB70005F68BB891B0762D53B69002B5FD0002330
:10CB800006AC6361203363761033A37635002B78CF
:10CB9000002B01D0252B5CD1AB1B04930CD03200B1
:10CBA00039000298FFF7BFFF431C00D1C4E062695F
:10CBB000049B9446634463612B78002B00D1BBE057
:10CBC000012200235242626002A9543252186E1CA4
:10CBD0002360E360A3601370A365317805225F488A
:10CBE00000F0D4FE751C002835D12268D30604D588
:10CBF000532302A95B1820211970130704D553236E
:10CC000002A95B182B21197033782A2B2CD0350000
:10CC100000210A20E3682A786E1C303A092A64D978
:10CC200000292ED026E04E4B9F4202D1029B9F68E6
:10CC30009FE74C4B9F429CD1029BDF6899E73900EC
:10CC4000029800F00FFC002899D0012040421FB04C
:10CC5000F0BD01359BE7414B2268C01A0123834098
:10CC6000134323602E00B8E7059B191D1B6805912F
:10CC7000002B01DB099304E05B42E36002231343D2
:10CC800023602B782E2B0AD16B782A2B35D1059B6C
:10CC900002351A1D1B680592002B2BDB0793324EC1
:10CCA00029780322300000F071FE002806D04023CE
:10CCB000801B8340226801351343236029780622B4
:10CCC0002A486E1C217600F061FE00283AD0284BDD
:10CCD000002B25D10722059B073393430833059387
:10CCE0006369039A9B18636150E7434301219B18D2
:10CCF000350090E701235B42D0E700230A201A00A9
:10CD00000135636029786E1C3039092903D9002B5D
:10CD1000C5D00792C3E74243012352183500F1E71B
:10CD200005AB00933A00134B2100029800E000BFCE
:10CD30000390039B0133D3D1BB895B0600D584E705
:10CD40000B9884E705AB00933A000A4B2100029848
:10CD500000F080F8ECE7C04614FC0000C0FB0000C7
:10CD600034FC0000F4FB0000C6FB0000CAFB00001E
:10CD70000000000027CB0000F7B5150001938A687A
:10CD80000B6900900C00934200DA130022002B6024
:10CD900043321278002A01D001332B6023689B06AE
:10CDA00002D52B6802332B60062723681F4027D04B
:10CDB000230043331B785A1E93412268920630D4D5
:10CDC0002200019943320098089EB047431C25D0A9
:10CDD000062320682A68E16803400025042B03D15C
:10CDE0008D1AEB43DB171D40A3682269934201DDD6
:10CDF0009B1AED180027BD4220D1002010E001371A
:10CE0000E3682A689B1ABB42D2DD22000123193253
:10CE100001990098089EB047431CF0D10120404280
:10CE2000FEBD3020E1184331087021005A1C453105
:10CE30000978A218433202331170C1E7220001239E
:10CE40001A3201990098089EB047431CE6D001377A
:10CE5000D1E70000F0B589B004920A00433205938F
:10CE6000039002920A7E0C000E9B6E2A00D186E08F
:10CE70001FD8632A33D008D8002A00D18CE0582A62
:10CE80004DD0250042352A7030E0642A01D0692A4D
:10CE9000F7D1196825680A1D280629D508681A607F
:10CEA000002803DA2D23029A404213706B4E0A27A2
:10CEB0004FE0732A74D008D86F2A1FD0702AE0D1AF
:10CEC000202209680A43226003E0752A16D0782AD6
:10CED000D7D12200782145321170614E22E0250021
:10CEE0001A684235111D196013682B70012365E023
:10CEF00008681A606906D3D500B2D1E719682568B9
:10CF0000081D186008682E0605D5544E08276F2A9C
:10CF10001BD00A2719E06D06F7D580B2F5E7453139
:10CF20004E4E0A7018682268011D006819601506C7
:10CF300021D5D30702D520231A43226010270028C9
:10CF400003D1202322689A43226023000022433326
:10CF50001A706368A360002B58DB04222168914398
:10CF60002160002854D1029D002B5AD0250033782F
:10CF700042352B7055E05506DBD580B2D9E71A68EB
:10CF80000D68101D4969186013682E0601D51960D7
:10CF900002E06D06FBD519800023029D23614FE05E
:10CFA0001A68111D1960156800216268280000F0D8
:10CFB000EDFC002801D0401B606063682361002302
:10CFC000029A13703CE023692A0004990398059D96
:10CFD000A847431C3ED023689B0715D4079BE068F5
:10CFE000984239DA180037E02200012319320499F7
:10CFF0000398059EB047431C2CD00135E368079A7F
:10D000009B1AAB42F0DCE9E70025F7E70028ADD03A
:10D01000029D3900FDF722FC735C013D2B70002856
:10D02000F7D1082F09D12368DB0706D56368226989
:10D03000934202DC3023013D2B70029B5B1B23617A
:10D04000059B07AA00932100049B0398FFF794FE19
:10D05000431CB8D10120404209B0F0BDD1FB000013
:10D06000E2FB00000D4B70B51C680500A36B002BA4
:10D070000FD1182000F06EFC094BA0630360094B30
:10D0800001224360084B83600B23838100230261EC
:10D0900043610022A36B1D615A6170BD8C000020AA
:10D0A0000E33CDAB34126DE6ECDE0500124B10B53D
:10D0B0001C68A36B002B0FD1182000F04BFC0F4B0A
:10D0C000A06303600E4B012243600E4B83600B2371
:10D0D0008381002302614361A46B0B4A206961696B
:10D0E0000A4BFDF7F7FC012200238018594120610B
:10D0F00061614800400810BD8C0000200E33CDABAC
:10D1000034126DE6ECDE05002D7F954C2DF4515860
:10D110000CB430B5164B9DB00C1E1D6808DA8B237D
:10D1200001202B6040421DB030BC08BC02B0184743
:10D13000822302A99B008B810023029008619C42FC
:10D1400000D0631E8B604B6101235B42CB81209A30
:10D1500021AB2800019300F055FD431C01DA8B231D
:10D160002B60002CDFD00023029A1370DBE7C0464F
:10D170008C0000200EB400B50B499CB01DAB029092
:10D180000690079104910948094904CB059100686C
:10D1900002A9019300F036FD0023029A13701CB01F
:10D1A00008BC03B01847C046FFFFFF7F8C0000207B
:10D1B0000802FFFF020010B51378541C002B05D1A4
:10D1C000CC5CD4540133002CFAD110BD2200F3E71B
:10D1D000C9B20378002B04D08B4200D170470130D4
:10D1E000F7E74B42594149420840F7E702780B788C
:10D1F000002A03D0013001319A42F7D0D01A70478B
:10D200000023C25C0133002AFBD1581E7047002363
:10D2100030B59A420AD0013AC45CCD5CAC4204D12C
:10D22000934202D00133002CF6D1631B180030BDAD
:10D2300030B50500002A00D130BD0C78013A6B1CD6
:10D240002C700131002C05D19A189A42F4D01C7030
:10D250000133FAE71D00EDE710B50378002B0FD17D
:10D260000B785A4253415B42184010BD0023CA5C00
:10D27000002AFAD0C45C944201D10133F7E70130AF
:10D280000378002BF2D11800EFE70000F0B51F0083
:10D290000E0087B00590019102920C98347800F04E
:10D2A000EAFA082200194378751C134036D12D2C58
:10D2B00036D1B51C74780126002F62D0102F09D109
:10D2C000302C07D120222B789343582B54D1102790
:10D2D0006C7802352D4B3900F31818000393FDF7D5
:10D2E000BDFA049101210023494202008C46180036
:10D2F0002100303909291AD80C00A74223DD591C16
:10D3000009D06346824206D302D10499A14202DBCE
:10D310000123784320182C780135E9E72E00BCE77B
:10D320002B2C01D01E00C7E7B51C7478FAE721004A
:10D330004139192901D8373CDFE721006139192922
:10D3400001D8573CD9E75A1C08D1059A23331360FA
:10D35000029B0398002B09D107B0F0BD002E00D02E
:10D360004042029A002AF7D0002B01D06B1E019395
:10D37000029B019A1A60EFE73024002FAAD10827F8
:10D38000A8E7302C9ED00A27A4E7C046FFFFFF7F06
:10D3900037B51300064A05001068046A002C00D156
:10D3A000044C0A0000942900FFF770FF3EBDC04600
:10D3B0008C000020F0000020F8B505000E001400DD
:10D3C000002804D08369002B01D100F0C1F9224B61
:10D3D0009C422DD16C68A369A360A3891B0731D53A
:10D3E0002369002B2ED023682269F7B2981A63694B
:10D3F000F6B2834205DC2100280000F03BF900284A
:10D4000026D1A3680130013BA36023685A1C226027
:10D410001F706369834204D0A389DB071AD50A2EE3
:10D4200018D12100280000F025F9002812D00FE0C3
:10D430000A4B9C4201D1AC68CDE7094B9C42CAD152
:10D44000EC68C8E72100280000F00CF80028CAD0DA
:10D45000012676423000F8BD14FC000034FC0000C8
:10D46000F4FB0000364B70B51D6806000C00002D63
:10D4700005D0AB69002B02D1280000F069F9314BCF
:10D480009C420FD16C680C23E25E93B219072DD435
:10D49000D90611D409230120336037331343A38104
:10D4A000404270BD284B9C4201D1AC68EBE7274B52
:10D4B0009C42E8D1EC68E6E75B0713D5616B002975
:10D4C00008D023004433994202D0300000F06AFAB9
:10D4D000002363632422A3899343A3810023636011
:10D4E000236923600823A2891343A3812369002BA6
:10D4F0000BD1A0218022A389890092000B40934286
:10D5000003D02100300000F0E1F90123A28913408B
:10D5100011D00023A36063695B42A36100202369EB
:10D520008342BED10C23E25E1306BAD540231343D7
:10D53000A3810138B5E7920700D46369A360EDE7E2
:10D540008C00002014FC000034FC0000F4FB000000
:10D5500010B5062000F090FC012000F0CFFD000087
:10D56000F7B58A8905000C00130760D44B68002BBF
:10D5700004DC0B6C002B01DC0020FEBDE76A002FF1
:10D58000FAD000232E682B6080235B01216A1A40A9
:10D5900034D0606DA3895B0706D56368C01A636BDE
:10D5A000002B01D0236CC01A0200216A002328003E
:10D5B000E76AB847A189431C06D12B681D2B30D8D8
:10D5C0002B4ADA40D3072CD50023636023692360FC
:10D5D000CB0405D5431C02D12B68002B00D160651C
:10D5E000616B2E600029C7D023004433994202D0DA
:10D5F000280000F0D7F900206063BEE7012328006F
:10D60000B847431CC6D12B68002BC3D01D2B01D0BB
:10D61000162B01D12E60AFE74023A2891343A381CB
:10D62000ABE740230B430120A3814042A5E70F69EC
:10D63000002FA1D00B680F60DB1B01930023920722
:10D6400000D14B69A360019B002B00DC94E7019B98
:10D650003A00216A2800A66AB047002803DC40236C
:10D66000A2891343DFE7019B3F181B1A0193EAE7E6
:10D67000010040200B6970B505000C00002B01D1A2
:10D68000002070BD002804D08369002B01D100F078
:10D690005FF80B4B9C4209D16C680C22A35E002BF7
:10D6A000EED021002800FFF75BFFEAE7054B9C4224
:10D6B00001D1AC68F1E7044B9C42EED1EC68ECE799
:10D6C00014FC000034FC0000F4FB0000002310B543
:10D6D000040003604360836081814366C28103610B
:10D6E00043618361190008225C30FFF7FFF9054BA5
:10D6F00024626362044BA362044BE362044B236322
:10D7000010BDC046B9DE0000E1DE000019DF0000F8
:10D7100045DF000010B5024900F08CF810BDC0468E
:10D7200075D6000070B568254A1E55430E002900C5
:10D73000743100F081F9041E08D000212A00016034
:10D7400046600C30A0606832FFF7D0F9200070BD51
:10D75000836913B50400002B28D18364C364036577
:10D76000134B144A1B6882620193984201D1012332
:10D770008361200000F020F86060200000F01CF8B9
:10D78000A060200000F018F80022E060042160682A
:10D79000FFF79CFF01220921A068FFF797FF0222F3
:10D7A0001221E068FFF792FF0123A36113BDC04679
:10D7B000BCFB000015D70000F8B51C4B07001E6825
:10D7C000B369002B02D13000FFF7C2FF4836B468BE
:10D7D0007368013B04D53368002B07D03668F6E741
:10D7E0000C22A55E002D0DD06834F2E7042138002C
:10D7F000FFF798FF30600028F0D10C2304003B6055
:10D800002000F8BD20000A4B656625606560A560B4
:10D81000E36025616561A561082229005C30FFF79E
:10D8200065F96563A563A564E564E9E7BCFB0000F1
:10D830000100FFFFF7B504000700002601914834FE
:10D84000002C01D13000FEBD6368A5680093009BE9
:10D85000013B009301D52468F2E7AB89012B08D97D
:10D860000E22AB5E013304D029003800019B98479B
:10D8700006436835EBE7EC300068704770B50E0082
:10D880001D000E23C95E96B01400002907DA00239C
:10D890002B60B3891B0611D48023DB000FE06A469E
:10D8A00000F088FB0028F2DBF022019B12021340FB
:10D8B000054A9B185A4253412B60EDE74023002054
:10D8C000236016B070BDC04600E0FFFFF7B502262A
:10D8D0008B8905000C00334206D0230047332360B8
:10D8E000236101236361F7BD01AB6A46FFF7C6FF01
:10D8F00000990700280000F09FF8002808D10C22AA
:10D90000A35E9A05EFD4032293431E43A681E4E766
:10D910000F4BAB628023A28920601343A381009B3D
:10D9200020616361019B002B0DD00E23E15E280076
:10D9300000F052FB002806D00322A38993431A006B
:10D9400001231343A381A0893843A081CBE7C046BC
:10D9500015D7000010B5034B0100186800F06CF8F3
:10D9600010BDC0468C00002082B0002900D101A962
:10D97000101E06D0002B06D013780B601078431EC3
:10D98000984102B0704702204042FAE7C9B28218BB
:10D99000904201D10020704703788B42FBD00130C8
:10D9A000F6E7000070B50500002910D00C1F2368B1
:10D9B000002B00DAE418280000F034FB1D4A13683D
:10D9C000002B05D163601460280000F02CFB70BDB3
:10D9D000A34209D9216860188342F3D118685B68B3
:10D9E00041182160EEE713005A68002A01D0A242D4
:10D9F000F9D919685818A0420BD12068091858188D
:10DA000019608242E0D110685268411819605A606A
:10DA1000DAE7A04202D90C232B60D5E72168601811
:10DA2000824203D1106852684118216062605C60D4
:10DA3000CAE7C0463C1C0020032370B5CD1C9D43A3
:10DA4000083506000C2D1ED20C25A9421DD8300029
:10DA500000F0E8FA254A14682100002919D1244C65
:10DA60002368002B03D1300000F0CAF920602900A0
:10DA7000300000F0C5F9431C2BD10C23300033607B
:10DA800000F0D1FA03E0002DDFDA0C233360002030
:10DA900070BD0B685B1B19D40B2B03D90B60CC1822
:10DAA000256003E04B688C420DD11360300000F01C
:10DAB000BAFA200007220B30231D9043C31AE7D087
:10DAC0005A42E250E4E763600C00EFE70C0049685B
:10DAD000C3E70323C41C9C43A042E1D0211A3000B9
:10DAE00000F08EF9431CDBD1C7E7C0463C1C002088
:10DAF000401C0020F8B507000D001600002905D1D4
:10DB00001100FFF799FF04002000F8BD002A03D19F
:10DB1000FFF748FF3400F7E700F086FA2C00B04228
:10DB2000F2D231003800FFF787FF041EECD0290045
:10DB30003200FEF7BFFF29003800FFF733FFE3E7AD
:10DB4000F0B58E6885B007000C00039201939E42E9
:10DB50003CD890238A89DB001A4234D00325096916
:10DB600023685B1A0293636902985D43EB0F5D19AA
:10DB7000019B6D1001331B18AB4200D91D005305EA
:10DB800032D529003800FFF757FF061E09D10C23B4
:10DB90003B6040230120A28940421343A38105B08A
:10DBA000F0BD029A2169FEF785FFA389144A1A4045
:10DBB00080231343A381029B2661F61826606561CA
:10DBC000019EED1AA560019B9E4200D9019E320084
:10DBD00003992068FEF777FFA36800209B1BA360D2
:10DBE00023689E192660DAE72A003800FFF782FFD3
:10DBF000061EE0D121693800FFF7D4FEC7E7C04612
:10DC00007FFBFFFFF0B59FB0029005938B890F005B
:10DC100016001B0611D50B69002B0ED14021FFF712
:10DC20000BFF38603861002805D10C23029A0138B7
:10DC300013601FB0F0BD40237B61002306AC63611D
:10DC4000203363761033A37635002B78002B01D078
:10DC5000252B46D1AB1B04930CD03200390002981F
:10DC6000FFF76EFF431C00D1AEE06269049B94464F
:10DC7000634463612B78002B00D1A5E001220023CF
:10DC80005242626002A9543252186E1C2360E36053
:10DC9000A3601370A365317805225448FFF776FE20
:10DCA000751C00281FD12268D30604D5532302A96E
:10DCB0005B1820211970130704D5532302A95B18A0
:10DCC0002B21197033782A2B16D0350000210A2019
:10DCD000E3682A786E1C303A092A4ED9002918D0F8
:10DCE00010E00135B1E7414B2268C01A012383409F
:10DCF000134323602E00CEE7059B191D1B68059179
:10DD0000002B01DB099304E05B42E3600223134331
:10DD100023602B782E2B0AD16B782A2B35D1059BCB
:10DD200002351A1D1B680592002B2BDB0793304E22
:10DD3000297803223000FFF729FE002806D040236F
:10DD4000801B834022680135134323602978062213
:10DD500028486E1C2176FFF719FE00283CD0264B80
:10DD6000002B25D10722059B0733934308330593E6
:10DD70006369039A9B18636166E7434301219B181B
:10DD80003500A6E701235B42D0E700230A201A00F2
:10DD90000135636029786E1C3039092903D9002BBD
:10DDA000C5D00792C3E74243012352183500F1E77B
:10DDB00005AB00933A00114B2100029800E000BF30
:10DDC0000390039B0133D3D1BB890B985B0600D42E
:10DDD0002FE7012040422CE705AB00933A00074BA8
:10DDE00021000298FFF736F8EAE7C046C0FB0000C2
:10DDF000C6FB0000CAFB00000000000041DB000081
:10DE0000002370B5064C05000800236000F060F99F
:10DE1000431C03D12368002B00D02B6070BDC0468B
:10DE2000D02F002070B504000D001F2904D916233F
:10DE300003600120404270BD436C002B04D08A0077
:10DE40009B181A68002A08D1200000F031F82A0037
:10DE50000100200000F01AF8EDE70020012AEAD0C6
:10DE6000511C03D1162301302360E4E7002428006D
:10DE70001C6090472000DEE710B5034B01001868D6
:10DE8000FFF7D0FF10BDC0468C000020002370B506
:10DE9000064C050008001100236000F001F9431C46
:10DEA00003D12368002B00D02B6070BDD02F002041
:10DEB00010B500F0E5F810BD70B50C000E25495FF7
:10DEC00000F0BAF8002803DB636D1B18636570BDB2
:10DED000A389024A1340A381F9E7C046FFEFFFFF81
:10DEE000F8B51F008B8905000C001600DB0505D571
:10DEF0000E23C95E0022022300F080F8A389054AA0
:10DF000028001340A38132000E23E15E3B0000F0A5
:10DF10002BF8F8BDFFEFFFFF70B50C000E25495F31
:10DF200000F06CF8A389421C03D1054A1340A38179
:10DF300070BD802252011343A3816065F8E7C0469B
:10DF4000FFEFFFFF10B50E23C95E00F021F810BDF2
:10DF50000B1E04D0FF2A04D98A2303608B3B1800D0
:10DF600070470A700123FAE770B505000800110038
:10DF70000022064C22601A0000F0B8F8431C03D1BE
:10DF80002368002B00D02B6070BDC046D02F00202E
:10DF9000002370B5064C05000800236000F060F80F
:10DFA000431C03D12368002B00D02B6070BDC046FA
:10DFB000D02F0020002370B5064C0500080011008A
:10DFC000236000F055F8431C03D12368002B00D0D8
:10DFD0002B6070BDD02F0020002370B5064C0500CB
:10DFE0000800236000F054F8431C03D12368002B81
:10DFF00000D02B6070BDC046D02F002070B505004A
:10E00000080011000022064C22601A0000F050F8AF
:10E01000431C03D12368002B00D02B6070BDC04689
:10E02000D02F0020704770470B1F1B68181F002B54
:10E0300001DA0B58C018704770B5050008001100D0
:10E040000022064C22601A0000F03AF8431C03D16B
:10E050002368002B00D02B6070BDC046D02F00205D
:10E0600058220120014B40421A607047D02F0020F7
:10E0700058220120014B40421A607047D02F0020E7
:10E0800058220120014B40421A607047D02F0020D7
:10E090005822024B00201A607047C046D02F002043
:10E0A00058220120014B40421A607047D02F0020B7
:10E0B00058220120014B40421A607047D02F0020A7
:10E0C00058220120014B40421A607047D02F002097
:10E0D000044A1368002B00D1034B18181060180075
:10E0E0007047C046441C0020D82F00205822012031
:10E0F000014B40421A607047D02F0020FEE7C04617
:10E10000F8B5C046F8BC08BC9E467047F8B5C04696
:10E11000F8BC08BC9E467047646174610000000052
:10E12000B4E10000EF010000BDE10000E50A0000DD
:10E13000C3E10000E3020000CBE10000990B000006
:10E14000D2E10000D50C0000D7E100000905000075
:10E15000DDE10000F5060000E8E1000053030000E7
:10E16000EDE100002D0F0000F9E100001F020000AA
:10E1700003E20000110A000011E200009506000011
:10E180001EE20000810800002AE20000550600009F
:10E1900072616E646F6D00616C6C006C6173740011
:10E1A00066616C7365007472756500252E31357378
:10E1B0002E2E2E006D616B654C6973740072616E5A
:10E1C0006765006164644C6173740064656C6574B8
:10E1D00065006A6F696E0073706C697400636F70BC
:10E1E0007946726F6D546F0066696E64006A6F697C
:10E1F0006E537472696E677300756E69636F6465E0
:10E20000417400756E69636F6465537472696E67FB
:10E21000006E65774279746541727261790061734D
:10E2200042797465417272617900667265654D6507
:10E230006D6F727900000000A5E20000211400005B
:10E24000AAE200003F140000CBE1000043140000EC
:10E25000B0E2000025140000BAE2000047140000FC
:10E26000C3E200004B140000CDE200004F14000098
:10E27000D6E2000053140000E1E200005714000051
:10E28000EDE2000029140000F6E20000371400005F
:10E2900000E300002D1400000BE300003B1400001D
:10E2A00066696C65006F70656E00636C6F73650006
:10E2B000656E644F6646696C6500726561644C69A1
:10E2C0006E650072656164427974657300726561A0
:10E2D00064496E746F00617070656E644C696E6540
:10E2E00000617070656E6442797465730066696C74
:10E2F0006553697A650073746172744C6973740054
:10E300006E657874496E4C697374007379737465C3
:10E310006D496E666F000000481800005818000034
:10E3200072180000EE180000261900005A190000AB
:10E3300092190000B8190000FC1900003E1A0000F4
:10E34000921A0000D61A0000381B0000801B000043
:10E35000A61B0000DE1B0000241C00004A1C00005D
:10E36000781C0000A61C0000B23300006C1D0000E9
:10E370003E1E0000B41E0000201F00006C1F0000A5
:10E380008C1F0000AE1F0000062100004A21000083
:10E39000C2210000F02100002222000070220000B3
:10E3A000D8220000402300009C230000FA23000034
:10E3B0006C240000DE2400003A25000094250000B3
:10E3C000D42500001A26000060260000A8260000C0
:10E3D000FC260000502700008E27000014280000B3
:10E3E0004A28000092280000DA28000022290000B4
:10E3F0005C290000AC290000F4290000562B000025
:10E40000781C0000DE1B00005C2A00004818000099
:10E41000922A0000BE2A0000F42A0000202B0000EF
:10E42000481800004818000048180000481800006C
:10E43000D22B0000142C00005A2C0000AA2C000043
:10E44000D62C00004E2D0000D62D0000042E00001A
:10E450004818000048180000282E0000582E000020
:10E46000882E0000BE2E0000E82E00001E2F0000A7
:10E47000482F0000702F0000982F0000C82F0000C8
:10E48000F82F0000223000004C3000007C300000EB
:10E49000A630000048180000481800004818000086
:10E4A0004818000048180000D63000000231000073
:10E4B0002E3100005A31000098310000CE310000AA
:10E4C000043200003A320000703200009C3200003A
:10E4D000C8320000FE320000481800004818000052
:10E4E00048180000481800004818000048180000AC
:10E4F000481800004818000048180000481800009C
:10E5000048180000481800002A3300002A33000091
:10E5100052340000883400005B2564206974656D06
:10E52000206C6973745D00282564206279746573BA
:10E530002900286F626A65637420747970653A20D7
:10E5400025642900537461636B20756E646572667F
:10E550006C6F7700626F6F6C65616E006E756D62D7
:10E56000657200737472696E67006C69737400621F
:10E570007974652061727261790000000700000003
:10E580000300000015E60000B13500001DE60000A4
:10E590006136000026E60000E93A00002FE60000A0
:10E5A000B535000038E60000ED3A000040E6000016
:10E5B0001538000049E60000D138000057E6000099
:10E5C0004537000062E60000753C00006DE6000083
:10E5D0002938000078E60000E93B000084E60000EE
:10E5E000F136000090E60000453C00001C000000F1
:10E5F000010000000200000004000000050000000F
:10E6000006000000100000001100000043616C6C67
:10E61000696F706500686173546F6E6500706C613E
:10E6200079546F6E6500686173536572766F00731D
:10E630006574536572766F00646163496E69740036
:10E64000646163577269746500736F6674577269A9
:10E65000746542797465007371756172655761768E
:10E660006500736574557365724C454400616E6155
:10E670006C6F675265616400616E616C6F675772A1
:10E68000697465006469676974616C5265616400EE
:10E690006469676974616C577269746500474320E7
:10E6A000746F6F6B2025642075736563733B206600
:10E6B00072656520256420776F726473003C496E33
:10E6C00074656765723E003C4C6973743E003C4F54
:10E6D000626A6563743E003C42797465417272619E
:10E6E000793E000D0A564D2050616E69633A20252F
:10E6F000730D0A006D6973630000000041E70000BC
:10E70000D54600004AE70000A147000052E700009C
:10E710006547000056E70000B517000065E70000F8
:10E72000294600006DE70000CF45000077E70000B4
:10E730006545000083E70000674400006E756C6C5F
:10E7400000686578546F496E740072657363616C1C
:10E75000650073696E0062726F6164636173745403
:10E760006F494445006A736F6E476574006A736F42
:10E770006E436F756E74006A736F6E56616C75656B
:10E780004174006A736F6E4B65794174000000003C
:10E7900084E80000114800008CE8000015480000E3
:10E7A00096E80000334800009FE800003D48000064
:10E7B000AAE8000047480000B6E800005148000001
:10E7C000C4E800005B480000CCE800006548000099
:10E7D000D2E800006F480000E7E800007948000038
:10E7E000FCE800008348000008E900008D480000B4
:10E7F00018E900009748000024E90000A148000043
:10E8000031E90000AB4800003AE90000B5480000DB
:10E8100042E90000BF48000050E90000C94800007C
:10E8200061E90000D348000074E90000DD48000001
:10E8300082E90000E748000091E90000F14800008B
:10E84000A4E90000FB480000BAE900000549000007
:10E85000C6E900000F490000D6E900001949000090
:10E86000E5E9000023490000F3E900002D4900001C
:10E87000FBE900001F48000003EA000029480000EF
:10E880006E657400686173576946690073746172DC
:10E8900074576946690073746F70576946690077E9
:10E8A000696669537461747573006D794950416488
:10E8B0006472657373007374617274535349447363
:10E8C00063616E0067657453534944006D794D412F
:10E8D000430068747470536572766572476574524C
:10E8E00065717565737400726573706F6E64546FD3
:10E8F00048747470526571756573740068747470CF
:10E90000436F6E6E65637400687474704973436F0F
:10E910006E6E6563746564006874747052657175B9
:10E920006573740068747470526573706F6E73658C
:10E930000075647053746172740075647053746F01
:10E94000700075647053656E645061636B6574002C
:10E95000756470526563656976655061636B657453
:10E960000075647052656D6F7465495041646472DE
:10E970006573730075647052656D6F7465506F7266
:10E980007400776562536F636B657453746172745E
:10E9900000776562536F636B65744C617374457681
:10E9A000656E7400776562536F636B657453656E53
:10E9B00064546F436C69656E74004D515454436FD9
:10E9C0006E6E656374004D5154544973436F6E6E9F
:10E9D0006563746564004D515454446973636F6E8C
:10E9E0006E656374004D5154544C61737445766583
:10E9F0006E74004D515454507562004D515454532F
:10EA00007562004D515454556E737562000D0E0FB2
:10EA100004050C0B0A06070809000000000008089E
:10EA20000800080A4A4000000A5FEA5FEA0ED92E91
:10EA3000D36E19324489330C924C924D0808000071
:10EA40000004880808040804848488000A448A4072
:10EA500000048EC480000000048800000EC0000086
:10EA60000000080001224488100C9252524C048C81
:10EA700084848E1C824C901E1EC244924C06CA5244
:10EA80005FE21FF01EC13E02448ED12E1FE2448879
:10EA9000100ED12ED12E0ED12EC4880008000800F1
:10EAA00000048004880244880482000EC00EC0085E
:10EAB000048244880ED126C0040ED135B36C0C926A
:10EAC0005ED2521C925C925C0ED010100E1C9252C0
:10EAD000525C1ED01C901E1ED01C90100ED01371C4
:10EAE0002E12525ED2521C8808081C1FE242524C61
:10EAF0001254981492101010101E113B75B1311160
:10EB00003935B3710C9252524C1C925C90100C929D
:10EB1000524C861C925C92510ED00C825C1FE48495
:10EB20008484125252524C1131312A44113135BB76
:10EB30007112524C9252112A4484841EC488101EB1
:10EB40000EC808080E10080482410EC242424E044C
:10EB50008A400000000000001F0804800000000E32
:10EB6000D2524F10101C925C000ED0100E02424E7A
:10EB7000D24E0C925C900E06C81C88080ED24EC273
:10EB80004C10101C92520800080808024002424C27
:10EB900010149814920808080806001B75B131007B
:10EBA0001C925252000C92524C001C925C90000E2F
:10EBB000D24EC2000ED010100006C8049808080EED
:10EBC000C807001252524F0011312A44001131354A
:10EBD000BB00124C8C9200112A4498001EC4881E5F
:10EBE00006C48C8486080808080818080C881800D1
:10EBF000000C836000000000010000000200000023
:10EC000003000000040000000500000006000000F2
:10EC10000700000008000000090000000A000000D2
:10EC20000B0000000C0000000D0000000E000000B2
:10EC30000F0000001000000012000000140000008F
:10EC400016000000180000001A0000001C00000060
:10EC50001E0000002000000023000000260000002D
:10EC6000290000002C0000002F00000032000000EE
:10EC7000360000003A0000003E00000042000000A4
:10EC8000460000004B00000050000000550000004E
:10EC90005A00000061000000680000006F000000E2
:10ECA000760000007D000000840000008B00000062
:10ECB0009200000099000000A0000000A7000000E2
:10ECC000AE000000B5000000BC000000C300000062
:10ECD000CA000000D1000000D8000000DF000000E2
:10ECE000E6000000ED000000F4000000FB00000062
:10ECF000FF0000004CED00005149000057ED0000FE
:10ED0000254F000061ED0000314B00006EED00006A
:10ED1000954C000075ED0000E54C00007EED000014
:10ED2000354D00008AED00002D4C00009BED0000E9
:10ED3000BD4B0000ABED0000254E0000B8ED00001B
:10ED4000894B0000646973706C6179006C69676855
:10ED5000744C6576656C006D62446973706C6179A2
:10ED6000006D62446973706C61794F6666006D6214
:10ED7000506C6F74006D62556E706C6F74006D62D4
:10ED8000447261775368617065006D6253686170A9
:10ED900065466F724C6574746572006D62456E6194
:10EDA000626C65446973706C6179006E656F50695F
:10EDB00078656C53656E64006E656F506978656C3C
:10EDC00053657450696E004E6F7420656E6F756781
:10EDD0006820726F6F6D206576656E206166746560
:10EDE0007220636F6D70616374696F6E00436F6D45
:10EDF00070616374656420466C61736820636F643E
:10EE0000652073746F72650A256420627974657376
:10EE1000207573656420282564252529206F6620C8
:10EE2000256400426164207265636F726420666FBE
:10EE3000756E6420647572696E6720696E697469A5
:10EE4000616C697A6174696F6E00256420256420A5
:10EE500025642028256420776F7264732900256457
:10EE6000207265636F7264732C20256420776F7243
:10EE700064732C206D617849442025642C20636FD5
:10EE80006D70616374696F6E206379636C65732064
:10EE9000256400526573746F726564202564207365
:10EEA0006372697074730053746172746564007284
:10EEB0006164696F000000004DEF000045590000DB
:10EEC0005AEF0000415C00006AEF0000C15B0000E7
:10EED00078EF0000D55D000083EF00005D59000071
:10EEE00093EF0000D9590000A7EF0000C1590000BE
:10EEF000B6EF0000855F0000C2EF0000035F000076
:10EF0000CBEF0000A75E0000D6EF0000215E0000FE
:10EF1000E1EF00005D5E0000EAEF0000915E00009E
:10EF2000F3EF00006D59000002F00000A15900004D
:10EF30000BF000007D59000025303878006E6F6EB0
:10EF400065006F746865720070616972006469734E
:10EF500061626C65526164696F006D6573736167AE
:10EF6000655265636569766564007061636B65749D
:10EF700052656365697665007061636B657453659E
:10EF80006E64007265636569766564496E74656771
:10EF900065720072656365697665644D657373615A
:10EFA0006765547970650072656365697665645359
:10EFB0007472696E670073656E64496E7465676527
:10EFC000720073656E64506169720073656E64539C
:10EFD0007472696E67007365744368616E6E656C08
:10EFE0000073657447726F757000736574506F7746
:10EFF0006572007369676E616C537472656E6774D5
:10F0000068006465766963654944006C6173744D9A
:10F01000657373616765494400556E6B6E6F776EFB
:10F02000207072696D6974697665205B25733A2575
:10F03000735D000000000000963007772C610EEE33
:10F04000BA51099919C46D078FF46A7035A563E93F
:10F05000A395649E3288DB0EA4B8DC791EE9D5E066
:10F0600088D9D2972B4CB609BD7CB17E072DB8E765
:10F07000911DBF906410B71DF220B06A4871B9F3BA
:10F08000DE41BE847DD4DA1AEBE4DD6D51B5D4F4F3
:10F09000C785D38356986C13C0A86B647AF962FD58
:10F0A000ECC9658A4F5C0114D96C0663633D0FFAA5
:10F0B000F50D088DC8206E3B5E10694CE44160D5AB
:10F0C000727167A2D1E4033C47D4044BFD850DD295
:10F0D0006BB50AA5FAA8B5356C98B242D6C9BBDBA8
:10F0E00040F9BCACE36CD832755CDF45CF0DD6DCA3
:10F0F000593DD1ABAC30D9263A00DE518051D7C84A
:10F100001661D0BFB5F4B42123C4B3569995BACFD4
:10F110000FA5BDB89EB802280888055FB2D90CC6F5
:10F1200024E90BB1877C6F2F114C6858AB1D61C16E
:10F130003D2D66B69041DC760671DB01BC20D2988D
:10F140002A10D5EF8985B1711FB5B606A5E4BF9F1A
:10F1500033D4B8E8A2C9077834F9000F8EA809960D
:10F1600018980EE1BB0D6A7F2D3D6D08976C649178
:10F17000015C63E6F4516B6B62616C1CD830658591
:10F180004E0062F2ED95066C7BA5011BC1F408826E
:10F1900057C40FF5C6D9B06550E9B712EAB8BE8BAF
:10F1A0007C88B9FCDF1DDD62492DDA15F37CD38C38
:10F1B000654CD4FB5861B24DCE51B53A7400BCA336
:10F1C000E230BBD441A5DF4AD795D83D6DC4D1A468
:10F1D000FBF4D6D36AE96943FCD96E34468867AD3F
:10F1E000D0B860DA732D0444E51D03335F4C0AAADE
:10F1F000C97C0DDD3C710550AA41022710100BBEE1
:10F2000086200CC925B56857B3856F2009D466B927
:10F210009FE461CE0EF9DE5E98C9D9292298D0B05C
:10F22000B4A8D7C7173DB359810DB42E3B5CBDB709
:10F23000AD6CBAC02083B8EDB6B3BF9A0CE2B6038A
:10F240009AD2B1743947D5EAAF77D29D1526DB043F
:10F250008316DC73120B63E3843B64943E6A6D0D8A
:10F26000A85A6A7A0BCF0EE49DFF099327AE000AD5
:10F27000B19E077D44930FF0D2A3088768F2011E68
:10F28000FEC206695D5762F7CB67658071366C19FF
:10F29000E7066B6E761BD4FEE02BD3895A7ADA1020
:10F2A000CC4ADD676FDFB9F9F9EFBE8E43BEB71701
:10F2B000D58EB060E8A3D6D67E93D1A1C4C2D8388B
:10F2C00052F2DF4FF167BBD16757BCA6DD06B53FF1
:10F2D0004B36B248DA2B0DD84C1B0AAFF64A033630
:10F2E000607A0441C3EF60DF55DF67A8EF8E6E31AF
:10F2F00079BE69468CB361CB1A8366BCA0D26F25F8
:10F3000036E2685295770CCC03470BBBB916022244
:10F310002F260555BE3BBAC5280BBDB2925AB42B59
:10F32000046AB35CA7FFD7C231CFD0B58B9ED92C6E
:10F330001DAEDE5BB0C2649B26F263EC9CA36A75D3
:10F340000A936D02A906099C3F360EEB856707728A
:10F3500013570005824ABF95147AB8E2AE2BB17BF1
:10F36000381BB60C9B8ED2920DBED5E5B7EFDC7C78
:10F3700021DFDB0BD4D2D38642E2D4F1F8B3DD68CF
:10F380006E83DA1FCD16BE815B26B9F6E177B06FCA
:10F390007747B718E65A0888706A0FFFCA3B0666B7
:10F3A0005C0B0111FF9E658F69AE62F8D3FF6B6144
:10F3B00045CF6C1678E20AA0EED20DD75483044EE6
:10F3C000C2B30339612667A7F71660D04D47694974
:10F3D000DB776E3E4A6AD1AEDC5AD6D9660BDF4087
:10F3E000F03BD83753AEBCA9C59EBBDE7FCFB2473A
:10F3F000E9FFB5301CF2BDBD8AC2BACA3093B3531F
:10F40000A6A3B4240536D0BA9306D7CD2957DE5427
:10F41000BF67D9232E7A66B3B84A61C4021B685D00
:10F42000942B6F2A37BE0BB4A18E0CC31BDF055A79
:10F430008DEF022D416C6C207461736B73207374BB
:10F440006F70706564007631373000202573202599
:10F4500073004D656D6F727920636C6561726564D0
:10F46000004E6F2066726565207461736B20656E57
:10F470007472696573000000F8F40000597A0000A6
:10F4800005F50000C977000011F50000997700002C
:10F4900017F50000A97700001DF50000B9770000FE
:10F4A00023F500004975000039F50000417900009E
:10F4B00047F50000A971000051F50000CD7900006A
:10F4C00059F500008975000062F50000D172000056
:10F4D00073F50000B17300007FF500008572000035
:10F4E00088F500000573000090F500009D74000091
:10F4F00073656E736F727300616363656C657261CF
:10F5000074696F6E0074656D706572617475726593
:10F510000074696C74580074696C74590074696C77
:10F52000745A00736574416363656C65726F6D65D1
:10F5300074657252616E6765006D61676E657469AE
:10F54000634669656C6400746F75636852656164D5
:10F55000006932635265616400693263577269748D
:10F560006500693263536574436C6F636B537065F8
:10F5700065640073706945786368616E67650073E0
:10F580007069536574757000726561644448540015
:10F590006D6963726F70686F6E650000A5E20000B0
:10F5A000657B0000AAE20000117B0000D3F500009B
:10F5B000A97C0000CDE200002D7B0000D8F5000002
:10F5C000317C0000DEF50000897B00007365726904
:10F5D000616C0072656164007772697465007772AE
:10F5E00069746542797465730000000068F6000074
:10F5F000D97C000076F60000E97C000083F600006C
:10F60000DD7C00008CF60000ED7C000096F600002A
:10F61000F17C00009FF60000F57C0000A4F60000DD
:10F62000F97C0000A9F60000FD7C0000B5F60000A2
:10F63000017D0000BCF60000057D0000C5F600005D
:10F64000097D0000CAF600000D7D0000D5F600001F
:10F65000117D0000DFF60000E17C0000E9F600000B
:10F66000E57C000074667400656E61626C654469D7
:10F6700073706C6179007365744261636B6C696768
:10F6800068740067657457696474680067657448D6
:10F69000656967687400736574506978656C006C9F
:10F6A000696E65007265637400726F756E6465647F
:10F6B0005265637400636972636C6500747269619A
:10F6C0006E676C65007465787400746674546F7549
:10F6D0006368656400746674546F75636858007479
:10F6E0006674546F7563685900746674546F7563FB
:10F6F000685072657373757265007661727300008D
:10F7000020F70000A18100002AF70000818100009D
:10F7100033F700005D8100003FF70000EB80000040
:10F72000766172457869737473007661724E616DAB
:10F730006564007365745661724E616D6564007630
:10F7400061724E616D65466F72496E6465780057EF
:10F75000656C636F6D6520746F204D6963726F42D5
:10F760006C6F636B732100705F73706920213D20A3
:10F770004E554C4C002F686F6D652F6769742F2EA6
:10F78000706C6174666F726D696F2F7061636B610D
:10F790006765732F6672616D65776F726B2D61722D
:10F7A0006475696E6F6E6F726469636E7266352F11
:10F7B0006C69627261726965732F5350492F53509F
:10F7C000492E63707000535049436C6173733A3A29
:10F7D000535049436C617373284E52465F535049EE
:10F7E0005F547970652A2C2075696E74385F742CAB
:10F7F0002075696E74385F742C2075696E74385F7B
:10F800007429000000000000000000007583000063
:10F810003183000057830000618300006B83000088
:10F8200055830000000000000100000002000000FD
:10F8300016000000040000000500000006000000A3
:10F840000700000008000000090000000A00000096
:10F850000B0000000C0000000D0000000E00000076
:10F860000F0000001A0000001B0000001400000040
:10F87000130000001100000017000000100000003D
:10F880001C0000001D0000001E000000120000000F
:10F89000150000000300000018000000190000001F
:10F8A000000000000000000061870000958F00004C
:10F8B000E1870000F5870000EB8700005D8700000E
:10F8C00051870000018800007D8700004D870000FF
:10F8D000000000000000304300000000000030C3C2
:10F8E0007371727400000000FB21F93FFB21094095
:10F8F0007CD91240FB2119407A6A1F407CD92240F2
:10F90000BBFD2540FB2129403A462C407A6A2F4016
:10F910005C4731407CD932409C6B3440BBFD354064
:10F92000DB8F3740FB2139401BB43A403A463C401C
:10F930005AD83D407A6A3F404C7E40405C47414047
:10F940006C1042407CD942408CA243409C6B4440A6
:10F95000AC344540BBFD4540CBC64640DB8F4740FD
:10F96000EB584840FB21494083F9A200444E6E0009
:10F97000FC291500D1572700DD34F50062DBC000FB
:10F980003C999500419043006351FE00BBDEAB0003
:10F99000B761C5003A6E2400D24D42004906E0002E
:10F9A00009EA2E001C92D100EB1DFE0029B11C00BB
:10F9B000E83EA700F535820044BB2E009CE9840098
:10F9C000B4267000417E5F00D69139005383390020
:10F9D0009CF439008B5F840028F9BD00F81F3B00C0
:10F9E000DEFF97000F980500112FEF000A5A8B00D9
:10F9F0006D1F6D00CF7E360009CB2700464FB70044
:10FA00009E663F002DEA5F00BA277500E5EBC70050
:10FA10003D7BF100F739070092528A00FB6BEA0048
:10FA20001FB15F00085D8D00300356007BFC46006F
:10FA3000F0AB6B0020BCCF0036F49A00E3A91D00A8
:10FA40005E619100081BE60085996500A0145F00C7
:10FA50008D40680080D8FF0027734D0006063100F6
:10FA6000CA561500C9A873007BE260006B8CC00009
:10FA700000000040FB21F93F000000002D44743ECF
:10FA8000000000809846F83C0000006051CC783BB4
:10FA900000000080831BF0390000004020257A38E8
:10FAA000000000802282E336000000001DF369356B
:10FAB0000200000003000000040000000600000037
:10FAC00020AC0000CAAB0000CAAB0000F8AC0000DC
:10FAD000C6AB0000C6AB0000EEAC0000F8AC000006
:10FAE000C6AB0000EEAC0000C6AB0000F8AC0000F6
:10FAF000FCAC0000FCAC0000FCAC000004AD00005D
:10FB0000FCB600006EB50000B2B5000016B50000EE
:10FB1000B2B50000A2B60000B2B5000016B50000F4
:10FB20006EB500006EB50000A2B6000016B500006C
:10FB30000EB500000EB500000EB50000B0B6000016
:10FB400024BE000026BD000026BD000044C0000009
:10FB500020BD000020BD00002CC0000044C00000FB
:10FB600020BD00002CC0000020BD000044C00000EB
:10FB70003AC000003AC000003AC0000048C000008F
:10FB80002C2066756E6374696F6E3A200061737322
:10FB9000657274696F6E2022257322206661696C1C
:10FBA00065643A2066696C6520222573222C206CDE
:10FBB000696E65202564257325730A009000002076
:10FBC000232D302B2000686C4C0065666745464746
:10FBD00000303132333435363738394142434445C9
:10FBE0004600303132333435363738396162636438
:10FBF000656600000000000000000000000000003A
:10FC000000000000000000000000000000000000F4
:10FC100000000000000000000000000000000000E4
:10FC200000000000000000000000000000000000D4
:10FC300000000000000000000000000000000000C4
:10FC400000000000000000000000000000000000B4
:10FC500000000000504F5349580000202020202071
:10FC6000202020202828282828202020202020206C
:10FC7000202020202020202020202088101010105C
:10FC800010101010101010101010100404040404B0
:10FC900004040404041010101010101041414141DC
:10FCA00041410101010101010101010101010101C4
:10FCB00001010101010110101010101042424242D6
:10FCC0004242020202020202020202020202020294
:10FCD00002020202020210101010200000000000B8
:10FCE0000000000000000000000000000000000014
:10FCF0000000000000000000000000000000000004
:10FD000000000000000000000000000000000000F3
:10FD100000000000000000000000000000000000E3
:10FD200000000000000000000000000000000000D3
:10FD300000000000000000000000000000000000C3
:10FD400000000000000000000000000000000000B3
:10FD500000000000000000000000000000000000A3
:08FD6000A803FF7F0100000071
:10FD6800FFFFFFFFE803000001000000E803DC05D7
:10FD7800DC05DC05DC050000FFFFFFFFFFFFFFFFE0
:10FD88001800000019FCFFFFFFFFFFFF0200000042
:10FD980040420F00FF01FF000024F40002000000B1
:10FDA80003000000FFFFFFFF00000000010000004B
:10FDB8000000020001000000FFFFFFFF000000003C
:10FDC800020000000000040002000000FFFFFFFF27
:10FDD800000000000300000000000800030000000D
:10FDE8000A00000008000000010000009000002048
:10FDF8000000000014FC000034FC0000F4FB0000CC
:10FE080000000000000000000000000000000000EA
:10FE180000000000000000000000000000000000DA
:10FE280000000000000000000000000000000000CA
:10FE380000000000000000000000000000000000BA
:10FE480000000000000000000000000000000000AA
:10FE58004300000000000000000000000000000057
:10FE6800000000000000000000000000000000008A
:10FE78004300000000000000000000000000000037
:10FE8800000000000000000000000000000000006A
:10FE98004300000000000000000000000000000017
:10FEA800000000000000000000000000000000004A
:10FEB80043000000000000000000000000000000F7
:10FEC800000000000000000000000000000000002A
:10FED80043000000000000000000000000000000D7
:10FEE800000000000000000000000000000000000A
:10FEF80043000000000000000000000000000000B7
:10FF080000000000000000000000000000000000E9
:10FF18004300000000000000000000000000000096
:10FF280000000000000000000000000000000000C9
:10FF380051DF000069D90000000000005AFC0000F1
:10FF4800B2E10000F3E60000F3E60000F3E600008B
:10FF5800F3E60000F3E60000F3E60000F3E6000035
:10FF6800F3E60000F3E60000FFFFFFFFFFFFFFFFDF
:10FF7800FFFFFFFFFFFF0000010041534349490015
:10FF88000000000000000000000000000000000069
:10FF980000000000000000000000415343494900F0
:10FFA8000000000000000000000000000000000049
:10FFB800000000000000000000000000E900000050
:10FFC8000183000055860000AD8A0000C1000000D2
:04000003000086F182
:00000001FF
